:020000040000FA
:1000000000040020990900002D0600007909000075
:1000100037060000410600004B060000000000000B
:10002000000000000000000000000000BD0900000A
:1000300055060000000000005F0600006906000091
:10004000730600007D060000870600009106000090
:100050009B060000A5060000AF060000B9060000E0
:10006000C3060000CD060000D7060000E106000030
:10007000EB060000F5060000FF060000090700007F
:10008000130700001D0700002707000031070000CC
:100090003B070000450700004F070000590700001C
:1000A000630700006D07000077070000810700006C
:1000B0008B070000950700009F070000A9070000BC
:1000C000B3070000BD070000C7070000D10700000C
:1000D000DB070000E5070000EF070000F90700005C
:1000E000030800000D0800001708000021080000A8
:1000F0002B080000350800003F08000049080000F8
:10010000530800001FB500F003F88DE80F001FBD75
:1001100000F038BC70B50B46010B184400F6FF70B8
:10012000040B4FF080500022090303692403406947
:1001300043431D1B104600F0E9F929462046BDE85F
:10014000704000F0E3B9F0B54FF6FF734FF4B475AB
:100150001A466E1E12E0A94201D3344600E00C4656
:10016000B1EB040130F8027B641E3B441A44F9D120
:100170009CB204EB134394B204EB12420029EAD17F
:1001800098B200EB134002EB124140EA0140F0BD8F
:10019000C34992B00446D1E90001CDE91001FF2224
:1001A0004021684600F094FB94E80F008DE80F00B2
:1001B000684610A902E004C841F8042D8842FAD12B
:1001C00010216846FFF7BFFF1090AA208DF8440069
:1001D00000F0FAF800F0DDF84FF01024A0691022CA
:1001E0006946803000F0DEF8A069082210A900F00E
:1001F000D9F800F0C2F870B504460068A94D072888
:1002000069D2DFE800F033041929561E2500D4E92D
:10021000026564682946304600F0FDF82A4621460A
:10022000304600F0BFF8AA002146304600F024FB1B
:10023000002800D0032070BD00F0D6FB4FF48050A2
:1002400007E0201D00F0C6F80028F4D100F0CCFB38
:1002500060682860002070BD241D94E807009200AB
:1002600000F00AFB0028F6D00E2070BD00F0BEF8AA
:100270000028FAD1D4E9010100EB81034FF080504E
:10028000026945696A43934209D84FF010225369C5
:1002900003EB81030169406941438B4201D9092085
:1002A00070BD5069401C01D10F2070BD2046FFF782
:1002B0006FFF00F09BF80028F7D1201D00F08AF8AE
:1002C0000028F2D160680028F0D100F07DF800F03D
:1002D00060F800F052F8072070BD10B50C461828E1
:1002E00002D00120086010BD2068FFF784FF206065
:1002F00010BD4FF01024A069401C05D0A569A66967
:1003000080353079AA2808D06069401C2DD06069FA
:100310000068401C29D060692CE010212846FFF7B6
:1003200012FF316881421CD1A16901F18002C03104
:1003300005E030B108CA51F8040D984201D10120FE
:1003400000E000208A42F4D158B1286810B1042896
:1003500003D0FEE7284600F070F85249686808604C
:1003600008E000F016F800F008F84FF4805001683B
:10037000491C01D000F012FBFEE7BFF34F8F4A4843
:1003800001684A4A01F4E06111430160BFF34F8FF5
:10039000FEE74FF010208169491C02D0806900F00F
:1003A0008CB870472DE9F04117460D4606460024EB
:1003B00006E03046296800F093F8641C2D1D361DB8
:1003C000BC42F6D3BDE8F0814FF0102080694FF4B5
:1003D00080519FE64FF080510A69496900684A439D
:1003E000824201D810207047002070474FF08050A3
:1003F0000169406941434FF01020826902F5805243
:10040000914201D2092070478069401C01D0002030
:1004100070470420704770B50C4605464FF480665F
:1004200008E0284600F049F8B44205D3A4F58064FA
:1004300005F58055002CF4D170BD4168044609B122
:10044000012600E000264FF010256869A26892009E
:1004500000F012FAF8B1A06881006869FFF75AFE4F
:10046000BEB16E694FF08050A56864680169426949
:100470005143A1420DD9016940694143A94208D9BC
:1004800029463046FFF7C7FF2A4621463046FFF788
:1004900089FFFFF772FFFFF797FFFFF77AFFF8E793
:1004A0000C0A0000000000200CED00E00400FA053A
:1004B000144801680029FCD07047134A02211160DA
:1004C00010490B68002BFCD00F4B1B1D18600868EF
:1004D0000028FCD00020106008680028FCD070477D
:1004E000094B10B501221A60064A1468002CFCD092
:1004F000016010680028FCD00020186010680028F7
:10050000FCD010BD00E4014004E5014070B50C468C
:10051000054600F073F810B900F07EF828B12146C6
:100520002846BDE8704000F007B821462846BDE8DF
:10053000704000F037B800007FB5002200920192B1
:10054000029203920A0B000B6946012302440AE05F
:10055000440900F01F0651F8245003FA06F635430B
:1005600041F82450401C8242F2D80D490868009A94
:1005700010430860081D0168019A1143016000F0F2
:100580003DF800280AD0064910310868029A104345
:100590000860091D0868039A104308607FBD0000C9
:1005A0000006004030B50F4C002200BF04EB0213E0
:1005B000D3F800582DB9D3F8045815B9D3F8085812
:1005C0001DB1521C082AF1D330BD082AFCD204EB1D
:1005D0000212C2F80008C3F804180220C3F8080881
:1005E00030BD000000E001404FF08050D0F83001F5
:1005F000082801D000207047012070474FF080503C
:10060000D0F83011062905D0D0F83001401C01D0B7
:1006100000207047012070474FF08050D0F8300123
:100620000A2801D0002070470120704708208F4918
:1006300009680958084710208C4909680958084773
:1006400014208A4909680958084718208749096809
:100650000958084730208549096809580847382053
:1006600082490968095808473C20804909680958A7
:10067000084740207D4909680958084744207B49BC
:1006800009680958084748207849096809580847FF
:100690004C20764909680958084750207349096871
:1006A00009580847542071490968095808475820D3
:1006B0006E490968095808475C206C49096809585F
:1006C0000847602069490968095808476420674954
:1006D00009680958084768206449096809580847A3
:1006E0006C20624909680958084770205F49096809
:1006F0000958084774205D49096809580847782057
:100700005A490968095808477C2058490968095816
:1007100008478020554909680958084784205349EB
:100720000968095808478820504909680958084746
:100730008C204E4909680958084790204B490968A0
:1007400009580847942049490968095808479820DA
:1007500046490968095808479C20444909680958CE
:100760000847A0204149096809580847A4203F4983
:10077000096809580847A8203C49096809580847EA
:10078000AC203A49096809580847B0203749096838
:1007900009580847B4203549096809580847B8205E
:1007A0003249096809580847BC2030490968095886
:1007B0000847C0202D49096809580847C4202B491B
:1007C000096809580847C82028490968095808478E
:1007D000CC202649096809580847D02023490968D0
:1007E00009580847D4202149096809580847D820E2
:1007F0001E49096809580847DC201C49096809583E
:100800000847E0201949096809580847E4201749B2
:10081000096809580847E820144909680958084731
:10082000EC201249096809580847F0200F49096867
:1008300009580847F4200D49096809580847F82065
:100840000A49096809580847FC20084909680958F5
:1008500008475FF480700549096809580847000097
:1008600003480449024A034B70470000000000207F
:10087000180A0000180A000040EA010310B59B079F
:100880000FD1042A0DD310C808C9121F9C42F8D0FA
:1008900020BA19BA884201D9012010BD4FF0FF30AB
:1008A00010BD1AB1D30703D0521C07E0002010BDC1
:1008B00010F8013B11F8014B1B1B07D110F8013B4D
:1008C00011F8014B1B1B01D1921EF1D1184610BD2E
:1008D00002F0FF0343EA032242EA024200F005B8B5
:1008E0007047704770474FF000020429C0F0128033
:1008F00010F0030C00F01B80CCF1040CBCF1020FD3
:1009000018BF00F8012BA8BF20F8022BA1EB0C01A7
:1009100000F00DB85FEAC17C24BF00F8012B00F89D
:10092000012B48BF00F8012B70474FF0000200B5C3
:10093000134694469646203922BFA0E80C50A0E802
:100940000C50B1F12001BFF4F7AF090728BFA0E8B0
:100950000C5048BF0CC05DF804EB890028BF40F87C
:10096000042B08BF704748BF20F8022B11F0804FBE
:1009700018BF00F8012B7047014B1B68DB68184754
:100980000000002009480A497047FFF7FBFFFFF706
:10099000B9FB00BD20BFFDE7064B1847064A1060B3
:1009A000016881F30888406800470000180A0000C9
:1009B000180A0000F3020000000000201EF0040FDF
:1009C0000CBFEFF30881EFF30981886902380078E2
:1009D000182803D100E00000074A1047074A1268B0
:1009E0002C3212681047000000B5054B1B68054A01
:1009F0009B58984700BD0000DB020000000000206B
:100A0000080A0000040000000010000000000000C0
:080A100000FFFFFF0090D0037E
:02000004000EEC
:10C0000018AB0020C9C30E00D1C30E00D3C30E006D
:10C01000D5C30E00D7C30E00D9C30E000000000028
:10C02000000000000000000000000000DBC30E0064
:10C03000DDC30E0000000000DFC30E00E1C30E00F0
:10C040005DDA0E00E3C30E00B9DC0E00E3C30E00A0
:10C05000E3C30E00E3C30E00E3C30E00E3C30E0010
:10C06000E3C30E00E3C30E00E3C30E00E3C30E0000
:10C07000E3C30E00E3C30E00E3C30E00E3C30E00F0
:10C0800075DE0E006DDA0E00E3C30E00E3C30E0092
:10C09000E3C30E00E3C30E00E3C30E00E3C30E00D0
:10C0A000E3C30E00E3C30E00E3C30E00E3C30E00C0
:10C0B000E3C30E00E3C30E00000000000000000018
:10C0C000E3C30E00E3C30E00E3C30E00E3C30E00A0
:10C0D000E3C30E00E3C30E00E3C30E000DDD0E004C
:10C0E000E3C30E00E3C30E00B1C50E000000000064
:10C0F00000000000E3C30E0000000000E3C30E00D8
:10C10000000000000000000000000000000000002F
:10C11000000000000000000000000000000000001F
:10C12000000000000000000000000000000000000F
:10C1300000000000000000000000000000000000FF
:10C1400000000000000000000000000000000000EF
:10C1500000000000000000000000000000000000DF
:10C1600000000000000000000000000000000000CF
:10C1700000000000000000000000000000000000BF
:10C1800000000000000000000000000000000000AF
:10C19000000000000000000000000000000000009F
:10C1A000000000000000000000000000000000008F
:10C1B000000000000000000000000000000000007F
:10C1C000000000000000000000000000000000006F
:10C1D000000000000000000000000000000000005F
:10C1E000000000000000000000000000000000004F
:10C1F000000000000000000000000000000000003F
:10C20000DFF80CD000F096F9004800472D1E0F0013
:10C2100018AB002080F308888E46104730B450E8F1
:10C22000012F93B2C48923448489A34228BF1B1BD6
:10C230000489A34202BFBFF32F8F002007E0C3EAA7
:10C24000020340E80134002CE9D14FF001000A60FC
:10C2500030BC704750E8012FC2EA024240E8012199
:10C260000029F7D1704730B450E8022F1FFAA2F32B
:10C27000C488A34202BFBFF32F8F00200DE0C48902
:10C2800023448489A34228BF1B1BC2EA034340E81E
:10C290000234002CE8D14FF001000A6030BC704736
:10C2A00050E8022FC2EA224240E802210029F7D1D9
:10C2B0007047034653E8022FD988B2EB324F4FF054
:10C2C000000017BF92B241EA014142EA014104E095
:10C2D0005A68B2EB324F08BF012043E80212002A2D
:10C2E000E8D1704730B4044654E8000F0D4644E8E6
:10C2F0000053002BF8D1156030BC704730B40446B1
:10C3000054E8000F40EA010544E80053002BF7D140
:10C31000156030BC704730B4044654E8000F00EAA2
:10C32000010544E80053002BF7D1156030BC70477D
:10C3300030B4044654E8000F80EA010544E8005395
:10C34000002BF7D1156030BC704730B4044654E878
:10C35000000F00EB010544E80053002BF7D11560F6
:10C3600030BC704730B4044654E8000FA0EB010520
:10C3700044E80053002BF7D1156030BC704770B40F
:10C3800004464FF0000054E8006F0D68AE4207BF4E
:10C3900044E80023012044E800630E60002B1CBF2A
:10C3A0000020F0E770BC704730B4044654E8000F3A
:10C3B00088422CBF451A054644E80053002BF5D1AE
:10C3C000156030BC704700000648804706480047AB
:10C3D000FEE7FEE7FEE7FEE7FEE7FEE7FEE7FEE735
:10C3E000FEE7FEE7DDDA0E0001C20E002DE9F05F88
:10C3F0000546002092469B468846064681464024D4
:10C400001BE0284641464746224600F083F8534643
:10C410005A46C01A914110D311461846224600F0E0
:10C4200016F82D1A67EB01084F462246012000211D
:10C4300000F00DF817EB00094E41201EA4F1010495
:10C44000DFDC484631462A464346BDE8F09F202AB5
:10C4500004DB203A00FA02F1002070479140C2F15B
:10C46000200320FA03F319439040704700487047B7
:10C4700004A50F0010B5441A0346944209D284184B
:10C48000114403E011F8013D04F8013D521EF9D2B8
:10C4900010BD40EA0104A40703D009E010C9121F2F
:10C4A00010C3042AFAD203E011F8014B03F8014B40
:10C4B000521EF9D210BDD2B201E000F8012B491E84
:10C4C000FBD270470022F6E710B513460A46044631
:10C4D0001946FFF7F0FF204610BD421C10F8011B63
:10C4E0000029FBD1801A704730B50446002003466E
:10C4F00000E05B1C934203D2E05CCD5C401BF8D0B3
:10C5000030BD034611F8012B00F8012B002AF9D1A8
:10C5100018467047202A04DB203A21FA02F0002155
:10C52000704721FA02F3D040C2F120029140084343
:10C5300019467047064C074D06E0E06840F00103DD
:10C5400094E8070098471034AC42F6D3FFF75CFE3E
:10C5500080AE0F00A0AE0F0070B58C1810F8015B14
:10C5600015F0070301D110F8013B2A1106D110F88C
:10C57000012B03E010F8016B01F8016B5B1EF9D190
:10C580002B0705D40023521E0DD401F8013BFAE716
:10C5900010F8013BCB1A921C03E013F8015B01F881
:10C5A000015B521EF9D5A142D8D3002070BD000016
:10C5B000054B4FF0FF321A6053F8042C034B1A60FE
:10C5C0001A68034B1A60704704BA0250148B00209B
:10C5D00008BA025001EB820204388A4201D10020DD
:10C5E000704752F8043D1BBA40F8043FF5E70000DD
:10C5F00000B5374B8FB019461A680092009AD207DF
:10C60000FAD5344B344A1A600A680192019AD0076D
:10C61000FAD5324A1A600A680292029AD207FAD50B
:10C620002F4A1A600A680392039AD007FAD52D4A56
:10C630001A600A680492049AD207FAD52A4A1A6044
:10C640000A680592059AD007FAD5284A1A600A683E
:10C650000692069AD207FAD5254A1A600A68079206
:10C66000079AD007FAD5234A1A600A680892089AEE
:10C67000D207FAD5204A1A600A680992099AD007A7
:10C68000FAD51E4A1A600A680A920A9AD207FAD59F
:10C690001B4A1A6008680B900B98C007FAD51A60FD
:10C6A0000A680C920C9AD007FAD5164A1A600A68E2
:10C6B0000D920D9AD207FAD5134A1A600E210D2356
:10C6C0000F22002000F088FD0FB05DF804FB00BFD2
:10C6D000B0B0025080B0025080430129406339213C
:10C6E000807001298020542100D13490C0403490C2
:10C6F000C0302029C0530D9000413890832308C8D2
:10C7000080E3102100413821CF4308C810B5504BB9
:10C7100096B01C461A680192019AD207FAD54D4B81
:10C720004D4A1A6022680292029AD207FAD54B4A01
:10C730001A604B4A42EA804022680392039AD20769
:10C74000FAD5186022680492049AD007FAD5454AAF
:10C750001A60A2F5800242EA814122680592059A98
:10C76000D207FAD5196022680692069AD007FAD540
:10C770003D4A1A6022680792079AD107FAD53B4AC8
:10C780001A6022680892089AD207FAD5384A1A60C5
:10C7900022680992099AD007FAD5364A1A602268A7
:10C7A0000A920A9AD107FAD5334A1A6022680B9284
:10C7B0000B9AD207FAD5314A1A6022680C920C9A69
:10C7C000D007FAD52E4A1A6022680D920D9AD10729
:10C7D000FAD52C4A1A6022680E920E9AD207FAD520
:10C7E000294A1A6022680F920F9AD007FAD5274A71
:10C7F0001A60216810911099C907FAD51A60144B74
:10C800001A46196811911199C807FAD5114B204998
:10C810001960116812911299C907FAD51D4919605A
:10C82000116813911399CC07FAD50B491960116857
:10C8300014911499C807FAD5174919601168159110
:10C840001599C907FAD5154A1A6016B010BD00BF70
:10C85000B0B0025080B002504004419000862929B7
:10C86000D81001C84014419040142129401465217A
:10C870000034409000310C90C0400C90C030202912
:10C8800040960D9000416090031645C80086112126
:10C8900000416021594644C84014459040142D90F1
:10C8A000F0B5464B89B01D461C680194019CE40715
:10C8B000FAD5434BDFF810C1DFF810E113449B00B9
:10C8C0000A181B681E2A88BFC0F11E011F330A18F0
:10C8D0005B095A43B2F5806F88BF4FF480614FF017
:10C8E000000484BFB1FBF3F1091A00F1A05000F578
:10C8F0002C402746A14233DC2A680492049AD207CE
:10C90000FAD5304A1268296805910599CF07FAD5FA
:10C910002D482E4C0260002216469A4202F1010177
:10C9200040D12A4C134621F0010100268B423CD312
:10C930002B680693069BDE07FAD5254B1B682C68EF
:10C940000794079CE407FAD5036000231F481C46A0
:10C950009A422DD11D4A00208B422CD309B0F0BD44
:10C960002A680292029AD207FAD502199200126836
:10C970002E680396039EF607FAD5CCF80020002215
:10C980009A4202F1010206D11E4622F001029642AD
:10C9900004D30134AEE7CEF80070F1E7CEF80070B2
:10C9A0000136F4E726600A46B7E726600133BDE7A3
:10C9B00004600133CCE710600133CDE7B4B002501E
:10C9C00024AC00147CB00250D4B00250D8B0025055
:10C9D00078B00250F0B5294D85B02C462E680096EF
:10C9E000009EF607FAD500F1A05000F52C4080001B
:10C9F0000568206801900198C707FAD52048214FA3
:10CA0000056002EB8306B24229D15A1C1D4E22F06A
:10CA100001020027934227D323680293029BDE077B
:10CA2000FAD5194B0B449B001B681F335B099A42D4
:10CA300013D2216803910399C907FAD5154400213F
:10CA40009B1A104A05600846994210D35A1C0D499A
:10CA500022F00102002093420CD305B0F0BD52F841
:10CA600004EBC7F800E0CEE737600133D2E710608F
:10CA70000131E9E708600133EDE700BFB4B00250CF
:10CA8000D4B00250D8B0025024AC001410B5494BB9
:10CA900094B019461A680092009AD207FAD5464B0C
:10CAA000464A1A600A680192019AD407FAD5444AA4
:10CAB0001A600A680292029AD007FAD541481860B3
:10CAC0000A680392039AD207FAD53F4A1A600A68A5
:10CAD0000492049AD407FAD53C4A1A600A6805926F
:10CAE000059AD207FAD53A4A1A600A680692069A57
:10CAF000D407FAD5374A1A600A680792079AD2070C
:10CB0000FAD5354A1A600A680892089AD407FAD505
:10CB1000324A1A600A680992099AD207FAD5304A4D
:10CB20001A600A680A920A9AD407FAD52D4A1A603E
:10CB30000A680B920B9AD207FAD52B4A1A600A6838
:10CB40000C920C9AD407FAD5284A1A600A680D92FA
:10CB50000D9AD207FAD5264A1A600A680E920E9AE2
:10CB6000D407FAD5234A1A600A680F920F9AD2079F
:10CB7000FAD5214A1A600F4B19461C681094109C74
:10CB8000E407FAD50C4B1860086811901198C40797
:10CB9000FAD51A600A681292129AD007FAD5174A83
:10CBA0001A600A681392139AD207FAD5144A1A60C7
:10CBB00014B010BDB0B0025080B00250809065211A
:10CBC00000040990409665908080612180200821B2
:10CBD0008020649000816190004610210081112125
:10CBE0000041442180202029024610C800860921E6
:10CBF00080206021402128294096652140962529E2
:10CC0000594614C810B5544B98B019461A68019289
:10CC1000019AD207FAD5514B514A1A600A6802921A
:10CC2000029AD407FAD54F4A1A600A680392039A07
:10CC3000D007FAD54C4818600A680492049AD207C3
:10CC4000FAD54A4A1A600A680592059AD407FAD5B5
:10CC5000474A1A600A680692069AD207FAD5454AE8
:10CC60001A600A680792079AD407FAD5424A1A60EE
:10CC70000A680892089AD207FAD5404A1A600A68E8
:10CC80000992099AD407FAD53D4A1A600A680A92AD
:10CC90000A9AD207FAD53B4A1A600A680B920B9A95
:10CCA000D407FAD5384A1A600A680C920C9AD2074F
:10CCB000FAD5364A1A600A680D920D9AD407FAD549
:10CCC000334A1A600A680E920E9AD207FAD5314A90
:10CCD0001A600A680F920F9AD407FAD52E4A1A6082
:10CCE0000A681092109AD207FAD52C4A1A601A4B89
:10CCF00019461C681194119CE407FAD5174B18606B
:10CD0000086812901298C407FAD51A600A6813923C
:10CD1000139AD007FAD5124A1A600A681492149A24
:10CD2000D207FAD51E4A1A600A681592159AD407D6
:10CD3000FAD51C4A1A600A681692169AD007FAD5D4
:10CD4000194A1A600A681792179AD207FAD5174A31
:10CD50001A6018B010BD00BFB0B0025080B00250D1
:10CD60000093652100043190409665900083612115
:10CD700000C3302100C364900081619000461021FF
:10CD8000008111210041442100C320290C4610C814
:10CD90000086312100C3602140C1282940966521C9
:10CDA0000013319040962529594614C84004324951
:10CDB0002DE9F041814B1D6898682033A0B01E46D4
:10CDC0001A680192019AD707FAD57D4B7D4A1A60FD
:10CDD00032680292029AD407FAD57B4A1A607B4ADB
:10CDE0001446116803910399C907FAD5784A116866
:10CDF000C1F3402137680497049FFF07FAD5754FA8
:10CE00001F6027680597059FFF07FAD51768002957
:10CE100000F0CF80B90540F1CC80316806910699C9
:10CE2000CF07FAD56C491960216807910799C9079E
:10CE3000FAD51168C1F3402137680897089FFF07AA
:10CE4000FAD5664F1F6027680997099FFF07FAD533
:10CE50001268002900F0AF80910540F1AC80326883
:10CE60000A920A9AD207FAD5564A1A6032680B9289
:10CE70000B9AD707FAD55A4A1A6031680C910C9967
:10CE8000CC07FAD55749196031680D910D99C9073A
:10CE9000FAD55549196031680E910E99CF07FAD528
:10CEA0005249196031680F910F99CC07FAD5504952
:10CEB0001960504B1E46196810911099C907FAD590
:10CEC0003F4C4D4B236033681193119BDB07FAD520
:10CED0004A4B236033681293129BDF07FAD5484B05
:10CEE00023603A4B9846196813911399C907FAD5EC
:10CEF000324F386033681493149BDB07FAD52260F5
:10CF000033681593159BD807FAD53E4B23603368D9
:10CF10001693169BD907FAD53B4B236033681793BA
:10CF2000179BDA07FAD5394B236033681893189B9F
:10CF3000DB07FAD5364B236033681993199BD80762
:10CF4000FAD5344B236033681A931A9BD907FAD564
:10CF5000314B236033681B931B9BDA07FAD52F4BA9
:10CF6000236000F0D3F908BBD8F800301C931C9B59
:10CF7000DB07F9D53D6033681D931D9BD907FAD5B2
:10CF8000274B236033681E931E9BDA07FAD5254B87
:10CF90002360D8F800301F931F9BDB07F9D50C4B9B
:10CFA0001B6813F4805F204B08BF184620B0BDE813
:10CFB000F0811E48FAE71E48F8E700BF90B0025023
:10CFC00080B0025000100251C01F7229B4B002504C
:10CFD00088B00250C0CF0129C01F0E29C03F0029D0
:10CFE00040010249003184A800001649400108A10F
:10CFF00080440888B0B00250C044708880077A41ED
:10D00000C0077E4100006A498006164940006E490B
:10D0100000020021008220214082202180822421E0
:10D0200040A161A100C861510308F1000108F100AD
:10D030000208F10008B540B1202801464FF0070270
:10D0400028BF20210020FFF72BFC024B00221A6092
:10D0500008BD00BF1CB802507FB51C681CB901F0A8
:10D060001F041F2C27D1174C254626680196019EC8
:10D07000F607FAD500F1A05000F52C4080000068BA
:10D080002C680394039CE407FAD50F4C00EB611065
:10D0900020600E4801F01F04006802901F2C18BF8A
:10D0A000C94302980FBF106001F01F0100FA01F19F
:10D0B00011600021196010684300C00F136004B0B4
:10D0C00070BD00BFB4B00250E4B00250DCB00250FA
:10D0D00030B51E4B85B01A46196800910099CC07EF
:10D0E000FAD500F1A05000F52C40800001681368CB
:10D0F0000193019BD807FAD5154B164C1868164DAD
:10D100001F30202390FBF3F00138002810DA0023B1
:10D110000130400153B1A0F120014FF00042134211
:10D1200004D1013881424FEA5202F8D105B030BD36
:10D1300013680393039BDB07FAD5431823602B681E
:10D140000293029B002BE3D10138DEE7B4B002501A
:10D15000ACB00250E4B00250DCB002500A460021EC
:10D16000AFF3008038B5A0F12003B3F5426F054658
:10D170002CD88F2826D800F1470300F16604DB067F
:10D180004FEA541400D0013464013F34A40901343F
:10D1900011B1A1421AD30C46E3004FF48050B0FB0A
:10D1A000F3F0202828BF202002B11060084B012294
:10D1B0001A60214600F068F82846214600F088F8F9
:10D1C000002038BD00F11F046409DDE7014838BDC7
:10D1D0001CB802502221F00070B5264888B00546E0
:10D1E00004680094009CE607FAD52348234C0460A9
:10D1F000234C44EA83432C680194019CE407FAD54C
:10D200000360930143EA824242F0104444F4C04474
:10D210002B680293029BDE07FAD504602B68039308
:10D22000039BDB07FAD5174B03608B0143EA81416F
:10D2300041F0104343F4C0432E680496049EF60761
:10D24000FAD503602B680593059BDE07FAD50460C9
:10D2500041F058412B680693069BDC07FAD5016024
:10D2600042F058422B680793079BDB07FAD5026010
:10D2700008B070BDB0B0025080B00250C021022989
:10D28000807100988061189030B500220C4C4900E4
:10D290001346023840F6FC75904202F10102CABF03
:10D2A000236025605B181E2A04F10404F4D1054AAA
:10D2B00019441360044B054A19609A6030BD00BFE1
:10D2C00000B0025078B002507CB0025020F80F003D
:10D2D0000C4B18603F3020F03F008901403058600F
:10D2E0009960D9601961596199611C3306481960C8
:10D2F00082B002680192019AD207FAD5196002B091
:10D30000704700BF90B00250B4B002502DE9F04118
:10D3100092B0012303930493624B1D461A68059251
:10D32000059AD207FAD5604C604B2360604B1946D2
:10D330001A680692069AD707FAD55E4B1A68D60481
:10D3400000F1A8802A680792079AD007FAD55A4AAE
:10D3500022600A680892089AD207FAD51E68C6F3B6
:10D360000036002E40F098801220FFF7B1FE0746ED
:10D370001320FFF7ADFE87428CBF12201320FFF76A
:10D38000A7FE471EFFF734F903AB01AA3946122066
:10D39000FFF762FE04AB804602AA39461320FFF76E
:10D3A0005BFE00EB4800022832D003283ED0012863
:10D3B00074D12B680993099BDB07FAD53F4B236097
:10D3C0002B680A930A9BD807FAD53D4B23602B683C
:10D3D0000F930F9BD907FAD53A4B23602B68109314
:10D3E000109BDA07FAD5384B23602B681193119BF9
:10D3F000DB07FAD5354B2360013F25D510231922D1
:10D4000018210020FFF7E8FE304612B0BDE8F08199
:10D410002B680B930B9BD907FAD52D4B23602B68F8
:10D420000C930C9BDA07FAD52A4BCFE72B680D93A8
:10D430000D9BDB07FAD5284B23602B680E930E9BC0
:10D44000D807FAD5254BC1E703AB01AA394612200C
:10D45000FFF702FE04AB044602AA39461320FFF789
:10D46000FBFD10EB440402D1FFF7CCFBC4E7FFF750
:10D470000DFB022C08D0032C09D0012C10D1172150
:10D480001620FFF743F9B7E715211420F9E70F211C
:10D490000E20F6E7124EB7E7124EB5E7124EB3E78D
:10D4A000124EB1E7B0B0025080B0025000084A51AD
:10D4B000B4B0025088B0025000084E5100065A49DC
:10D4C00040065E49000442410014424940042E498E
:10D4D000000652494006564900063A4940063E4970
:10D4E0000608F1000708F1000408F1000508F10042
:10D4F000014B1860704700BF08BA0250014B18601A
:10D50000704700BF04BA0250094BC2431A60043B83
:10D5100082B01B680193074B019A104204D0064A5F
:10D520001060186802B0704720BF1A680192F3E7D4
:10D5300004BA0250148B002008BA0250FEF79ABFBA
:10D54000FEF7C2BF0A460021FEF7BEBF2DE9F74332
:10D5500005460E469946114600F060FA044600283A
:10D5600040F08480002E00F08580002900F0848047
:10D57000B9F1200F40F0828005F14404082205F142
:10D5800004082046FFF726F805F124070822314653
:10D590004046FFF71FF806F1200108223846FFF742
:10D5A00019F802A94FF4807041F8049DFFF7D6FDE9
:10D5B000002865D1334A4FF48073136001219360D2
:10D5C0000823314AFFF706FA0121084605232F4AAE
:10D5D000FFF700FA0823424601211C20FFF7FAF961
:10D5E00008233A4601210320FFF7F4F922460823D5
:10D5F00001210220FFF7EEF90823254A01211A2014
:10D60000FFF7E8F90523234A01211B20FFF7E2F980
:10D610000823214A01211420FFF7DCF908231F4ABF
:10D6200001211520FFF7D6F9082305F16402012135
:10D630001620FFF7CFF9082305F1840201211720F6
:10D64000FFF7C8F90823164A01210B20FFF7C2F99A
:10D65000FFF7AEFB04460198FFF7ECFC114B002CE2
:10D6600018BF1C46A4212846FFF76CFF204603B0D4
:10D67000BDE8F0830C4CF9E70C4CF7E70C4CF5E7F0
:10D68000084CEFE790B00250F4AD0F006CAE0F0005
:10D69000B4AD0F0058AE0F0018AE0F0038AE0F003B
:10D6A000D4AD0F008408F0007608F0008008F00088
:10D6B0008108F00038B50D460446B0B1A022002123
:10D6C0000430FFF73DFF95B12946082204F16400BC
:10D6D000FEF780FF082205F1200104F18400FEF727
:10D6E00079FF044B2360002038BD034838BD034850
:10D6F00038BD00BFDD55AABB7108F0008308F000FB
:10D700002DE9F041069F044615461E46FFF7D2FF5D
:10D7100038B93B46324629462046BDE8F041FFF77E
:10D7200015BFBDE8F08100002DE9FF41144B044610
:10D730000E460FCB8DE80F00204600F07FF98046A3
:10D74000B0B9CEB1636A251D01953BB9012363626F
:10D75000226F04F13001684600F088F82B46043E41
:10D76000243453F8042B12BAA34246F8042FF8D1FC
:10D77000404604B0BDE8F081DFF80880F8E700BF5C
:10D7800084AD0F000502F00038B5044668B1051DF0
:10D7900028467021FFF7D6FE284620220449FFF7CD
:10D7A000CDFE044B2360002038BD034838BD00BFC8
:10D7B00094AD0F00DD55AABB0002F000294B2DE906
:10D7C000F04304460E4615460FCB85B06F468DE8F4
:10D7D0000F002DB94FF00009484605B0BDE8F083B1
:10D7E000204600F02BF981460028F5D1231D019336
:10D7F000636AA3BB236F8BB1C3F14008A84528BF60
:10D80000A84604F13000314618444246FFF796FE20
:10D81000236F434446442367A5EB0805226F402A43
:10D8200006D104F13001384600F020F800232367C8
:10D8300005F03F0835F03F0505D031462A46384609
:10D8400000F014F82E44B8F1000FC3D04246314620
:10D8500004F13000FFF772FEC4F87080BCE7DFF817
:10D860000890B9E784AD0F000C02F0002DE9F74FE6
:10D87000314B44688046924699461A68002AFCD18A
:10D880002E4B9B461A68002AFCD14FF0FF300191C5
:10D89000FFF72EFE8020FFF731FE294D294A2A4F3F
:10D8A0002A4E012307202B60A2F59E72C2F83C018C
:10D8B0001360636A3B60A36A3360D8F8003042F8B3
:10D8C000043CD8F80830204698470199D9F8003030
:10D8D000002BFBD1BAF1000F20D11D4B04221A609E
:10D8E000D9F80030002BFBD1DBF800A0BAF1000F13
:10D8F000FAD1D8F80C30204698473B686362336809
:10D90000A362144BC3F800A0C3F844A1D9F80030B7
:10D91000002BFBD12B6003B0BDE8F08F236A012BF5
:10D9200004BF0C4A13600C4B40201960C3F804A0DC
:10D93000FFF7EAFDD4E700BF10B9025020BC025047
:10D9400018B8025000B90250CCB70250D0B70250FC
:10D95000C8B7025084B6025028BC0250084B1B685E
:10D960001B0EF02B08D1074B1A68074B9A4205D1C2
:10D97000064B00201860704705207047062070474E
:10D9800028B9025024BA02500000E0200CBA02501C
:10D990000C4B1B68C3610C4B1B6883610B4B1B68F2
:10D9A00043610B4B1B6803610A4B1B68C3600A4B46
:10D9B0001B688360094B1B684360094B1B6803604D
:10D9C000704700BF5CB6025058B6025054B60250C1
:10D9D00050B602504CB6025048B6025044B60250FF
:10D9E00040B602500C4BC2691A60826943F8042C9D
:10D9F000426943F8082C026943F80C2CC26843F8CA
:10DA0000102C826843F8142C426843F8182C0268E2
:10DA100043F81C2C704700BF5CB6025030B102685E
:10DA2000034B04489A4208BF0020704702487047E1
:10DA3000DD55AABB8208F0007108F00030B1026821
:10DA4000034B04489A4208BF0020704702487047C1
:10DA5000DD55AABB0202F0000002F00010B509F08B
:10DA6000EDF8BDE8104009F04BB80000024902484B
:10DA7000091F0968006808474401002000F00ABA3D
:10DA800070B50E46144900EB400001EBC00514468A
:10DA9000E86A183520B101280FD0022805D113E01B
:10DAA000284600F02DFAA04201D2002411E02246BF
:10DAB0003146284600F071FA0BE0284600F020FAC3
:10DAC000A042F4D20446F2E73146284600F038FA84
:10DAD0000446204670BD00006461002030B54FF060
:10DAE000805000228300D0F83011C3F80C21C3F815
:10DAF0001021624B1A60624B1B68624C2360604BC2
:10DB00001B1D1B68241D23605D4B08331B68241DEF
:10DB100023605B4B0C331B68241D2360584B103370
:10DB20001B68241D2360564B14331B68241D23607F
:10DB3000534B18331B68534C20342360504B1C3319
:10DB40001B68241D23604E4B20331B68241D23605B
:10DB50004B4B24331B68241D2360494B28331B681F
:10DB6000241D2360464B2C331B68241D2360444B2B
:10DB700030331B68434C40342360414B34331B68C3
:10DB8000241D23603E4B38331B68241D23603C4B0F
:10DB90003C331B68241D2360394B40331B68241D14
:10DBA00023600124082902D1D0F8343113B10829A7
:10DBB00004D006E0354B3449196005E0D0F8343123
:10DBC00013B1082904D006E0314BFB21196005E0B0
:10DBD000D0F8343113B1082908D00EE090F858324B
:10DBE0002C48016863F30301016002E0D0F834318E
:10DBF0001BB929494FF40070086028480168C9071B
:10DC000002D06FF0010101602548016841F4700104
:10DC10000160BFF34F8FBFF36F8F4FF01021D1F82A
:10DC20000002002803DBD1F80402002822DA1D4B91
:10DC30001C601D480468002CFCD01224C1F800426E
:10DC40000568002DFCD0C1F8044201680029FCD011
:10DC50001A6001680029FCD0BFF34F8F10487C3850
:10DC60000168124A01F4E06111430160BFF34F8F74
:10DC700000BFFDE70F490E48086030BD3805004081
:10DC80000404001020C50040488103008C56004069
:10DC900018F50040E40E00404096024000040040A9
:10DCA00088ED00E004E5014000E401400400FA05CD
:10DCB0000090D003C001002010B5054C206818B9B1
:10DCC00004A12B2001F0E8FE2068BDE810400047C9
:10DCD000B00000202E2E5C2E2E5C2E2E5C2E2E5C94
:10DCE0002E2E5C6D6F64756C65735C6E7266785C0D
:10DCF000647269766572735C7372635C7072735C74
:10DD00006E7266785F7072732E6300002DE9F05FAB
:10DD10005448D0F8045300242E464FF0010913E074
:10DD200096FAA6F0B0FA80F7B80000F58070804649
:10DD300008F0E0FD28B1404608F0E4FD09FA07F0DC
:10DD4000044309FA07F08643002EE9D107F080F872
:10DD5000002869D0444AD078F0BBA00264D543497A
:10DD600040F2A978C1F80080081D036813F0FF0C89
:10DD700002D0036803EA0C0C40F2AA7AC1F800A0B2
:10DD8000036813F0FF0301D00668334040F2AB7B19
:10DD9000C1F800B0066816F0FF0601D007683E40E3
:10DDA00040F2AC770F60076817EA0C0709D0D2F889
:10DDB00010C04CEA070CC2F810C0C1F80080076020
:10DDC000076840F2AD770F6007681F4009D01369FC
:10DDD00043EA0743136100E026E0C1F800A00760B2
:10DDE000036840F2AE730B60036833400BD0DE076C
:10DDF00001D044F40004DE0601D544F00104C1F86A
:10DE000000B003600068106930F0011102D005F025
:10DE100080710C4310F0011F06D0690504D520F075
:10DE2000011044F480641061C4F3C05624F400046B
:10DE30004F46DFF83C8009E094FAA4F0B0FA80F590
:10DE400058F82500804707FA05F08443002CF3D1E9
:10DE50000BF044FE002E03D0BDE8F05F03F07CBB66
:10DE6000BDE8F09F00700240800000200078024072
:10DE7000A8A10F00064808B50021016000680090C5
:10DE800008F0AAF907F07AFF0028FBD108BD0000CE
:10DE90000001014010B5124C02202061606111A008
:10DEA000A06104F17800E0614FF48050206200200E
:10DEB000A06260620BA1A164E0620D49E1641021DF
:10DEC000A065C4E91410E0650AA1E01DFEF719FB86
:10DED00009A12046FEF715FB2020A07110BD00000F
:10DEE000646100205465726D696E616C0000000011
:10DEF000DC710020525454005345474745520000FE
:10DF00000269C1688A4203D88068401A104400E060
:10DF1000501A401E70470000C11700EBD161074B3B
:10DF20004A1153F8222021F01F01411A0120884094
:10DF3000024201D0012070470020704700E100E05C
:10DF40002DE9F047C4681746894606464FF0000899
:10DF50003069A04201D9051B02E0B168201A0D1AF0
:10DF6000B0686D1E001BA84200D80546BD4200D314
:10DF70003D4670682A4620444946FEF77BFAB06861
:10DF80007F1B2C44A844A944A04200D10024F46083
:10DF9000002FDDD14046BDE8F0872DE9F041044671
:10DFA0008846D4E90207C51BE16860681646084444
:10DFB000B54206D94146FEF75DFAB819E060BDE802
:10DFC000F0812A464146FEF755FA761B08EB05011B
:10DFD00032466068FEF74EFAE660F0E70FB41CB513
:10DFE0000A46521ECDE9000207A9054B6A4606986B
:10DFF00000F018F8009A002111701CBC5DF814FBA9
:10E0000087E40E0002E008C8121F08C1002AFAD1F6
:10E0100070477047002001E001C1121F002AFBD1A8
:10E02000704700002DE9FF4F8DB00F4605460026D2
:10E0300006E025280BD0DDE90F1290476D1C761CF9
:10E0400028780028F5D111B03046BDE8F08F0024C3
:10E05000A246A1460122EC4900E0044315F8013F25
:10E06000203B02FA03F00842F7D128782A2810D082
:10E070006FF02F022878A0F13001092914D80AEB9B
:10E080008A0102EB410144F0020400EB010A6D1C1D
:10E09000F0E701CF5FEA000A03D544F40054CAF167
:10E0A000000A44F002046D1C28782E2817D115F8B8
:10E0B000010F44F004042A280ED06FF02F022878B4
:10E0C000A0F1300109290AD809EB890102EB4101CD
:10E0D00000EB01096D1CF2E757F8049B6D1C2878D2
:10E0E0006C280FD006DC4C2817D068280DD06A2881
:10E0F00014D104E0742810D07A280FD10DE044F434
:10E1000000140AE044F4801401E044F440146978F7
:10E11000814202D104F580146D1C6D1C2A786E2A90
:10E120001FD00CDC632A31D004DC002A8BD0582AA3
:10E1300011D1A3E0642A68D0692A0CD165E0732A62
:10E140002ED004DC6F2A73D0702A04D19BE0752A8C
:10E150006FD0782A6ED01046DDE90F129047761CFA
:10E1600050E1C4F30250022806D0032809D0042845
:10E1700001CF09D0066045E101CFF117C0E9006188
:10E1800040E101CF06803DE106703BE117F8040B4A
:10E190008DF8000000208DF80100EB46012003E01F
:10E1A00057F804BB4FF0FF3061074FF0000102D475
:10E1B0000DE008F10101884649450FDA8045F8DB9A
:10E1C0001BF808100029F4D108E008F10101884685
:10E1D0008142FADB1BF808100029F6D1DDE90F2394
:10E1E000AAEB08008146214600F036F9304400EBE6
:10E1F000080604E0DDE90F121BF8010B9047B8F1A7
:10E200000108F7D221464846F7E00A21C4F3025339
:10E210004FF0000B0891022B04D001CFC117032B44
:10E2200009D00AE0FF1D27F00707F7E8020108E020
:10E2300032E01FE020E000B2C117042B01D140B250
:10E24000C117031E71F1000307DA4FF0000CD0EB89
:10E250000C006CEB01012D2302E0230504D52B23D8
:10E260008DF82430012303E0E30701D02023F7E7F2
:10E27000984658E00A2110E010210EE010204FF0DF
:10E28000000B08900CE010214FF0000B44F0040448
:10E290004FF00809089103E008214FF0000B0891A6
:10E2A000C4F30253022B04D001CF0021032B06D06C
:10E2B00006E0FF1D27F00707F7E8020103E080B240
:10E2C000042B00D1C0B24FF0000823072BD5702AD1
:10E2D00007D0DDF820C08CF0100C5CEA0B0C05D0E8
:10E2E0000EE040238DF82430012308E050EA0103BA
:10E2F00006D030238DF824308DF82520022398464F
:10E30000DDF820C08CF0080C5CEA0B0C0BD150EA55
:10E31000010301D1630706D530238DF824304FF077
:10E320000108A9F10109582A04D038A20B9208AAC1
:10E330000A920BE03AA2F9E75B46089AFEF756F814
:10E340000B9B9B5C0A9A521E0A92137050EA0102C0
:10E35000F2D10A98ADEB000000F1200B600702D566
:10E3600024F4803401E04FF00109D94502DDA9EB26
:10E370000B0000E0002000EB0B0141440890AAEBE9
:10E38000010AE00306D4DDE90F232146504600F0E0
:10E3900063F806444FF0000908E009A911F80900E4
:10E3A000DDE90F12904709F10109761CC145F4DB44
:10E3B000E0030CD5DDE90F232146504600F04CF870
:10E3C000064404E0DDE90F1230209047761C0899DE
:10E3D000481E08900029F5DC08E00A980A990078A0
:10E3E000491C0A91DDE90F129047761CBBF1000130
:10E3F000ABF1010BF1DC21465046DDE90F2300F0C3
:10E4000019F806446D1C1BE609280100303132332F
:10E410003435363738396162636465660000000060
:10E42000303132333435363738394142434445464A
:10E43000000000002DE9F041044600251E46174665
:10E44000880404D405E039462020B0476D1C641EC2
:10E45000F9D52846BDE8F0812DE9F04104460025B4
:10E460001E469046C80301D5302700E020278804C7
:10E4700004D505E041463846B0476D1C641EF9D509
:10E480002846BDE8F0814A68002A06D00A68531C75
:10E490000B6010704868401E48607047800701D0CC
:10E4A000002070470120704740680068401E084205
:10E4B00001D10120704700207047C3688B4206D805
:10E4C00011440069491E814201D801207047002093
:10E4D000704700002DE9F05FDFF894B05C46DBF890
:10E4E0004890DBF8245004F063FC216B214E00EBD4
:10E4F00001086F1A31884FF0040A0AEB01401EA18F
:10E5000007F09CFD216B40464944414500D100275E
:10E5100008233A4603F032FA07004FF0010806D00C
:10E52000318808EB01401BA107F088FD1CE004F0D6
:10E530003FFC0022294602F095FADBF82820044629
:10E540003188D946A24209D10AEB014018A107F04F
:10E5500075FDC9E90748C9F8185005E008EB014006
:10E560002346194907F075FD3846BDE8F09F0000C5
:10E57000BC17002030020020456E746572206E7258
:10E58000665F6466755F6170705F636F6E74696EFD
:10E59000756500004661696C656420746F20636F67
:10E5A0007079206669726D776172652E00000000D7
:10E5B00053657474696E6720617070206173207692
:10E5C000616C696400000000A4A50F0008B5134643
:10E5D0000246064800930123008803EB00400B46E7
:10E5E00003A107F03EFD08F0E3FF00003002002029
:10E5F00052656365697665642061206661756C7437
:10E60000212069643A203078253038782C207063D6
:10E610003A203078253038782C20696E666F3A20A1
:10E6200030782530387800000246054801210088FE
:10E6300001EB004003A107F005FD08F0B9FF000061
:10E6400030020020526563656976656420616E2042
:10E650006572726F723A2030782530387821000068
:10E660002DE9F047244C8146924660880E4681424F
:10E670003FD84FF6FF77002001F0A0F922786078AC
:10E68000A188884201DA401C00E00020C0B290421C
:10E6900003D1002001F0C0F929E065784FF00008AF
:10E6A0006078884201DA401C00E0002060700020A1
:10E6B00001F0B2F9BD421AD0A068B9F1000F40F8DC
:10E6C00035A00DD066B16188E068324605FB0100D7
:10E6D0004946FDF7CFFEA06800EBC500868003E049
:10E6E00000EBC500A0F804800020BDE8F0870420FE
:10E6F000FBE70920F9E70000B800002010B50E4C38
:10E7000003E0401C00E00020207020786178814206
:10E7100010D022786188E068A36802FB010003EB57
:10E72000C20153F83220898890472078A188884216
:10E73000E9DAE6E710BD0000B800002030B5CB00F4
:10E7400008339DB293074FF0000401D0072030BD7D
:10E75000044B9A602A44DA605C701C70588099807F
:10E76000002030BDB8000020014802F002BC0000CB
:10E77000D000002070B514460E46050004D10B49A8
:10E7800040F2C51001F088F93CB12868012EC46040
:10E790000AD000218160002070BD04494FF4E3706D
:10E7A00001F07AF9072070BD0121F3E728A90F00D5
:10E7B00038B50E4808235822416800910C4900687A
:10E7C00003F0D8FB00280FD10A4A69460A4802F034
:10E7D000D5FB040008D10121074802F09AFC064944
:10E7E000012008390870204638BD000044A20F00FF
:10E7F000D81E0020FD830F00D000002070B5164603
:10E800000D46040004D10C4940F2D51001F044F942
:10E810000A48854201D9072070BD0948266102F0E7
:10E82000A8FB28446060A06800B1A5602146BDE84F
:10E83000704000200AF0FABD28A90F0017FCFF0065
:10E84000D000002010B5040004D106494FF4F57043
:10E8500001F022F9002021462076BDE81040012079
:10E860000AF0E4BD28A90F0070B5054606484468C3
:10E8700007E02946204602F079F8204600F0A8FA81
:10E880000446002CF5D170BDF000002070B50A4898
:10E8900045680EE02E7A002405E02146284600F067
:10E8A0008DFE641CE4B2B442F7D3284600F090FA1F
:10E8B0000546002DEED170BDF00000202DE9F0419D
:10E8C0000E4840F2AB67456814E02E7A00240BE056
:10E8D00000222146284600F0D3FE18B108A1384690
:10E8E00001F0DAF8641CE4B2B442F1D3284600F037
:10E8F0006FFA0546002DE8D1BDE8F081F000002058
:10E900002E2E5C2E2E5C2E2E5C2E2E5C2E2E5C630C
:10E910006F6D706F6E656E74735C6C69627261723C
:10E920006965735C757362645C6170705F75736256
:10E93000642E630070B506460948062544680AE05F
:10E940003146204602F012F80546062805D1204639
:10E9500000F03EFA0446002CF2D1284670BD0000BB
:10E96000F00000202DE9FC4115460E00074604D1B9
:10E97000294940F2A73001F08FF8384601F05CFBDE
:10E980000446007DC0070DD0002001F017F8A069F3
:10E9900050B1206AD8B31124002001F03DF8204680
:10E9A000BDE8FC810820FBE7E06EA8420DD32A46B3
:10E9B0003046A16EFDF75EFDE06E401BE066A06E86
:10E9C00065672844A0660024E6E7C4E90665384682
:10E9D00002F087F8054611480069CDE90004E26EAF
:10E9E0006AB1A16EA069FDF745FDE169E06E091A03
:10E9F000E161A1690144A16120670020E0666946E8
:10EA0000284600F013FC0400C6D19224C4E7FFE7B7
:10EA1000C4E90865F9E700006CA90F00A4A20F0083
:10EA2000FEB515460E46044601F006FB007D10F0CB
:10EA3000010F0AD0204602F04BF800210096CDE9E4
:10EA40000151694600F03CFCFEBD0820FEBD0000FF
:10EA5000F8B5040004D138A140F2EF4001F01CF8F1
:10EA6000606820B934A14FF49E6001F015F8606829
:10EA7000006820B930A140F2F14001F00DF82068A3
:10EA8000006820B12CA140F2F24001F005F806F038
:10EA900063FB10B906F06AFB20B927A140F2F640EB
:10EAA00000F0FAFF00250FE0002705E0007800F0F5
:10EAB000D1FB08B11120F8BD3946781CC7B23046E9
:10EAC00000F0BEF80028F1D12946681CC5B22046E6
:10EAD00000F01AF90600E7D100250DE0002703E059
:10EAE0000078214600F0BCFB3946781CC7B230469E
:10EAF00000F0A6F80028F3D12946681CC5B22046CC
:10EB000000F002F90600E9D1184D40F21C5607E06A
:10EB1000A04203D108A1304600F0BEFF2868056876
:10EB200028680028F4D112482C606946406900909A
:10EB3000204601F01BFFF8BD2E2E5C2E2E5C2E2EE3
:10EB40005C2E2E5C2E2E5C636F6D706F6E656E7426
:10EB5000735C6C69627261726965735C757362641F
:10EB60005C6170705F757362642E6300F400002056
:10EB700058A20F002DE9F04F87B04FF000081D4656
:10EB8000934689460446DDF840A04646CDF80C8001
:10EB900000E0761C6068012300224768214603A834
:10EBA000B8470028F5D140468DF800800027B846C8
:10EBB00001903BE0606801236A46D0F804C021461A
:10EBC00001A8E0476068012305AAD0F804C02146E7
:10EBD00001A8E0479DF8141049451AD1D84514D131
:10EBE0009DF80000CAF8000005F8010B6A1C85F8C2
:10EBF000009060689DF800302146456801A89B1E82
:10EC0000A847002007B0BDE8F08F08F1010000F030
:10EC1000FF0860689DF800300022D0F804C021464B
:10EC200001A89B1EE0479DF800000744B742C1D3EE
:10EC30000520E7E70148406870470000F000002029
:10EC400070B50D46040004D106A14FF48E7000F09B
:10EC500023FF6078A84201D8002070BDA07820442E
:10EC6000284470BD2E2E5C2E2E5C2E2E5C2E2E5C2B
:10EC70002E2E5C636F6D706F6E656E74735C6C6965
:10EC8000627261726965735C757362645C617070F5
:10EC90005F757362645F636C6173735F62617365F8
:10ECA0002E68000070B50D46040004D106A14FF493
:10ECB0008E7000F0F1FE6078A84201D8002070BD8F
:10ECC000A0782044284470BD2E2E5C2E2E5C2E2E63
:10ECD0005C2E2E5C2E2E5C636F6D706F6E656E7495
:10ECE000735C6C69627261726965735C757362648E
:10ECF0005C6170705F757362645F636C6173735F96
:10ED0000626173652E68000070B50D46040003D182
:10ED100006A1E92000F0C0FE207AA84201D8002018
:10ED200070BD05EB45000934204470BD2E2E5C2ECD
:10ED30002E5C2E2E5C2E2E5C2E2E5C636F6D706F03
:10ED40006E656E74735C6C69627261726965735C26
:10ED5000757362645C6170705F757362645F636C2D
:10ED60006173735F626173652E68000070B50D4654
:10ED7000040003D106A1E92000F08EFE207AA8420B
:10ED800001D8002070BD05EB45000934204470BD5A
:10ED90002E2E5C2E2E5C2E2E5C2E2E5C2E2E5C6378
:10EDA0006F6D706F6E656E74735C6C6962726172A8
:10EDB0006965735C757362645C6170705F757362C2
:10EDC000645F636C6173735F626173652E680000DA
:10EDD00010B5040004D104494FF4F97000F05CFE52
:10EDE0002068006810BD00002CF50E0010B504006E
:10EDF00004D104A14FF4F97000F04EFE20680068C1
:10EE000010BD00002E2E5C2E2E5C2E2E5C2E2E5C55
:10EE10002E2E5C636F6D706F6E656E74735C6C69C3
:10EE2000627261726965735C757362645C61707053
:10EE30005F757362642E680002484078002800D035
:10EE400001207047F00000202DE9F041484E0D46AA
:10EE5000024609780624307801270F2964D2DFE8BA
:10EE600001F063080C0E63204863636363252D364D
:10EE70003F0003200AF0E4FC56E0002454E03C4844
:10EE8000001D03F0B9F828B13A480760BFF36F8F4F
:10EE9000BFF34F8F30780028EFD137A140F20B40FD
:10EEA00009E0104600F0A4F804463DE00028E4D054
:10EEB00031A140F2164000F0EFFDDEE7012804D05A
:10EEC0002DA140F21C4000F0E7FD002005E039488C
:10EED000006810F0010F0AD002200AF0B1FCCCE764
:10EEE000022804D224A14FF4866000F0D5FD012051
:10EEF000F3E7E878032817D0A87830B1802804D049
:10EF00001DA140F23E4000F0C7FD1949E8780831E4
:10EF10000A6832B100230B6049689047040006D0AC
:10EF200000E00E2406F07CF92046BDE8F0810AF0EE
:10EF3000E1FB28B1A8780028F6D106F034F9F3E710
:10EF40001D480078082810D11B48001D00780007D4
:10EF50000BD119480830007810F0F00F05D1164891
:10EF60000C30007810F0F00FDED006F019F9DBE776
:10EF7000100100205C7002402E2E5C2E2E5C2E2E86
:10EF80005C2E2E5C2E2E5C636F6D706F6E656E74E2
:10EF9000735C6C69627261726965735C75736264DB
:10EFA0005C6170705F757362645F636F72652E631E
:10EFB0000000000038040040E00F00F0024A014663
:10EFC000D2E9000210470000781F002070B50C46FF
:10EFD000054606F0DFF8A84201D0102070BD0348B6
:10EFE000D4E90012C0E90212002070BD1001002017
:10EFF0007FB5054605208DF8000006240DF10100BF
:10F0000006F0E6F80AF076FB2949002008609DF832
:10F01000010010F01F0006D001280FD0022826D0D2
:10F02000032833D106E06946284609F0EBFC044684
:10F0300006282AD16846FFF77DFC25E09DF80500EB
:10F0400003A900F0F9FA050008D06A469DF80C10F3
:10F0500000F0B0FA0446062802D016E0102415E0AD
:10F060006A469DF80C10284609F026FE0CE09DF833
:10F070000500010705D0694600F07EF80446062821
:10F0800003D1684609F068FD044624B106F0C8F8CB
:10F0900004B0204670BD0AF02DFB30B106F07AF8BE
:10F0A0000028F5D106F07FF8F2E706F079F8EFE7EF
:10F0B00018010020FEB5C08814460E46A04201D2B9
:10F0C000054600E01546844207D2802005F0EEFC9C
:10F0D000B4FBF0F100FB114068B100200096CDE9CF
:10F0E0000150002000F06AFC6946802000F0E8F83A
:10F0F000040002D006E00120F0E705498020FFF778
:10F1000065FF0446002000F087FC2046FEBD00009D
:10F11000D4A20F0008B140210160014870470000EF
:10F12000CC1F002010B506F029F820B104A140F250
:10F130006F3000F0B1FCBDE8104005F0BFBA000030
:10F140002E2E5C2E2E5C2E2E5C2E2E5C2E2E5C63C4
:10F150006F6D706F6E656E74735C6C6962726172F4
:10F160006965735C757362645C6170705F7573620E
:10F17000642E630005F0E2BA10B50C46010600F0FB
:10F180000F02092A08D200F009F8006820B12146D0
:10F19000BDE8104001F0EABB102010BD10B501061B
:10F1A00000F00F0408D5092C04D309A140F2611026
:10F1B00000F072FC134808E0092C04D304A140F2CB
:10F1C000671000F069FC0F48483000EBC40010BD28
:10F1D0002E2E5C2E2E5C2E2E5C2E2E5C2E2E5C6334
:10F1E0006F6D706F6E656E74735C6C696272617264
:10F1F0006965735C757362645C6170705F7573627E
:10F20000642E6300301F002010B5044600F00F008C
:10F21000082805D2204605F073FB204605F0C8FCFF
:10F220002046BDE8104005F08FBB000070B50C46CD
:10F23000054605F0D9FB18B105480078022801D031
:10F24000082070BD21462846BDE8704005F0D4BBBB
:10F25000F000002010B5FFF7A1FF006810BD00000E
:10F2600070B50D460646FFF799FF0446056015B1D7
:10F270006868006808E00EB1802E04D103A140F256
:10F280008B1000F009FC0020606070BD2E2E5C2EFB
:10F290002E5C2E2E5C2E2E5C2E2E5C636F6D706F9E
:10F2A0006E656E74735C6C69627261726965735CC1
:10F2B000757362645C6170705F757362642E630065
:10F2C00070B50C46054605F08FFB18B1054800786F
:10F2D000022801D0082070BD21462846BDE87040B4
:10F2E00005F0F2BCF0000020014909680847000061
:10F2F000C01F002070B57D4C0546606820B97CA118
:10F3000040F2C33000F0C8FB01F0CAFB072804D26A
:10F3100077A140F2CA3000F0BFFB2878092872D0EC
:10F3200007DC16D2DFE800F07085A98C96B2B7151D
:10F33000DA00812814D006DC0A28F0D00F28EED09D
:10F34000802806D13CE082281FD0832843D084281F
:10F350004AD0BDE8704066A140F2AB4000F09CBBD3
:10F360007048FFF72BFE6F48FFF77EFA0D200AF07A
:10F370006DFDA06810B96C48007A00B1012005F05D
:10F3800053FFFFF783FA012073E0FFF77FFA05F0E0
:10F390009FFF002009F064FF6248401CFFF764FAF9
:10F3A0006048401CFFF70AFE0E200AF04FFD20784F
:10F3B00000F0EAFA00283BD0BDE8704005F054B8F0
:10F3C0002078052803D0062803D0072830D1022052
:10F3D0004FE008204DE02078032829D105F0C0FF38
:10F3E000002825D0042044E02078032805D105F02A
:10F3F000B7FF10B1042009F033FF06F07DF80028B4
:10F4000016D0062035E06AE000200AF01FFDA4684F
:10F4100040F20E260AE02946204601F0A7FA1CB960
:10F4200042A1304600F038FB20684468002CF2D13D
:10F4300070BDFFF72BFA022009F012FF012003E054
:10F44000052009F00DFF03200AF000FD2846FFF714
:10F45000B5FD46E003200AF0F9FC3248801CFFF7B6
:10F46000ADFD3048801CFFF7FFF920780628AED1AB
:10F470000720BDE8704009F0F3BE032009F0F0FE5C
:10F4800002200AF0E3FC2846FFF7EEF92846BDE823
:10F490007040FFF793BDA878FFF780FE0446006830
:10F4A00020B913A140F2874000F0F6FA606820B955
:10F4B0000FA14FF4916000F0EFFAD4E90002294661
:10F4C00090470028B4D0A8780107B1D000F00F0110
:10F4D0000829ADD2BDE8704005F038BB08200AF01D
:10F4E000B5FC2846BDE87040FFF7BEB9F00000202B
:10F4F0002E2E5C2E2E5C2E2E5C2E2E5C2E2E5C6311
:10F500006F6D706F6E656E74735C6C696272617240
:10F510006965735C757362645C6170705F7573625A
:10F52000642E630069A20F00C01F00202E2E5C2EE7
:10F530002E5C2E2E5C2E2E5C2E2E5C636F6D706FFB
:10F540006E656E74735C6C69627261726965735C1E
:10F55000757362645C6170705F757362642E6800BD
:10F56000FFF7C2BE10B520B104A140F2272000F081
:10F5700093FABDE810400E48FFF7B6BE2E2E5C2E63
:10F580002E5C2E2E5C2E2E5C2E2E5C636F6D706FAB
:10F590006E656E74735C6C69627261726965735CCE
:10F5A000757362645C6170705F757362642E630072
:10F5B00058A20F00114601F0D9B9000070B50446F9
:10F5C00040680D46C2680AB120469047207AA8429A
:10F5D00004D20CA140F2BF2000F05EFA294620467A
:10F5E000FFF792FB05464678002408E021462846AE
:10F5F000FFF726FB007805F053F9641CE4B2B4422F
:10F60000F4D370BD2E2E5C2E2E5C2E2E5C2E2E5C26
:10F610002E2E5C636F6D706F6E656E74735C6C69BB
:10F62000627261726965735C757362645C6170704B
:10F630005F757362642E63002DE9F04180460F48C8
:10F640000E46456816E02F7A00240DE02146284634
:10F65000FFF75AFB0178414504D106B134702846C2
:10F66000BDE8F081641CE4B2BC42EFD32846FFF74A
:10F67000AFFB0546002DE6D10020F1E7F0000020A9
:10F6800070B50446406815460E4683681BB1204697
:10F690009847062809D1207AB04204D20E494FF487
:10F6A000287000F0F9F90DB1072070BD31462046F1
:10F6B000FFF72AFB05464678002408E02146284645
:10F6C000FFF7BEFA0078FFF79FFD641CE4B2B44276
:10F6D000F4D3002070BD000004F60E0003460020A5
:10F6E0005A681269002A01D0184610477047000076
:10F6F0002DE9F843044604F061FF20B92DA14FF431
:10F70000367000F0C9F9384805F0E4FC00284DD106
:10F71000364908704860886048213548FCF7D2FEB9
:10F72000334848214830FCF7CDFE3148314D803018
:10F730004CB194E80E00103080E80E002C48903058
:10F74000016821B105E005F12C010EC9F3E72A4952
:10F750000160002004F038FF18B1852801D0FEF7C1
:10F7600063FF264E00240DE0002703E000783146B9
:10F77000FFF776FD3946781CC7B24046FFF760FABE
:10F780000028F3D12146641CE4B23046FFF7BCFAEE
:10F790005FEA0008E8D1686800906946304601F0E9
:10F7A000E5F8040004D005F099FE2046BDE8F88392
:10F7B0000020FBE72E2E5C2E2E5C2E2E5C2E2E5C67
:10F7C0002E2E5C636F6D706F6E656E74735C6C690A
:10F7D000627261726965735C757362645C6170709A
:10F7E0005F757362642E630061F50E00F000002007
:10F7F000301F002058A20F00F5F20E0014A30F00D6
:10F8000040B1012808D0022809D007A140F20E20FB
:10F8100000F042B9114804E01048001D01E00F4813
:10F820000830FFF761BD00002E2E5C2E2E5C2E2EC0
:10F830005C2E2E5C2E2E5C636F6D706F6E656E7429
:10F84000735C6C69627261726965735C7573626422
:10F850005C6170705F757362642E630072A20F004A
:10F8600010B505F083FC10B105F076FC08B1082056
:10F8700010BD044804F0B8FE08B1FEF7D5FE002024
:10F8800010BD000080A20F0070B54FF0805086B010
:10F89000D0F8A810D0F8A40089B241F440430090F9
:10F8A0000BA20D2101A8FEF799FB0C4E40F21A3075
:10F8B00001AD3080002404E0285D06EB4401641CA7
:10F8C00048802846FCF709FEA042F5D806B070BD76
:10F8D00025303458253038580000000024200020FE
:10F8E00010B505F039FC20B909A140F2763000F0DE
:10F8F000D3F814480168C1F3400121B1BDE81040BC
:10F900001148FFF7F1BC016811F0010FF2D110BDF1
:10F910002E2E5C2E2E5C2E2E5C2E2E5C2E2E5C63EC
:10F920006F6D706F6E656E74735C6C69627261721C
:10F930006965735C757362645C6170705F75736236
:10F94000642E6300380400405DA20F00034808B530
:10F95000806800906846FFF7C7FC08BD58A20F00FA
:10F96000074918B1052803D300207047086870477D
:10F97000044A105C0028FAD051F8200070470000BB
:10F9800028010020B6A30F00092808D2DFE800F004
:10F99000070705070705050505000120704700203A
:10F9A0007047092808D2DFE800F0070705070707B6
:10F9B00007070500012070470020704710B508F0C8
:10F9C000E1FB012803D004A11D2000F065F8BDE88B
:10F9D000104000F04FB800002E2E5C2E2E5C2E2E14
:10F9E0005C2E2E5C2E2E5C636F6D706F6E656E7478
:10F9F000735C6C69627261726965735C7574696C61
:10FA00005C6170705F7574696C5F706C6174666F57
:10FA1000726D2E630000000010B508F0B3FB0128E2
:10FA200003D004A12B2000F037F8BDE8104000F00F
:10FA300029B800002E2E5C2E2E5C2E2E5C2E2E5C05
:10FA40002E2E5C636F6D706F6E656E74735C6C6987
:10FA5000627261726965735C7574696C5C61707007
:10FA60005F7574696C5F706C6174666F726D2E6324
:10FA70000000000072B602480168491C016070472E
:10FA80003C01002003490868401E086000D162B6AE
:10FA9000704700003C0100201CB56A46ADF800002C
:10FAA0000191002144F20200FEF790FD1CBD1028D8
:10FAB00002D31038C0B2704740F080007047000099
:10FAC000F8B51F480146446AC06A8D6CAC2802D163
:10FAD000486B0544241A1B4E0094042730882B469B
:10FAE00007EB0040184A19A106F0BBFA2246294646
:10FAF0001548FCF7F9FCE8B13088234607EB0040D5
:10FB00002A4620A106F0A5FA06F038F90028FBD114
:10FB100002F054FE2146284603F05CFD040007D0A5
:10FB20003088012101EB004022A100BF06F086FAD7
:10FB30002046F8BD3088002407EB004024A1F5E7FB
:10FB4000BC1700203002002000C00E00566572690C
:10FB50006679696E6720424C3A20416464723A20AB
:10FB60003078253038782C205372633A203078254D
:10FB70003038782C204C656E3A2030782530387833
:10FB800000000000436F7079696E6720626F6F74C8
:10FB90006C6F616465723A205372633A2030782545
:10FBA0003038782C204C656E3A2030782530387803
:10FBB000000000005265717565737420746F2063D6
:10FBC0006F707920424C206661696C6564000000AA
:10FBD0004E6F20626F6F746C6F6164657220636F2B
:10FBE0007079206E65656465642C20626F6F746C3B
:10FBF0006F616465722075706461746520636F6DF8
:10FC0000706C6574652E000011480421008801EBBA
:10FC1000004010A106F012FA06F0DEFA06F0AEF887
:10FC20000028FBD1114E64254FF47A47741C3846E6
:10FC3000A0476D1EFAD1BFF34F8F0D4801680D4AE2
:10FC400001F4E06111430160BFF34F8F00BFFDE796
:10FC500030020020526573657474696E6720626FAC
:10FC60006F746C6F616465722E000000909F0F00CE
:10FC70000CED00E00400FA052DE9FC410646C00742
:10FC80004FF000050ED0104F00240122385D009582
:10FC900000231146019505F021FF641C042CF4D3C8
:10FCA00000F064F8B0070DD5074E0024361D002281
:10FCB000305D032300951146019505F00FFF641C8C
:10FCC000042CF4D3BDE8FC81869F0F0010B50446D8
:10FCD000042803D305A12120FFF7DEFE0E480121F1
:10FCE000005DBDE8104005F06FBF00002E2E5C2EB9
:10FCF0002E5C2E2E5C2E2E5C2E2E5C636F6D706F34
:10FD00006E656E74735C626F617264735C626F6166
:10FD10007264732E63000000869F0F0010B50446C6
:10FD2000042803D305A11B20FFF7B6FE0E480021CF
:10FD3000005DBDE8104005F047BF00002E2E5C2E90
:10FD40002E5C2E2E5C2E2E5C2E2E5C636F6D706FE3
:10FD50006E656E74735C626F617264735C626F6116
:10FD60007264732E63000000869F0F0010B500249C
:10FD70002046FFF7ABFF641C042CF9D310BD000034
:10FD80002DE9F0470546861C90460F464FF00109C5
:10FD90000020FFF713FE1B4C20683860D4E90001F7
:10FDA000401AA168081A44F21C0167180EE00121EC
:10FDB000384602F02AF901F0E3FF0146384602F026
:10FDC00024F9D4E90001401AA168081A401C8642AF
:10FDD000EDD8B8F1000F03D0052065F3891002E0DB
:10FDE000062065F39F50A2682168114004EB810151
:10FDF000C8602068304420600020FFF70DFE4846B0
:10FE0000BDE8F0874021002010B543689C1844608D
:10FE100021B905E013F8010B01F8010B521EF9D2CC
:10FE2000012010BD30B482680468531C8360A15463
:10FE3000D0E901128A4202D330BC05F0C3BB30BC0A
:10FE400070470000034803C8814201D10120704778
:10FE5000002070474021002010B50548012102F024
:10FE6000EAF8BFF35F8F08B1002010BD012010BD7C
:10FE70005000002010B5064C2068012803D005A1D1
:10FE80006D20FFF709FEBFF35F8F0020206010BDDB
:10FE9000500000202E2E5C2E2E5C2E2E5C2E2E5C12
:10FEA0002E2E5C636F6D706F6E656E74735C6C6923
:10FEB000627261726965735C6D757465785C6E728F
:10FEC000665F6D74782E680004490020086004495C
:10FED0004FF48060C1F880017047000000A5025017
:10FEE00004E000E003490120086003498002C1F8F2
:10FEF0000001704700A5025004E000E070B500F179
:10FF00000806106815460C46202802D248F2145004
:10FF100070BDFFF7A1FF80B1FFF7E4FF2146304637
:10FF2000FDF702FC0646FFF7CFFFFFF7A3FF3046C1
:10FF300001F000FD060003D004E048F2045070BD5B
:10FF4000202028602021204602F090FE304670BD1F
:10FF500010B50830FDF718FCBDE8104001F0EABC10
:10FF60002DE9F04700F108090E461446FFF774FF2B
:10FF7000B8B1FFF7B7FF4FF480584546AC4200D800
:10FF800025462A4631460E48FCF774FA2A460C49A3
:10FF90004846FDF713FC0700A4EB05042E4404D0EB
:10FFA00005E048F20450BDE8F087002CE5D1FFF7EA
:10FFB0008BFFFFF75FFF3846BDE8F04701F0BABCA2
:10FFC0006006002070B50B4800240460BFF35F8F0B
:10FFD000094D01202860FDF7C1FC01002C604FF0A5
:10FFE000030004D0052901D148F2035070BD002060
:10FFF00070BD00005000002000A502500149002003
:02000004000FEB
:100000000860704700A502504360CA699A420DD348
:100010008A690260886918448861086F1844086713
:10002000C869C01AC86100D00120704701F12802D8
:10003000026000208B67704710B5040003D10649A9
:100040003920FFF729FD206818B903493A20FFF746
:1000500023FD2068083010BD6CA90F0070B50C4658
:10006000060004D1224940F2B720FFF715FD24B95C
:100070001F494FF42E70FFF70FFD207800250F2841
:1000800033D2DFE800F033083333320C1132320858
:10009000323333333300304600F09DFB26E02146F7
:1000A000304608F0A3FD0FE0304600F0C9FC0146E1
:1000B000A0780025814219D00106E1784FF00300B5
:1000C00004D531B901210CE005460FE021B1012929
:1000D0000CD00329F8D109E0304600F08DFB05462D
:1000E0000021304609F0A4FE00E00625284670BD38
:1000F0006CA90F002DE9FF5F05460198DFF8F0932A
:100100001F46017A89F800101646019800F042FB5C
:10011000804625B9F74940F2E920FFF7BDFC296880
:100120004FF0000A40F21F325446A1F21F304FF048
:10013000020B914256D04CDC40F20132A1F2013068
:10014000914272D029DC40F2F120A1F2F1228142E9
:100150006CD015DC40F2EE22A1F2EE2391426ED07B
:1001600009DC4FF43B73E1B3994270D0A1F5007103
:10017000ED395ED17AE0012B74D0022B59D19BE08E
:10018000092A70D004DC012A6ED0022A51D1B7E0CE
:100190000A2A6AD00F2A4CD1DDE00E2871D00EDC7D
:1001A00007286ED006DC01286CD005286BD0062805
:1001B0003FD116E10C2867D00D283AD138E1153827
:1001C000092836D2DFE800F0F535353535F4F3F29D
:1001D000F10013286FD010DCA0F10300102828D202
:1001E00001E02EE079E1DFE800F0F0EFEEEDEC2445
:1001F00024EBEAE9E82424E7E6E537280CD00CDC18
:10020000292878D004DC142876D0282811D125E2BA
:100210002D2872D032280CD150E244286ED006DC52
:100220003E286CD03F2804D16FE29FE04CE0492883
:10023000F4D00020C5F800A004B0BDE8F09F24E091
:1002400005E008212971002F01D82B607FE20EB153
:10025000297931700B2101242971012F06D840F230
:10026000ED2073E21CE059E03AE062E00EB129793A
:10027000315598F81410641C2971BC4205D32A60CA
:1002800065E2BAE07FE0A1E0C7E00EB1297931551F
:10029000641C85F804B0BC4202D340F2EF2055E262
:1002A0000EB129793155641C85F804B0BC4203D3E2
:1002B0004FF43C704AE2A6E10EB129793155641C35
:1002C00085F804B0BC42CCD20EB12879305598F8EC
:1002D0001900641C2871BC4202D340F2F22035E2BE
:1002E0000EB128793055641C85F804A0BC4207D3B0
:1002F00040F2F3202AE2BCE191E1CDE117E2F9E11D
:100300000EB12879305589F801A0641C35E2092026
:100310002871BC4202D340F2FA2017E20EB12879CC
:1003200030550420641C2871BC4202D340F2FB20EB
:100330000CE20EB12879305599F80110641C01982F
:10034000FEF714FDC9F8040000782871BC4202D3FE
:100350004FF44070FAE10EB128793055641C85F8ED
:1003600004A0BC4202D340F20130EFE10EB1287983
:100370003055D9F80400641CBC424078287102D37F
:1003800040F20230E2E10EB128793055D9F804008C
:1003900098F81410641C0078814233D185F804B0B9
:1003A000BC4213D340F20630D0E18BE07FE073E033
:1003B00067E054E01BE10FE103E1F7E0EBE0DFE091
:1003C000D3E0C7E0B9E0ADE0A1E095E00EB1287957
:1003D0003055641C85F804B0BC4202D340F20730AB
:1003E000B4E10EB12879305598F81900641C2871D1
:1003F000BC4202D34FF44270A8E10EB128793055C7
:10040000641C25E098F8161081421CD10A2028713E
:10041000BC4202D340F20D3098E10EB1287930553C
:10042000641C85F804A0BC4202D340F20E308DE17A
:100430000EB128793055641C85F804A0BC42DCD389
:1004400040F20F3082E12B4940F21330FFF724FBDA
:1004500085F804A0BC4202D340F2163076E10EB11A
:1004600028793055D9F8040098F81410641C0078E5
:1004700081426ED105202871BC4202D340F21B306C
:1004800064E10EB1287930552420641C2871BC42E7
:1004900002D34FF4477059E10EB128793055641CEE
:1004A00085F804A0BC4202D340F21D304EE10EB1EB
:1004B000287930551020641C2871BC4202D340F2C8
:1004C0001E3043E10EB1287930550120641C28719B
:1004D000BC4202D340F21F3038E10EB128793055CA
:1004E0000520641C2871BC4206D340F222302DE165
:1004F000040100206CA90F000EB12879305524208A
:10050000641C2871BC4202D340F223301EE10EB1BC
:10051000287930550120641C2871BC4202D34FF465
:10052000497013E10EB1287930550320641C2871FD
:10053000BC4202D340F2253008E10EB12879305593
:1005400098F81600641C2871BC4203D340F2263090
:10055000FCE069E00EB1287930550420641C287154
:10056000BC4202D340F22930F0E00EB12879305578
:100570002420641C2871BC4202D340F22A30E5E0FA
:100580000EB128793055641C85F804B0BC4202D302
:1005900040F22B30DAE00EB128793055641C85F832
:1005A00004B0BC4202D34FF44B70CFE00EB12879B7
:1005B00030550520641C2871BC4202D340F22F3014
:1005C000C4E00EB1287930552420641C2871BC4247
:1005D00002D34FF44C70B9E00EB1287930550620A3
:1005E000641C2871BC4202D340F23130AEE00EB13F
:1005F0002879305598F81400641C2871BC4202D345
:1006000040F23230A2E00EB12879305598F8160049
:10061000641C2871BC4202D340F2333096E00EB124
:1006200028793055641C08E098F81610814204D0EF
:1006300057494FF44F70FFF72FFAD9F80410484686
:10064000497889F80210514689F803A08CE0072008
:100650002871BC4202D340F2473077E00EB12879CE
:1006600030550520641C2871BC4202D34FF45270EF
:100670006CE00EB12879305599F80310641CD9F854
:100680000400FEF70FFBC9F8080000782871BC428F
:1006900002D34FF4537059E00EB128793055D9F890
:1006A000040098F81410641C007881420BD10320D8
:1006B0002871BC4202D340F2513047E00EB1287994
:1006C0003055641C0FE098F81610814206D185F869
:1006D00004B0BC42F2D340F2563037E02C4940F22D
:1006E0005A30FFF7D9F940202871BC4202D340F2BA
:1006F0005D302BE00EB128793055641C85F804A0DC
:10070000BC4202D340F25E3020E00EB12879305571
:10071000D9F8040098F81410641C007881420BD1B9
:1007200010202871BC4202D340F263300EE00EB1BB
:1007300028793055641C11E098F81610814208D1D0
:1007400085F804A0BC42F2D34FF45A70286001200F
:1007500072E50F494FF45B70FFF79EF999F80310AB
:100760004846491C89F803108278C9B29142FFF4C7
:100770006EAF4178491C89F8011099F8011099F879
:1007800000008142FFF4C3AD40F27330DEE70000A9
:100790006CA90F0010B5040003D103492C20FFF70A
:1007A0007BF9204610BD00006CA90F0010B508B100
:1007B000032010BD0846FFF73FFC0178202901D037
:1007C000062010BDD0F80210C160C1880182017AF4
:1007D0008174002010BD10B5FFF7DCFFFFF72CFC83
:1007E0000021818281610162C16601674167816781
:1007F00000F12801816610BD2DE9FC478146FFF715
:10080000C9FFFFF719FC0446484600F06AF907469D
:100810002F4800268068CDE90004E069B0B1D4F823
:1008200078804546404500D205462A4604F1280115
:10083000A069FBF71FFE206F2844C4E91C60A8EBE9
:100840000500E06660192830A06627E0206F606729
:100850002667E666216A304621B1626AA161C4E971
:1008600007202CE0A06130E004F11802616A82E800
:100870004300E26E1AB38A4215D3A36E0A461946A4
:10088000FBF7F8FDE16EE069091AE166A16E01442B
:10089000A16660670021484609F0CAFA206A00286C
:1008A000E2D1A66111E0A16EFBF7E4FDE06E2067E6
:1008B000E169091AE161A1690818A06105D06946DA
:1008C0003846FEF7B3FCBDE8FC870020FBE70000DC
:1008D000A4A20F004360CA699A4204D38A690260E5
:1008E0000B67CB6103E001F1280202608B670020F7
:1008F0007047000010B589B102291CD101220E49B0
:100900000E48FEF72FF802460D4802210088BDE888
:10091000104001EB00400BA105F094BB06490122F9
:10092000A1F1550006F004FF012203490348FEF738
:1009300019F80028F2D010BDD18A002030A40F0091
:1009400038020020436F756C64206E6F74207265EE
:1009500061642066726F6D204344432E204572729D
:100960006F723A20307825782E00000070B50D4661
:10097000040003D10BA1E120FFF78EF8606818B9DD
:1009800008A1E220FFF788F86068006818B905A19F
:10099000E320FFF781F86068294602682046BDE839
:1009A000704010472E2E5C2E2E5C2E2E5C2E2E5C60
:1009B0002E2E5C636F6D706F6E656E74735C6C6908
:1009C000627261726965735C757362645C61707098
:1009D0005F757362642E630070B5084C050009D022
:1009E00010342168002907D008682060496828462B
:1009F0008847F6E70834F4E770BD00008C1C00203F
:100A0000054A012120B1012805D19170FFF7E4BF0B
:100A100051700020FAE770478C1C002010B50400CC
:100A200003D10549C520FFF737F80448C16B616061
:100A3000006CA06010BD000000A70F00BC170020D4
:100A400010B50021FEF792F90021FEF72BF900788E
:100A500010BD40684968884201D8012070470020D5
:100A600070470000F0B54FF0FF3622B11268D24354
:100A700000230A4D0DE03246FAE7C45C62400824C8
:100A8000D70700D037462F4087EA5202641EF7D1BD
:100A90005B1C8B42F1D3D043F0BD00002083B8ED46
:100AA000EFF30580C005C00D10D0103840B200280B
:100AB00006DA00F00F0000F1E02090F8140D03E0DA
:100AC00000F1E02090F80004400970470F207047C3
:100AD00010B50121FEF74AF90021FEF7E3F800788E
:100AE00010BD10B50121FEF741F90121FEF7DAF83A
:100AF000007810BDF0B5146906468DB02068154623
:100B0000271DE0B1022920D00A2000906B4609AAD7
:100B1000304607F04BFB00280FD009A901A8009A26
:100B200007F0CAF901AE96E80F0005AE86E80F009F
:100B3000236869683A4605A898470DB0F0BD0DB026
:100B40003046BDE8F04007F02BBA6946304607F062
:100B5000BDF90028F1D0236869683A46684698478D
:100B60000028EAD002980028F5D101987060012091
:100B7000E3E753685B7813F0C00303D0402B03D046
:100B80000020704700F002B8FFF7B4BF2DE9FF4125
:100B90000B465168064614464878334D00F00F0264
:100BA00010F0300055F8225006D0102806D020282A
:100BB00008D0302856D13EE022694DE0616901201D
:100BC000087047E0022B28D1042A26D84FF00108EC
:100BD00069463046676907F079F900281AD009E0BC
:100BE0000B79226913FB00226846A84770B1387858
:100BF000401C3870029820B1616838784A79904278
:100C0000EED301987060029860BB02E04FF00008DC
:100C1000F7E7404604B0BDE8F081D4E904300F792D
:100C2000027817FB023349798A421BD2521C0270A8
:100C30001A46616810E008786169072A087009D1CE
:100C4000606801792069FBF73DFC60682169806874
:100C500007F057F92269616804B03046AC46BDE838
:100C6000F04160470020D5E75CA40F0038B51D496E
:100C700001200A68D20301D5000407E01A490A6876
:100C800012F0A90F04D0086800F056000860002098
:100C900002F020F8154C0425D0B1192000906846C8
:100CA00004F064FFD0F810050099C84010F0010F5F
:100CB00013D00D48001F006810F0B10007D0208845
:100CC0000BA105EB004000BF05F0B8F9012038BDCD
:100CD000208810A105EB0040F6E7208816A105EB5F
:100CE0000040F1E7000400402005004030020020F1
:100CF000444655206D6F6465207265717565737427
:100D00006564207669612047505245475245542E0C
:100D100000000000444655206D6F646520626563E5
:100D20006175736520617070206973206E6F742027
:100D300076616C69642E0000444655206D6F6465D1
:100D400020726571756573746564207669612062CF
:100D50007574746F6E2E0000FEB51849044608685D
:100D600008B1401E08601648D4E9015300880426E3
:100D7000227806EB00409DB10E6821690296CDE90C
:100D800000312B46012A16D00EA210A105F07CF9E5
:100D90006169002911D0E06803B0BDE8F040084760
:100DA00009680091012A04D006A217A105F059F99B
:100DB000EEE71FA2F9E71EA2E7E7FEBD58000020FC
:100DC000E40100206572617365000000466C617388
:100DD00068202573206661696C6564202830782559
:100DE00078293A20616464723D25702C206C656E10
:100DF0003D307825782062797465732C2070656E9B
:100E000064696E6720256400466C617368202573F1
:100E100020737563636573733A20616464723D2562
:100E2000702C2070656E64696E6720256400000078
:100E3000777269746500000010B508281BD2DFE8DE
:100E400000F004121A1A1A041A040120FEF714FF03
:100E50000020FEF763FF0120FEF760FFBDE81040B1
:100E60000220FEF733BF0120FEF730FFBDE810403F
:100E70000220FEF753BF10BD10B50446032806D06C
:100E8000042C04D0062C0ED0072C04D10BE007490B
:100E9000074801F0BFFA07480168002905D020463D
:100EA000BDE810400847FEF7AFFE10BD251B0F0040
:100EB000C0D401000800002010B50446062802D165
:100EC000002002F0ABFF04480168002903D020464F
:100ED000BDE81040084710BD5400002070B54278AE
:100EE00005460C46012A07D00E480221008801EB76
:100EF00000400DA105F0A6F8287808280BD16088DD
:100F0000401E81B26180208800280AD0002908D1C3
:100F100060800320287029462046BDE8704007F015
:100F200077B970BD34020020444655207265717552
:100F300065737420636F6D706C6574656420776988
:100F4000746820726573756C743A20307825780067
:100F500010B50021024801F06EF880F3100010BDBA
:100F60005C6100204FF4A07202EB810189B200F0B5
:100F7000EFBB0068D0F80405704700002DE9F0478A
:100F800015460E46040003D134492F20FEF784FD98
:100F90001EB932493020FEF77FFD1DB92F4931209F
:100FA000FEF77AFD60792E49DFF8B480DFF8B4905F
:100FB00041F82050617908F1040808EBC10000797C
:100FC00038B10824B9F80000022101EB004026A145
:100FD0003FE035882768B5F5805F03D32BA1FD205E
:100FE000FEF75AFDC7F80855B67894F90450082E54
:100FF00003D331A14520FEF74FFD002D4FEA4610E7
:1010000006DA05F00F0101F1E02181F8140D03E08B
:1010100005F1E02585F8000494F90410012201F09F
:101020001F0302FA03F04909890001F1E021C1F828
:101030008002C1F80001617908EBC1010A71617990
:1010400048F83140B9F80000032101EB00400024CA
:1010500024A104F0F3FF2046BDE8F087B8A90F00F3
:10106000400100200C02002052544320696E73742A
:10107000616E636520616C726561647920696E6977
:101080007469616C697A65642E0000002E2E5C2EF6
:101090002E5C2E2E5C2E2E5C2E2E5C6D6F64756C7D
:1010A00065735C6E7266785C68616C2F6E72665FE9
:1010B0007274632E680000002E2E5C2E2E5C2E2E85
:1010C0005C2E2E5C2E2E5C696E746567726174698D
:1010D0006F6E5C6E7266785C6E7266785F676C7558
:1010E000652E68005254433A20696E697469616CD8
:1010F000697A65642E00000090F90400012100F077
:101100001F0291404009800000F1E020C0F8001269
:1011100070470A46022100F007BB4FF4827100F0CD
:1011200017BB000010B5040003D104496120FEF78D
:10113000B3FC20680121016010BD0000B8A90F00B8
:1011400010B5040003D104496720FEF7A5FC206810
:101150000121416010BD0000B8A90F002DE9F8433E
:10116000994616460F46050003D12B498620FEF707
:1011700093FC29684FF480344FF4A070BC4000EB1E
:10118000870080B226F07F46C1F808432968C1F87D
:101190004843296800220A5008580090286800EB4C
:1011A0008701D1F84005C1F840652968D1F80415D8
:1011B0001A4F401A20F07F404FF00408012809D14F
:1011C000398808EB014016A104F038FF21494FF49B
:1011D000046088472868C0F844432968D1F804357A
:1011E000F01A20F07F40020201D540F07F40C9F1A3
:1011F000000290420BDD022809DC3988324608EBF8
:10120000014015A104F025FF0D20BDE8F883C1F8C9
:1012100004430020F9E70000B8A90F000C020020E9
:101220005254433A2044656C617920696E74726F40
:1012300064756365642064756520746F20726973DA
:101240006B206F66207072652D666972696E672EFD
:1012500000000000C1A30F005254433A2057696EAA
:10126000646F77656420636F6D706172652073656C
:10127000742074696D656F757420286162735F7680
:10128000616C75653A25642C20636F756E746572A8
:101290003A2564292E00000010B50446010600F02E
:1012A0000F00092804D306494FF42B70FEF7F4FB16
:1012B0006FEA0460C10F204661F31F1010BD0000EB
:1012C000A09A0F0070B50546000605F00F0402D580
:1012D000092C09D301E0092C08D307A140F2992079
:1012E000FEF7DAFB280601D5124801E011489038D4
:1012F00000EB041070BD00002E2E5C2E2E5C2E2EF6
:101300005C2E2E5C2E2E5C636F6D706F6E656E743E
:10131000735C647269766572735F6E72665C757316
:1013200062645C6E72665F6472765F757362642E6F
:1013300063000000301D002010B50446010600F0D7
:101340000F00092804D303494FF41F70FEF7A4FBD4
:10135000204610BDA09A0F002DE9FC4180461F4693
:1013600015460E4600240D4800F04CFE38B1112001
:10137000BDE8FC8106EB043005F006F8641CAC42C5
:10138000F8D1064800F035FECDE90057334600227B
:101390000221404600F0ACF90020E9E74C010020B2
:1013A00010B508F057FB8020FFF78CFF817B0124EC
:1013B000032902D00068002809D18020FFF76CFFC4
:1013C0008440E143BDE81040014800F024BE10BD58
:1013D0008C000020812005F069B9822005F066B9F3
:1013E000832005F063B9842005F060B9852005F0FD
:1013F0005DB9862005F05AB9872005F057B98820D5
:1014000005F0A4B938B508F025FB0020FFF75AFF16
:10141000817B0124032905D0006868B1BDE838400C
:1014200003F0C1BE0020FFF737FF8440E143BDE871
:1014300038400A4800F0EFBD0020FFF72DFF844040
:10144000E143064800F0E7FD05480449C0680C394F
:10145000009049686846884738BD00008C0000202D
:1014600060A10F00012005F0B3B9022005F0B0B96A
:10147000032005F0ADB9042005F0AAB9052005F058
:10148000A7B9062005F0A4B9072005F0A1B900000E
:1014900038B5082408F0DEFA2046FFF713FF817BF9
:1014A000032915D00068002812D12046FFF7F4FE6A
:1014B00001218140C943074800F0ADFD06480549B8
:1014C000406900900C398DF80240496868468847A9
:1014D00038BD00008C00002060A10F0070B51548D9
:1014E00004680460BFF36F8FBFF34F8FBFF36F8F3C
:1014F000BFF34F8F03F0ACFC38B10F48016921F006
:10150000011201F001111443016101266CB194FA3A
:10151000A4F0B0FA80F52846FEF7C9FA06FA05F1FC
:101520008C43294608F02EFCF0E7BDE8704008F037
:10153000D5BA00006C7402408000002010B5054C44
:10154000A078FFF7A9FE0146A078BDE8104008F09A
:1015500019BC000080000020F8B51A4800681A4D38
:10156000C6B2A878FFF798FE012404FA00F1288992
:10157000EA68C04380B21043014202D0A87808F064
:1015800079FB06F08000A8700020FFF785FE04FAC2
:1015900000F68020FFF780FE04FA00F006430A48B8
:1015A000F1430C3000F037FD8020FFF775FE8440DA
:1015B000A86804430548AC60006A00906968684602
:1015C0008847F8BD807402408000002060A10F00B1
:1015D00038B5002000900B480068ADF80200882064
:1015E000FFF75AFE012505FA00F40820FFF754FE24
:1015F000054985402C43886804438C6049686846E7
:10160000884738BD207502408000002070470000E8
:10161000F8B51C480568284605F080F9BFF36F8FC0
:10162000BFF34F8F184E194CE80506D501206070A6
:10163000706A0090616868468847A8054FF0000707
:1016400005D56770B06A009061686846884768058C
:1016500016D56078002813D005F06AF920B10CA1E6
:1016600040F2C540FEF718FA67701849012008607B
:10167000582005F065F9F06A00906168684688476F
:10168000F8BD00000074024060A10F00800000203F
:101690002E2E5C2E2E5C2E2E5C2E2E5C2E2E5C634F
:1016A0006F6D706F6E656E74735C6472697665726F
:1016B000735F6E72665C757362645C6E72665F64A3
:1016C00072765F757362642E6300000008750240D5
:1016D000054908B5002048708870044840680090AB
:1016E00049686846884708BD8000002060A10F0057
:1016F0002DE9F04387B00446DDE90E8980681D4678
:1017000016460F4600280BD018216846FAF7DAFE75
:1017100002A88DF8007080E86003A16868468847D9
:1017200007B0BDE8F083000070B516460C46050012
:1017300003D10649B920FEF7AFF92868C0F8444341
:10174000002E02D02868C0F8044370BDB8A90F006D
:1017500038B50C46050003D10749CA20FEF79CF9AD
:101760002868015929B10021015100590090012038
:1017700038BD002038BD0000B8A90F000B2803D3E6
:101780000B38C0B200F00AB87047000002490022CE
:1017900008780A70704700005C000020014908705A
:1017A0000B2070475C000020014901200870704741
:1017B000490000202DE9FE4307004FF0200090462D
:1017C00089464FF00106029004D12A494FF4FA707D
:1017D000FEF762F9284C0425434620884A4605EB6B
:1017E000004026A104F035FC02A93348CDE90001F0
:1017F00043464A463149A0F59A7001F047F9020084
:1018000007D02088012101EB00402DA104F01AFC33
:101810002CE007F16F0120220F462748FAF764FEFB
:1018200028B32088022101EB004032A104F006FC1D
:10183000208837A105EB004004F000FC208820221E
:1018400005EB0040394604F0A5FB208835A105EBE7
:10185000004004F0F3FB2088202205EB00401649ED
:1018600004F098FB04F08AFA0028FBD100263046E9
:10187000BDE8FE8394A80F00F00100204861736862
:1018800020766572696669636174696F6E2E2046A1
:1018900069726D776172652073746172742061641E
:1018A00064726573733A20307825782C2073697AD6
:1018B000653A2030782578006C1C0020CC9F0F0002
:1018C000436F756C64206E6F742072756E20686152
:1018D000736820766572696669636174696F6E20EA
:1018E000286572725F636F64652030782578292ED1
:1018F000000000004861736820766572696669635C
:101900006174696F6E206661696C65642E00000009
:101910004578706563746564204657206861736814
:101920003A00000041637475616C2046572068617D
:1019300073683A0010B50F4C48F20351031B48F28C
:101940001652A04211D007DC00280AD00A4BC0185A
:1019500008D0012804D10BE00A2B01D00D2B07D0B1
:10196000104610BD48F2015010BD48F2025010BDA3
:10197000084610BD0202F00000FE0FFF2DE9FC5FDB
:101980000646DFF804A1984615460F464FF0040BB3
:10199000B1420BD1BAF8000033460BEB00403A4697
:1019A0003AA104F056FB0020BDE8FC9F04D2434955
:1019B0004FF02900FEF770F8B8F1000F03D13F494E
:1019C0002A20FEF769F8300503D03C492B20FEF7AA
:1019D00063F8B81B040B03D138492E20FEF75CF8DE
:1019E0000020009005F6FF704FEA103900F0F8FE75
:1019F0004046A04500D20446A04641E04946C145C4
:101A000004D808462C46CDF8049004E040464FEA3E
:101A10000834CDF8048001460022304601F096FCDF
:101A20000028C1D10094BAF8001033460BEB0140F6
:101A30003A4623A104F015FB601E00F00300221AB1
:101A4000002339463046D21C01F012FD0028ABD1EC
:101A500001992448A9EB01092D1B016B264421445F
:101A600001632744002002F0E3F8009040B1BAF887
:101A70000000012101EB00401BA104F0DFFA01E0AE
:101A8000002DBBD100988FE7300200204E6F2063FD
:101A90006F7079206E6565646564207372635F6141
:101AA0006464723A20307825782C206473745F6106
:101AB0006464723A203078257800000054A50F0045
:101AC000436F7079696E67203078257820746F20B5
:101AD000307825782C2073697A653A20307825781B
:101AE00000000000BC1700204661696C656420742A
:101AF0006F20777269746520696D61676520636F17
:101B00007079696E672070726F6772657373207485
:101B10006F2073657474696E677320706167652EDA
:101B20000000000004480321008801EB004003A1ED
:101B300004F084FAFEF768F830020020496E616311
:101B40007469766974792074696D656F75742E0097
:101B50000149416000207047D8A30F002DE9FC5FC8
:101B60000E008346DDE90C47C6F100009846924618
:101B7000814600D40846012503E000BF90FBFAF03F
:101B80006D1C5045FADAA84500D9454624B1002E0F
:101B900001DB780700D5641EB80702D5B8F1000F45
:101BA0000AD0F80708D13CB1A54205D220215846F9
:101BB000641EFEF737F9F6E7002E02DA4E462D21B5
:101BC00002E0780703D52B215846FEF72BF907F0E2
:101BD000030002280BD1B8F1000F08D13CB1A54297
:101BE00005D230215846641EFEF71CF9F6E7CDE910
:101BF0000047434652463146584607F071FCBDE85F
:101C0000FC9F000010B5024600201268930702D026
:101C1000530702D410BD500719D502F00300012864
:101C200007D002280BD00D494FF49170FDF734FF17
:101C30000BE0C2F383100B68801C184404E00223FD
:101C4000086803EB925210440860012010BD086838
:101C500000EB9253C2F38910401CEEE798AA0F00E4
:101C600002480068002800D0012070474C01002085
:101C700038B54FF440531A4A5D6800F5005195425B
:101C800004D04868904201D1012400E0002495422C
:101C900024D14868904221D11878142801D95A6972
:101CA00000E000220F48B2FBF0F30A78142A01D9B1
:101CB000496900E00021B1FBF0F0834203D0012428
:101CC00009A2009002E0002409A200900A48032122
:101CD000008801EB004009A104F0C3F9204638BD9B
:101CE000DBE5B15140420F006D616A6F7200000088
:101CF0006D696E6F72000000F0010020536F667412
:101D000044657669636520757064617465206973E4
:101D100020612025732076657273696F6E2075705F
:101D2000646174652E2043757272656E743A202565
:101D3000642E204E65773A2025642E0002681346F3
:101D400002E08A4204D01268002AFAD10B600160D6
:101D5000704770B5054608680C464A68866828468C
:101D6000314605F0EFFF6068286104F10C006861FE
:101D700070780221B1EB901F01D1241D2C6170BD40
:101D80002DE9FF410026264800F039F92448001FBC
:101D9000074600F034F9234C60680090A56800E025
:101DA00000986946284004EB80000C30FFF72AFFBA
:101DB0000028F5D101AA009901EA050304EB830389
:101DC000491CDB6842F82030401C00910228F2D305
:101DD000019800F0030001281AD002280ED0124901
:101DE0004FF4AF70FDF758FE384600F005F908B122
:101DF0000098606004B03046BDE8F081019803218E
:101E000001EB90500099BDF80A6001EB900005E0ED
:101E10000198BDF80A60C0F3831008440090E3E71E
:101E2000586100204021002098AA0F0070B50022C0
:101E30004FF48051104600F0F5FAC8B9124800225C
:101E4000C0F57E2100F0EEFA90B94FF400410F4842
:101E500004F07EF903F07CFF0D4C03250DA12088D2
:101E600005EB004004F0EAF80D4800F0F7FB08B17C
:101E7000FCF7DAFB00F0EAF920880AA105EB004044
:101E800004F0DCF8002070BD00C00E0069E70E0011
:101E900030020020496E73696465206D61696E00CF
:101EA000390E0F004166746572206D61696E000025
:101EB0002DE9F05FC7888A46191D1646B1FBF7F277
:101EC000B1FBF7F507FB121999193944C91CB1FB8D
:101ED000F7F104464079C9B2DDF828B0884206D24D
:101EE00017499420FDF7D8FD01E024686D1E002DF0
:101EF000FBD1A846A7EB0905B5421AD81CE000BFE4
:101F0000BBF1000F06D004EB09010AEB08002A46DA
:101F1000091D05E004EB09000AEB08012A46001D33
:101F2000FAF7A8FA2468761B4FF00009A844B742D4
:101F300001D9354600E03D46002EE1D1BDE8F09FD5
:101F4000FCA90F0030B5024659B104F02DF900216B
:101F5000074C09E004EB810315685B88AB4202D1B2
:101F60001160002030BD491C8142F3D3052030BDF3
:101F7000D801002010B531B1B2FBF3F403FB1424F7
:101F80001CB1092010BD0E2010BD01600021416070
:101F900081608281C381084610BD70B50C4605463C
:101FA000FAF73CF9002802D021882868084470BD5F
:101FB00010B50A8849888A4203D1FAF771F90120DD
:101FC00010BD002010BD70B50C460546FAF74BF960
:101FD000002802D061882868084470BD10B50A88BE
:101FE00049888A4203D1FAF735F9012010BD002053
:101FF00010BD002100F00FB8002100F012B801213F
:1020000000F01EB8012100F011B808B56A46FAF7D1
:102010009CF9009808BD08B56A46FAF77CF9009863
:1020200008BD08B56A46FAF776F908BD08B56A46EC
:10203000FAF764F908BD08B56A46FAF753F908BD1E
:1020400008B56A46FAF75AF9009808BD08B56A4615
:10205000FAF788F9009808BD70B5040003D113A100
:10206000FE20FDF719FD00252846FDF7A7FC206896
:1020700062680168914214D9491E01600D781CB94B
:1020800018A1C220FDF708FDA08AE16805FB001534
:102090002068217A0278891A0279C9B28A4200D26C
:1020A00001710020FDF7B8FC284670BD2E2E5C2E75
:1020B0002E5C2E2E5C2E2E5C2E2E5C636F6D706F50
:1020C0006E656E74735C6C69627261726965735C73
:1020D00062616C6C6F635C6E72665F62616C6C6F88
:1020E000632E63002E2E5C2E2E5C2E2E5C2E2E5C1C
:1020F0002E2E5C636F6D706F6E656E74735C6C69B1
:10210000627261726965735C62616C6C6F635C6E54
:1021100072665F62616C6C6F632E630070B50C4613
:10212000050004D110A140F22110FDF7B5FC24B93F
:102130000DA14FF49170FDF7AFFC0020FDF73EFCC0
:102140001DB91749CF20FDF7A7FCE8682A68211AB6
:10215000A88AB1FBF0F11068431C13600170BDE860
:1021600070400020FDF758BC2E2E5C2E2E5C2E2ECB
:102170005C2E2E5C2E2E5C636F6D706F6E656E74C0
:10218000735C6C69627261726965735C62616C6CCC
:102190006F635C6E72665F62616C6C6F632E63006E
:1021A000E4200F0010B5040002D0206830B901E02F
:1021B0000E2010BD17A1D920FDF76EFC606818B97C
:1021C00014A1DA20FDF768FCA06818B911A1DB2082
:1021D000FDF762FCE06818B90EA1DC20FDF75CFC9D
:1021E000A08A18B90BA1DD20FDF756FC207A6168A2
:1021F0002268401AC0B2116004E0226811684B1CCA
:1022000013600870401EC0B2F7D221680020087128
:1022100010BD00002E2E5C2E2E5C2E2E5C2E2E5C11
:102220002E2E5C636F6D706F6E656E74735C6C697F
:10223000627261726965735C62616C6C6F635C6E23
:1022400072665F62616C6C6F632E63002DE9F04112
:10225000164C4FF4805204272088154607EB0040A7
:1022600013A103F0EFFE4FF0E026D6F8802120887E
:102270001DA107EB004006F5C07603F0E3FE7017E2
:102280003060C6F8000101F0B1F930B120880121B9
:1022900001EB00401FA103F0D1FE03F06FFD002809
:1022A000FBD12846BDE8F04100F050B830020020D4
:1022B00052756E6E696E67206E72665F626F6F74C4
:1022C0006C6F616465725F6170705F73746172746A
:1022D000207769746820616464726573733A203092
:1022E000782530387800000044697361626C696E4B
:1022F0006720696E74657272757074732E204E5605
:1023000049432D3E494345525B305D3A20307825A4
:10231000780000004661696C65642072756E6E69B4
:102320006E67206E72665F6466755F6D62725F696C
:1023300072715F666F72776172645F616464726507
:1023400073735F73657428290000000070B506463A
:102350001F4888B0C0F58011002200F063F8021E0B
:102360004FF0FF3507D01B480121008801EB0040EA
:1023700019A103F067FEEFF30580D6E90046C0051A
:10238000C00D4FF0000181F3148881F3108881F3B0
:10239000118881F3138813D020221D496846FAF76B
:1023A00069F8203C2022694620460696FAF762F832
:1023B0006FF0060229462046F9F72CFF08B070BDE1
:1023C00008B0324629462046BDE87040F9F722BFE2
:1023D00000C00E0030020020436F756C64206E6FE9
:1023E000742070726F7465637420626F6F746C6FA9
:1023F0006164657220616E642073657474696E67D0
:10240000732070616765732C20307825782E00006A
:10241000989F0F000A4601460148006807F022B85D
:10242000B89F0F0070B50B0502D1B0F57F2F01D911
:10243000072070BD0AB1062500E00225104A114BA5
:102440001468082C01D3042070BD03EB0416C6F8F1
:102450000008C6F80418C6F80858641C146003EB9A
:102460000414D4F8F0678642EAD1D4F8F4678E42B7
:10247000E6D1D4F8F847AC42E2D1002070BD0000AC
:102480000C00002000E001402DE9F0473D4C042500
:102490003B4E2088002705EB00403BA103F0CEFD1A
:1024A000B06801280FD0A52816D0AA281DD0AC28C6
:1024B000208824D0032101EB00403CA103F0BEFDA5
:1024C0000020BDE8F08720883FA105EB004003F025
:1024D000B5FDFBF7FFFF10E020883EA105EB0040B3
:1024E00003F0ACFD06F012F810E020883CA105EBEB
:1024F000004003F0A3FDFDF7E3FA024608E005EB18
:1025000000403AA103F09AFD06F0D0F802460127F8
:102510004FF0010932B12188B36809EB014037A1BE
:1025200003F097FD304600F067FCDFF804810021DE
:1025300088F800103F4801F07BFB064698F8000041
:1025400020B93D4940F27910FDF7A6FA46B121883D
:1025500009EB014039A103F071FD03263046B0E7D5
:102560000126002FFAD0012000F0B4FB0028F5D09E
:102570002088394905EB004003F060FD0226EDE7B5
:10258000E017002030020020456E746572206E72E4
:10259000665F626F6F746C6F616465725F66775FB0
:1025A0006163746976617465000000004E6F206697
:1025B00069726D7761726520746F206163746976EA
:1025C0006174652E0000000056616C6964204170E2
:1025D0007000000056616C696420534400000000E4
:1025E00056616C696420424C0000000056616C69C1
:1025F00064205344202B20424C0000004163746946
:10260000766174696F6E206661696C6564207769B4
:102610007468206572726F72202564202862616E72
:102620006B20636F64653A203078257829000000BC
:1026300049000020A9170F0054A50F00436F756CC7
:1026400064206E6F7420777269746520736574748A
:10265000696E67732E000000ECA50F00F8B5364CCC
:1026600005460426208835A106EB004003F0E6FC71
:102670003848056019200090684603F077FA009A00
:10268000354900EB8200C0F80017002001F03AFA4B
:10269000002844D1FFF7F8FE20B1012820D00228FD
:1026A0003DD104E02D4DFEF7E1FA10B934E042F2DD
:1026B000107500F095F82A4A20211820FCF73EF802
:1026C00008B1FBF7B1FF2748016811F0B10F03D043
:1026D000016801F04E01016000F060FFF8B901E00F
:1026E000FDF792FA20492846FFF794FE1F4800F0B4
:1026F0000DFFA0B920881EA106EB004003F09EFC50
:1027000000F05CF8FBF7FAFF03F038FB0028F7D184
:1027100020BF40BF20BFF3E701F0D0F908B103208C
:10272000F8BDFFF793FD2088012101EB004014A1C3
:1027300003F084FCF3E7000030020020496E206EB5
:1027400072665F626F6F746C6F616465725F696EF1
:1027500069740000080000200C000300C0D40100D0
:10276000400200201C050040251B0F00790E0F00C1
:10277000456E746572206D61696E206C6F6F7000BC
:1027800053686F756C64206E6576657220636F6D3B
:102790006520686572653A204166746572206E72C4
:1027A000665F626F6F746C6F616465725F61707099
:1027B0005F737461727428290000000010B504F082
:1027C000CBF8002803D0BDE8104007F057BB10BD80
:1027D0000A4601460148406806F044BEB89F0F0013
:1027E0002DE9F041224C207800283FD104F0B4F8C4
:1027F000204E03274FF0010800282FD01E48006804
:102800001EA1450930882A4607EB004003F01AFC58
:1028100005EB4500850842F21070854201D2012087
:1028200000E00020607007F029FB607820B91248B2
:1028300008300068C0070AD030882A4607EB0040FD
:1028400014A103F0FFFB1F492846FFF7C1FF4FF01B
:10285000E0214FF48030C1F8000105E030881AA172
:1028600007EB004003F0EAFB84F80080BDE8F0814C
:102870004A000020E0010020040501405744542094
:10288000656E61626C6564204352563A2564206D22
:10289000730000005374617274696E672061207464
:1028A000696D657220282564206D732920666F721A
:1028B0002066656564696E67207761746368646F1C
:1028C000672E0000B99E0F00574454206973206E94
:1028D0006F7420656E61626C6564000000F1804079
:1028E0000068002800D00120704708B500F1804042
:1028F000002101600068009008BD70B504460D46D7
:102900002022083000F078F9202205F1200104F19E
:10291000280000F071F9002070BD0000F0B599B0FA
:102920000D4621491E9E944607460160202B00D388
:1029300020231C461A46614611A800F05DF92022AA
:10294000314601A800F026F918480121FFF773FB72
:10295000BFF35F8F002618B148F2045019B0F0BDE4
:10296000FDF7C0FA11AB01AA05F108013846009441
:10297000FAF7C6FE0446FDF7A7FA0C4D28680128B1
:1029800003D00BA16D20FDF787F8BFF35F8F2E609A
:1029900044B11448C44202D148F24250DEE748F242
:1029A0001650DBE70020D9E7DD55AABB5000002018
:1029B0002E2E5C2E2E5C2E2E5C2E2E5C2E2E5C631C
:1029C0006F6D706F6E656E74735C6C69627261724C
:1029D0006965735C6D757465785C6E72665F6D7445
:1029E000782E68007CF70FFF70B516460C4605463A
:1029F00000F0E9F800280ED1AA791946304600F017
:102A0000EFF8002807D131462046FFF776FF00286F
:102A100001D10149216070BD7052464D2DE9F84F3A
:102A20006C460E46D4E90A7905469A469046164900
:102A3000304600F0BCF80028A54611D17068494620
:102A400040794200384600F0CBF80028A54607D16F
:102A5000B8F1000001D02DB107E0A54648F21050B2
:102A6000BDE8F88FAAB06D464DB182B0024653461C
:102A7000314628460097FFF751FFA546F0E748F298
:102A80001550A546ECE700007052464D2DE9F04187
:102A90001D46DDE906871646044600F02DF800289D
:102AA0000DD12A463146204600F03CF8002806D1D8
:102AB0003A4641462046BDE8F04100F002B8BDE884
:102AC000F08170B515460E46044607F0C7F9002898
:102AD00007D13EB160682968C268914205D248F2C8
:102AE000145070BD48F2135070BD83682A463146B9
:102AF0002046BDE87040184710B550B161B1416043
:102B0000096804468847002802D105482060002053
:102B100010BD48F2015010BD48F2105010BD000029
:102B20006E52464870B515460E46044607F096F9B3
:102B300000280BD146B155B160682A46314643683A
:102B40002046BDE87040184748F2105070BD002084
:102B500070BD00002DE9F0410B480C4D0C4F401B9F
:102B6000C60801203870002406E000BF55F8340084
:102B70008047002805D1641CB442F7D30220387086
:102B80000020BDE8F0810000A8AE0F00A0AE0F004D
:102B90004C00002070B514460D46064600F02CF897
:102BA000291930192246BDE8704000F025B828B137
:102BB0000068884205D048F24050704748F21050F3
:102BC00070470020704728B139B10022C1E90020C8
:102BD0001046704748F21050704748F21350704743
:102BE00020B1914205D048F21150704748F2105080
:102BF000704700207047000070B516460C4605006F
:102C000003D10AA11F20FCF747FF1CB907A1202010
:102C1000FCF742FFA919491E04E000BF14F8010B9C
:102C200001F80109A942F9D270BD00002E2E5C2ED8
:102C30002E5C2E2E5C2E2E5C2E2E5C636F6D706FC4
:102C40006E656E74735C6C69627261726965735CE7
:102C500063727970746F5C6E72665F6372797074A0
:102C60006F5F7368617265642E63000070B50D4616
:102C7000040003D107A10D20FCF70EFF6019401ED0
:102C800005E02178027804F8012B00F80119A04230
:102C9000F7D270BD2E2E5C2E2E5C2E2E5C2E2E5C5E
:102CA0002E2E5C636F6D706F6E656E74735C6C69F5
:102CB000627261726965735C63727970746F5C6E65
:102CC00072665F63727970746F5F73686172656456
:102CD0002E6300002DE9F041174C0746042520889B
:102CE00016A105EB004003F0A9F91B4E306A01283C
:102CF00004D0208819A105EB00400FE09FB1F069D6
:102D000088B100F055F80022B169FDF7ABFEF1691A
:102D1000814208D0208819A105EB004003F08EF90C
:102D20000020BDE8F081208819A105EB004003F0E8
:102D300085F90120F5E7000030020020456E74653A
:102D400072206E72665F6466755F6170705F697332
:102D50005F76616C69640000BC1700205265747571
:102D6000726E2066616C736520696E2076616C6995
:102D7000642061707020636865636B0052657475D0
:102D8000726E2066616C736520696E204352430049
:102D900052657475726E20747275652E2041707064
:102DA000207761732076616C69640000AFF3008066
:102DB0004FF44050074A4168914207D18068411E54
:102DC000C1F30B01401A00F6FF7070474FF48050BA
:102DD00070470000DBE5B15100B5FFF7E9FF054999
:102DE00089690A18401E0844C0F30B00101A00F647
:102DF000FF7000BDBC1700200021016041608160B0
:102E00000148016370470000BC1700202DE9FF5FF7
:102E1000854D042485A1288804EB004003F00EF9B9
:102E200028888AA104EB0040009A03F00BF901986E
:102E300008B18CA200E08DA228888EA104EB00408E
:102E400003F000F9029808B186A200E087A2288862
:102E50008DA104EB004003F0F5F8039808B181A2BE
:102E600000E082A228888CA104EB004003F0EAF87D
:102E70004FF4405041688E48814201D179A200E070
:102E80007AA228888BA104EB004003F0DBF82888A5
:102E90008CA104EB004003F0D1F88E4E28888EA15F
:102EA00004EB0040B369326A03F0D3F8288892A19A
:102EB00004EB0040736AF26A03F0CBF84FF00008AD
:102EC000DFF854B2A946A2461AE00127C0B1012892
:102ED00020D0B8F1020F2CD09049A420FCF7DCFDE3
:102EE00000255D4503D98D49A920FCF7D5FD8C4807
:102EF0000099401BA0F5405088421DD201261CE0DD
:102F0000FFF76AFF0546029888B17248006A0128F7
:102F10000BD00CE0FFF74CFF0546039828B94FF49F
:102F2000405041686248814201D00127D9E700271B
:102F3000D7E74FF48055D4E700260198B9F8001080
:102F400046EA00040AEB0140424676A103F07AF813
:102F5000B9F800102A460AEB014075A103F072F897
:102F60000EB140A200E041A2B9F800104D460AEBB4
:102F7000014075A103F066F80FB13AA200E03BA250
:102F80002888A94655460AEB004075A103F05AF877
:102F90000CB134A200E035A2B9F8000075A105EB30
:102FA000004003F04FF8BC4308D0B8F1020F05D23F
:102FB00008F10100C0B28046022886D95EB1B9F896
:102FC0000000022101EB00406FA103F037F804205C
:102FD00004B0BDE8F09FB8F1020F09D3B9F80010B2
:102FE0000AEB014073A103F029F800F0D3FE02E0E0
:102FF000B8F1000F0AD0B9F800100AEB014074A133
:1030000003F01CF833481830FFF7F6FE314A002071
:1030100010610120506102F12400FFF7EDFE0098DD
:1030200050620020D4E7000030020020456E746535
:1030300072206E72665F6466755F63616368655F68
:103040007072657061726528290000007265717583
:10305000697265645F73697A653A20307825782EE5
:1030600000000000747275650000000066616C73FA
:103070006500000073696E676C655F62616E6B3A34
:103080002025732E000000006B6565705F61707015
:103090003A2025732E0000006B6565705F736F66C4
:1030A000746465766963653A2025732E000000001C
:1030B000DBE5B15153445F50524553454E543A20DD
:1030C00025732E0042616E6B20636F6E74656E74A3
:1030D000733A0000BC17002042616E6B2030206301
:1030E0006F64653A203078253032783A2053697A17
:1030F000653A20307825780042616E6B203120637C
:103100006F64653A203078253032783A2053697AF6
:10311000653A20307825780000900E004CA70F000B
:1031200000C00E00706173733A2025642E00000009
:1031300063616368655F616464726573733A2030CC
:103140007825782E0000000063616368655F746F06
:103150006F5F736D616C6C3A2025732E0000000068
:103160006B6565705F6669726D776172653A20257F
:10317000732E000064656C6574655F6D6F72653AEF
:103180002025732E0000000041626F7274696E6723
:103190002E2043616E6E6F7420666974206E6577B1
:1031A000206669726D77617265206F6E2064657646
:1031B00069636500496E76616C69646174696E6704
:1031C00020536F66744465766963652E00000000C5
:1031D000496E76616C69646174696E6720617070B4
:1031E0002E00000070B50C46050004D1224940F2C3
:1031F0002D10FCF751FC24B91F494FF49770FCF7D0
:103200004BFC2A7804201D49092A2DD2DFE802F060
:103210002C052C0B182C1E2C120021462846BDE82C
:10322000704003F0B1BD098800EB014014A102F029
:1032300005FF14E021462846BDE8704003F03EBE7D
:1032400021462846BDE8704003F0DABD098800EB4E
:10325000014014A102F0F2FE4FF48070E0602046BD
:10326000BDE87040FDF7DABBBDE87040024940F2AE
:103270004D10FCF711BC000000A70F00E801002072
:1032800048616E646C65204E52465F4446555F4F00
:10329000505F4352435F4745542028636F6D6D6113
:1032A0006E64290048616E646C65204E52465F442E
:1032B00046555F4F505F4F424A4543545F53454C1C
:1032C0004543542028636F6D6D616E6429000000D2
:1032D00070B50E46040004D11B4940F24620FCF7AD
:1032E000DBFB26B9184940F24720FCF7D5FB2078D4
:1032F0000125092820D2DFE800F01F051F0F141F49
:103300001A1F0A003146204603F062FE19E03146DA
:10331000204604F0A7F814E03146204603F01CFED6
:103320000FE03146204603F067FF054609E03146CD
:10333000204604F04FF804E003494FF41A70FCF7FC
:10334000ABFB284670BD000000A70F002DE9F84335
:10335000134C0746134E20680D4600903088042118
:10336000904601EB00402B463A460FA102F079FE51
:1033700043462A4639461C4802F078FA05000AD02E
:103380003088022101EB00402A4618A102F05AFEC3
:103390002846BDE8F8832068401C2060F8E700005C
:1033A00058000020E40100206E72665F6673746F3F
:1033B000726167655F657261736528616464723DFF
:1033C000307825702C206C656E3D25642070616717
:1033D0006573292C20717565756520757361676546
:1033E0003A20256400000000C40100206E72665F70
:1033F0006673746F726167655F65726173652829B2
:10340000206661696C6564207769746820657272F2
:103410006F7220307825782E00000000074810B524
:103420000088042101EB004005A102F007FEBDE881
:1034300010400D4900220D4802F078BAE401002046
:10344000496E697469616C697A696E67206E72662B
:103450005F6673746F726167655F6E766D6320621D
:1034600061636B656E642E00E4A30F00C40100204D
:103470002DE9FC47154C8046154E20680F46CDE9D6
:103480000020308804219946154601EB00403B4658
:103490004246104902F0EEFD2B463A4641460E48A0
:1034A000CDF8009002F09EFA05000AD03088022183
:1034B00001EB00402A4609A102F0C4FD2846BDE800
:1034C000FC872068401C2060F8E7000058000020BE
:1034D000E401002048A60F00C40100206E72665F60
:1034E0006673746F726167655F77726974652829A6
:1034F000206661696C656420776974682065727202
:103500006F7220307825782E0000000070B51049C9
:10351000104D08602888032101EB00400EA102F045
:103520008DFD0020FDF7C8FC104800F0D5FC04001C
:1035300009D02888012101EB004022460CA102F0AD
:1035400081FD204670BDBDE87040084800F0CEB84F
:103550005400002030020020456E746572696E6769
:1035600020444655206D6F64652E0000B90E0F0093
:10357000436F756C64206E6F7420696E6974616C42
:10358000697A6520444655207472616E73706F725B
:10359000743A20307825303878000000054810B59E
:1035A0000088042101EB004003A102F047FD002048
:1035B00010BD000030020020696E207765616B202D
:1035C0006E72665F6466755F696E69745F75736558
:1035D000720000001FB58908002201AB009283E849
:1035E0000700684618DF04B010BD00002DE9FF4158
:1035F000114E04274FF48055308810A107EB00408E
:1036000002F01CFD134A1069D2E90612CDE900054B
:10361000CDE90212684618DF0446072802D1680483
:103620000024056030880CA107EB004002F006FD85
:1036300004B02046BDE8F0813002002072756E6E45
:10364000696E6720697271207461626C65207365B0
:1036500074000000FCA00F00416674657220727552
:103660006E6E696E6720697271207461626C65208C
:103670007365740070B50E460178124C062901D0AE
:10368000012901D1017C21702178012501290FD068
:10369000022911D00C480121008801EB00400BA148
:1036A00002F0CCFC0020207005207070284670BD10
:1036B0003146FFF797FDF9E73146FFF709FE05466A
:1036C000F4E7000060000020E8010020496E766108
:1036D0006C6964206F626A65637420747970652018
:1036E000696E20726571756573742E0010B50400E3
:1036F00011D00020FFF792FE00280BD100F046FC0D
:1037000000F05CFD48B10949081F00F0CDFC01281C
:1037100003D0032010BD072010BD04480838C46042
:103720000020FEF73BF8002010BD000068000020DC
:1037300010B5816879B1094A1821FAF791FF0400A0
:1037400007D007480221008801EB004005A102F0E4
:1037500075FC204610BD072010BD000081370F000A
:10376000E80100205363686564756C6572207261BE
:103770006E206F7574206F66207370616365210021
:10378000AFF30080F0B50446806887B020B94649A1
:103790004FF42870FCF780F9182244496846F8F77E
:1037A00069FE20788DF8000022780426404F414DB4
:1037B0000D2A5AD2DFE802F0075237525259523ED0
:1037C000522D0F28480028883BA106EB004002F04C
:1037D00035FC012024E0288840A106EB004002F0DF
:1037E0002DFC4FF08050D0F800110191D0F8041159
:1037F0000291D0F80C1189020491D0F810118902BD
:103800000391006905903AE06946204603F0F8FE0E
:1038100035E028883AA106EB004002F00FFC207C3E
:103820008DF804002BE028883BA106EB004002F055
:1038300005FC24E0288841A106EB004002F0FEFBD5
:10384000208AADF804001AE0288843A106EB004066
:1038500002F0F4FBF9680720884710E0694620462B
:10386000FFF708FF58B907B0F0BD2888032101EB26
:1038700000403FA102F0E6FB02208DF801002888FD
:103880009DF8012006EB004041A102F0DBFBD4E9EA
:103890000112684690479DF801000128E3D0F968BD
:1038A00005208847DFE7000000A70F0034A10F00C4
:1038B00060000020E801002048616E646C65204EC5
:1038C00052465F4446555F4F505F50524F544F43EE
:1038D0004F4C5F56455253494F4E000048616E644D
:1038E0006C65204E52465F4446555F4F505F4841DD
:1038F0005244574152455F56455253494F4E00007E
:1039000048616E646C65204E52465F4446555F4F79
:10391000505F50494E47000048616E646C65204E10
:1039200052465F4446555F4F505F524543454950AC
:10393000545F4E4F5449465F5345540048616E648E
:103940006C65204E52465F4446555F4F505F4D5464
:10395000555F47455400000048616E646C65204E19
:1039600052465F4446555F4F505F41424F525400AC
:10397000496E76616C6964206F70636F6465207254
:10398000656365697665643A20307825782E000095
:10399000526571756573742068616E646C696E67D9
:1039A00020636F6D706C6574652E20526573756C45
:1039B000743A203078257800F0B5521E87B00F4653
:1039C00005464C1C96B2182227496846F8F752FD66
:1039D000397826488DF800100195042200880C29BA
:1039E00002EB00402DD2DFE801F02C150A2C2C2C24
:1039F0001226203A2C0620788DF8100021E02A8823
:103A00001BA102F01FFB20882880688019E0207825
:103A1000049016E028886880207804902179D4F8F2
:103A2000010061F31F6005900BE00494ADF8146091
:103A3000A868039008E016A102F000FBA889ADF881
:103A40001000A968204688476846FFF771FE0028E5
:103A500003D01449E220FCF71FF807B0F0BD22782C
:103A600011A102F0EFFAC6E718A40F0034020020FB
:103A70005365742072656365697074206E6F746934
:103A800066207461726765743A2025640000000046
:103A900052656365697665642073657269616C203F
:103AA0006D7475004CAB0F00526563656976656493
:103AB0002070696E6720256400000000054810B57D
:103AC0000088022101EB004003A102F0B7FA0020B8
:103AD00010BD0000EC0100204E6F20616464697429
:103AE000696F6E616C2064617461206572617365D9
:103AF00064000000002258210148FCF7B3BF000019
:103B0000C01700202DE9F0411F4C054604262088EF
:103B10001EA106EB004002F091FA2846FFF77EFC5A
:103B200002004FF0010504D0208821A105EB0040E0
:103B300023E04FF4AE78424628492948F8F79AFC2A
:103B4000274F3868401C04D0FFF7D4FF3968814202
:103B500018D0208823A106EB004002F06FFA4146FE
:103B60001F48F8F7AFFC00207D6000F061F802000C
:103B700008D0208823A105EB004002F063FA03205F
:103B8000BDE8F0810020FBE7EC01002043616C6C94
:103B9000696E67206E72665F6466755F73657474C4
:103BA000696E67735F696E697428292E2E2E000076
:103BB0006E72665F6466755F666C6173685F696E7E
:103BC00069742829206661696C6564207769746866
:103BD000206572726F723A202578000000F00F00A5
:103BE000BC170020526573657474696E6720626F3C
:103BF0006F746C6F616465722073657474696E674D
:103C0000732E00006E72665F6466755F666C61732A
:103C1000685F77726974652829206661696C6564DC
:103C20002077697468206572726F723A2025780077
:103C30002DE9F04105464FF4AE773A462149224836
:103C4000F8F752FC214C04260028208806EB00409F
:103C500015D01FA102F0F2F920881A4A06EB0040A5
:103C600020A102F0EFF9002201211648FFF76EFBB8
:103C7000012668B1208823A106EB00401DE02AA19F
:103C800002F0DCF90DB10020A8470020BDE8F0816A
:103C9000FFF730FF0C493A460860A1F5AE70F8F71F
:103CA000E9FB2B463A4630490648FFF7E1FB00287E
:103CB000ECD020882DA106EB004002F0BFF90320D4
:103CC000E4E7000000F00F00BC170020EC0100202A
:103CD00057726974696E672073657474696E67736F
:103CE0002E2E2E0045726173696E67206F6C642002
:103CF00073657474696E67732061743A2030782537
:103D000030387800436F756C64206E6F7420657274
:103D1000617365207468652073657474696E677378
:103D200020706167652100004E65772073657474AB
:103D3000696E677320617265206964656E7469637A
:103D4000616C20746F206F6C642C207772697465CD
:103D5000206E6F74206E65656465642E20536B69F8
:103D60007070696E672E000060160020436F756CDE
:103D700064206E6F742077726974652074686520A2
:103D80004446552073657474696E6773207061676B
:103D90006521000010B54FF4405411496068884215
:103DA0001CD1002304220F49201DFFF761FB48B1FD
:103DB0000D4801210088BDE8104001EB00400BA137
:103DC00002F03CB91248016A012901D100210162C7
:103DD0008169A2681144A1F58051816110BD000084
:103DE000DBE5B1514CA10F0030020020436F756C30
:103DF00064206E6F7420696E76616C6964617465AD
:103E000020536F66744465766963652E0000000078
:103E1000BC1700204FF48050704700002DE9F04798
:103E200082461548154FDFF85880C01BC608B8F801
:103E300000104FF0040909EB01400025324611A1A2
:103E400002F000F9002411E007EBC400416850467D
:103E50008847050009D0B8F800102B4609EB01404F
:103E6000224612A102F0F5F802E0641CB442EBD342
:103E70002846BDE8F0870000B0AE0F00A8AE0F00E6
:103E8000300200205368757474696E6720646F7720
:103E90006E207472616E73706F7274732028666F17
:103EA000756E643A20256429000000004661696C43
:103EB000656420746F2073687574646F776E207406
:103EC00072616E73706F72742025642C206572723B
:103ED0006F722025640000002DE9F04782461448E7
:103EE000144FDFF85480C01BC608B8F800104FF01C
:103EF000040909EB01400025324610A102F0A2F8A6
:103F0000002410E057F8341050468847050009D0C7
:103F1000B8F800102B4609EB0140224610A102F030
:103F200098F802E0641CB442ECD32846BDE8F08760
:103F3000B0AE0F00A8AE0F0030020020496E6974C9
:103F400069616C697A696E67207472616E73706FF3
:103F50007274732028666F756E643A202564290098
:103F60004661696C656420746F20696E697469616B
:103F70006C697A65207472616E73706F727420253B
:103F8000642C206572726F722025640070B5114D2B
:103F9000114CA86B30B105F015F918B1686A08B179
:103FA000012000E000202070FEF7D4FD18B10B497D
:103FB0008E20FBF771FD4023094A0A490A48FEF7A3
:103FC00013FD002805D0BDE8704004499620FBF79A
:103FD00063BD70BDBC1700207000002094A80F00C6
:103FE0003C9F0F00C41B0020C09F0F002DE9F04133
:103FF000134C07460D46E06BA26B01264119914216
:1040000009D910480121008801EB00400EA102F0FF
:1040100015F8032610E00A492A465C31084439465F
:10402000F8F728FAE06B064A2844E0634032294654
:104030003846FCF717FD20643046BDE8F0810000EB
:10404000BC170020F0010020496E697420636F6D79
:104050006D616E64206C6172676572207468616E58
:104060002065787065637465642E000070B5050086
:104070004FF0010404D0B5F5807F03D904240CE08F
:1040800003240AE006490020064E08702021306310
:1040900006F13800F8F716FAB563204670BD000047
:1040A00070000020BC1700202DE9F047304C0E4670
:1040B0008046D4E90E010125DFF8B8902F468142F1
:1040C00008D0B9F800002CA107EB004001F0B6FFC2
:1040D000082549E0DFF8BCA09AF8000030B1FEF7EF
:1040E0007BFEC8F80000606A30603DE005F06AF8C9
:1040F00088B3294890F89C1009B9017859B3041D78
:104100000021C8F80010316090F89C300A462BB1AD
:10411000214C90F83811A03404F1990294F8590018
:1041200004F078FE054601281ED1201D00F0CAF8D3
:104130000546012818D18AF800703146201D05F087
:104140006BFA054601280FD14246201D316805F063
:1041500021FA054608E0FFE7B9F800000FA107EBD8
:10416000004001F06BFF05252846BDE8F087000000
:10417000BC170020F0010020457865637574652048
:1041800077697468206661756C7479206F666673F0
:104190006574000070000020181900204661696CE9
:1041A000656420746F206465636F646520696E695F
:1041B00074207061636B6574000000000148007832
:1041C00070470000700000202DE9F0470646304897
:1041D0002F4D8A4690F89C00012708B1A43500E0D5
:1041E00008350A4631462846FDF7E4FA294C4FF0D7
:1041F000000968B195F8550060B100F00101C0F305
:10420000400288463346284603F016FF00B31BE001
:10421000172727E00120E0621F480421008801EBF6
:1042200000401EA101F00AFF2846C4F8209005F0C6
:1042300059FA08B9FFF7AEFD95F88F0010B195F85F
:10424000900008B96868A060A06CC4E909A00DE0FE
:104250000527B8F1000F05D0FFF7DCFDB04201D112
:10426000FFF798FD0B482430FEF7C6FD09482021D2
:104270003830F8F727F90748FF22F4215C30F8F7C7
:104280001AF9C4F830903846A664BDE8F0870000FB
:1042900018190020BC170020F0010020496E76613B
:1042A0006C69646174696E67206F6C642061707002
:1042B0006C69636174696F6E20696E2062616E6BF8
:1042C00020302E002DE9F04104004FF0010503D10C
:1042D00040497F20FBF7E0FB94F854003E4E012755
:1042E00040B194F8550050B1012808D0022806D0FA
:1042F000032804D0308839A107EB004064E01CB9E2
:1043000034496720FBF7C8FB94F86D00032807D0F9
:10431000308838A107EB004001F090FE142556E0EC
:1043200094F88F00B84618B194F8900000284ED148
:10433000207A58B1E068022734280CD0308832A1A6
:1043400007EB004001F07AFE112540E0318808EBD0
:10435000014032A138E0204604F006FA18B1207876
:1043600050B394B907E0308830A107EB004001F06A
:1043700065FE12252BE017498C20FBF78DFB20787A
:1043800018B914498D20FBF787FB94F855002B4989
:1043900068B101280BD06068C968884217D8308896
:1043A00027A107EB004001F049FE10250FE06068EF
:1043B000896888420BD2F2E794F85500012806D0AC
:1043C000318808EB014023A101F038FE0F25284673
:1043D000BDE8F081DCA80F00F4010020496E766191
:1043E0006C6964206669726D77617265207479709A
:1043F000652E0000496E76616C696420686173689F
:1044000020747970652E00004661756C74792048BF
:10441000572076657273696F6E2E00004E6F2048CC
:10442000572076657273696F6E2E000053442072B8
:104430006571206E6F74206D65742E00BC170020AE
:1044400046572076657273696F6E20746F6F206CAB
:104450006F772E0046572076657273696F6E206DF8
:10446000697373696E672E0010B5104C207820B9FF
:104470000FA140F21F10FBF70FFB606820B90CA1E1
:104480004FF49070FBF708FB0020FBF797FA606889
:10449000401E6060606818B902F0C8FA00206070C1
:1044A000BDE810400020FBF7B7BA00008C1C0020CC
:1044B0002E2E5C2E2E5C2E2E5C2E2E5C2E2E5C69FB
:1044C0006E746567726174696F6E5C6E7266785C3B
:1044D0006C65676163795C6E72665F6472765F6358
:1044E0006C6F636B2E63000070B5184C0546207826
:1044F00018B917A1FE20FBF7CFFA607838B115B1D3
:104500006968002088470020FBF758FA0CE000207B
:10451000FBF754FA25B10D4829460830FDF70EFC8B
:10452000606808B902F052FA6068401C60600020C0
:10453000FBF772FA6068002806D1BDE8704004A15C
:104540004FF48D70FBF7A8BA70BD00008C1C0020E2
:104550002E2E5C2E2E5C2E2E5C2E2E5C2E2E5C695A
:104560006E746567726174696F6E5C6E7266785C9A
:104570006C65676163795C6E72665F6472765F63B7
:104580006C6F636B2E63000070B50A4C207808B125
:1045900085250CE00020A06060602061E060064896
:1045A00002F07CFA054602F0DFF90120207028466F
:1045B00070BD00008C1C0020010A0F00014800782B
:1045C000704700008C1C002010B500B9044802F0B0
:1045D000F7FA002802D1034A0121117010BD000032
:1045E00050A10F007C00002010B5044600F007F831
:1045F000204602F0B9FB02F0B0FB002010BD10B560
:1046000002F0A4FBBDE8104002F0B8BB0349024829
:10461000C1F80403704700000414800100700240D8
:104620002DE9F0411D46174606460C46AA4204D223
:1046300013A140F2C310FBF72FFA206838B102F043
:1046400093FA20B90EA14FF4E270FBF725FA6068E7
:10465000A84204D2002171602168316007E07560D2
:104660002168401B31606060216829442160AF42AD
:1046700003D110B10120BDE8F0810020FBE700006C
:104680002E2E5C2E2E5C2E2E5C2E2E5C2E2E5C632F
:104690006F6D706F6E656E74735C6472697665724F
:1046A000735F6E72665C757362645C6E72665F6483
:1046B00072765F757362642E6300000010B50D4C56
:1046C000207820B90CA140F2EF60FBF7E5F900F08B
:1046D000FFFD1849D1F80403C1F80803164900206A
:1046E0000860BFF36F8FBFF34F8F05F0B3F9012060
:1046F000207010BD800000202E2E5C2E2E5C2E2EF1
:104700005C2E2E5C2E2E5C636F6D706F6E656E740A
:10471000735C647269766572735F6E72665C7573E2
:1047200062645C6E72665F6472765F757362642E3B
:104730006300000000700240007502402DE9F04760
:10474000DFF8049199F80000012804D03FA140F25D
:104750008C60FBF7A1F94FF40068404602F0DEF8E8
:1047600000F050FB484E494D49F2753450B10020DD
:10477000FBF724F929680320002952D0306000207B
:10478000FBF74AF90020FBF719F929683F4FC020D1
:10479000143700294AD038600020FBF73DF93C4926
:1047A00001200860BFF36F8FBFF34F8F3948016856
:1047B0000905FCD5404602F0B1F80020FBF7FEF8F1
:1047C0002868A846002580B33D600020FBF724F947
:1047D00000F018FB50B10020FBF7F0F8D8F80010FB
:1047E000404669B335600020FBF716F92A4940F2CC
:1047F000E37008604020091D0860BFF36F8FBFF3AE
:104800004F8F234980201C3108604C4640F2FF1036
:10481000C4E9020505F01EF9A57002202070BDE86C
:10482000F0872C6030602C60A9E703E02C603860D2
:104830002C60B1E7C8F800403D60C8F80040C4E70C
:10484000046035600460CEE7800000202E2E5C2ED0
:104850002E5C2E2E5C2E2E5C2E2E5C636F6D706F88
:104860006E656E74735C647269766572735F6E7286
:10487000665C757362645C6E72665F6472765F75A7
:104880007362642E6300000014ED064000EC0640E5
:1048900000750240007402400078024005F0EAB959
:1048A00070B5054605F0E6F92846FCF745FD0446D7
:1048B00000F00F00092804D30E4940F2B640FBF780
:1048C000EBF804F00F0122064FF0010001D50A4A6F
:1048D00001E0094A121D1368884083431360BFF347
:1048E0006F8FBFF34F8F284600F0B4F90349C1F82A
:1048F000080370BDAC540F001075024000700240F8
:1049000070B5010600F00F050446092D04D30C49CB
:1049100040F28240FBF7C0F8082D04D3084940F26A
:104920008340FBF7B9F807480460BFF34F8F44F4A6
:1049300080710160BFF36F8FBFF34F8F70BD0000B8
:10494000AC540F000C75024070B5054600F082F9BA
:104950002149C1F80403284601F072FE00283AD12B
:104960002846FCF7E9FC044600F00F00092804D3B0
:104970001A4940F2A540FBF78FF804F00F0021061A
:104980004FF0010401D5164901E01549091D0A68D7
:1049900004FA00F002430A60BFF36F8FBFF34F8F3A
:1049A000280718D0280616D405F00F00082812D2C0
:1049B0000020FBF703F8284600F00EFD2846FCF720
:1049C0006BFC84400748C168A143C160BDE87040EA
:1049D0000020FBF721B870BD00700240AC540F00FE
:1049E000107502408000002010B5FCF7A5FCBDE862
:1049F000104001F025BE00002DE9F0410E460746AB
:104A0000FCF74AFC054626B918A140F65600FBF70C
:104A100043F80020FAF7D2FF234C380704D1A078DE
:104A2000874201D010241BE02089E168C04380B296
:104A30000843012101FA05F5284201D011240FE0B5
:104A40003846FCF73FFC00218160326802607268E2
:104A500042608173E0680543E5600C4605F0DEF9CD
:104A60000020FAF7D9FF2046BDE8F0812E2E5C2EFB
:104A70002E5C2E2E5C2E2E5C2E2E5C636F6D706F66
:104A80006E656E74735C647269766572735F6E7264
:104A9000665C757362645C6E72665F6472765F7585
:104AA0007362642E630000008000002010B5FCF7E4
:104AB00009FC808910BD000070B50C00054602D0CD
:104AC000601E044204D011A140F29B70FAF7E4FF8B
:104AD00005F00F0008280CD31B480068C1B28029DC
:104AE00004D04FF48060A0420AD204E04FF400707A
:104AF000F9E7402C04D905A140F29D70FAF7CCFFEC
:104B00002846FCF7DFFB848170BD00002E2E5C2E52
:104B10002E5C2E2E5C2E2E5C2E2E5C636F6D706FC5
:104B20006E656E74735C647269766572735F6E72C3
:104B3000665C757362645C6E72665F6472765F75E4
:104B40007362642E630000001C75024010B5FCF710
:104B5000F3FB044600F00F00082804D3064940F296
:104B6000CF40FAF799FF054944F480700860BFF31D
:104B70006F8FBFF34F8F10BDAC540F0018750240FC
:104B800010B5FCF7D9FB00F00F01082901D3002074
:104B900010BD0206054800EB810002D5D0F82004C4
:104BA00001E0D0F844040128F1D110BD00700240AA
:104BB00010B5FCF7C1FB044600F00F00082804D331
:104BC000054940F2D740FAF767FF04480460BFF395
:104BD0006F8FBFF34F8F10BDAC540F00187502409C
:104BE00070B50446000604F00F0502D5092D09D35F
:104BF00001E0092D08D307A140F26310FAF74CFF3A
:104C0000200601D5124801E01148123030F8150095
:104C100070BD00002E2E5C2E2E5C2E2E5C2E2E5C87
:104C20002E2E5C636F6D706F6E656E74735C647254
:104C300069766572735F6E72665C757362645C6ED2
:104C400072665F6472765F757362642E6300000043
:104C50000CA20F0070B50546000605F00F0402D542
:104C6000092C09D301E0092C08D307A14FF4C67021
:104C7000FAF712FF280601D5124801E01148093061
:104C8000015D0120884070BD2E2E5C2E2E5C2E2EE4
:104C90005C2E2E5C2E2E5C636F6D706F6E656E7475
:104CA000735C647269766572735F6E72665C75734D
:104CB00062645C6E72665F6472765F757362642EA6
:104CC0006300000030A20F002DE9F0410D460646BA
:104CD000FCF7E2FA044625B930A140F2E770FAF792
:104CE000DBFE0020FAF76AFE3B48310704D18178E9
:104CF0008E4201D0102438E001898046C943C06843
:104D000089B201270143A740394201D011242CE088
:104D10003046FCF7D7FA044606F00F00310600EBE8
:104D200040002AD52D4901EB8006286801F01CFFC0
:104D30000028287A4FEAC07004D008B1284803E060
:104D4000284801E0B8B12848206095E8070086E8C7
:104D500007000020C4E90160A073D8F80C100446D5
:104D60000F43C8F80C7005F059F80020FAF754FE0C
:104D70002046BDE8F0811D48E6E718496C3101EB9B
:104D80008006286838B101F0EFFE20B903A14FF486
:104D90000460FAF781FE1648D6E700002E2E5C2E3E
:104DA0002E5C2E2E5C2E2E5C2E2E5C636F6D706F33
:104DB0006E656E74735C647269766572735F6E7231
:104DC000665C757362645C6E72665F6472765F7552
:104DD0007362642E6300000080000020C01D00206C
:104DE00045500F00C54F0F00214F0F00854E0F009B
:104DF00021460F0010B5FCF79FFABDE8104001F006
:104E00004DBD000010B500F013F858B10748007808
:104E1000C0F30310012805D10448001D007810F0EC
:104E2000F00F01D0002010BD012010BDE80F00F0F0
:104E300006480078082804D10448001D00780007BF
:104E400001D000207047012070470000E00F00F003
:104E500010B5FFF7EDFF50B10748007810F0F00FE4
:104E600005D10548001D007810F0F00F01D000209A
:104E700010BD012010BD0000E80F00F00048704791
:104E8000981E00202DE9F041804616460C46086821
:104E900001F06AFE20B112A14FF40B70FAF7FCFD8D
:104EA00065681E4FB54200D93546402D04D90CA186
:104EB00040F23620FAF7F0FD2A4638462168F7F727
:104EC000D9FAC8E900756068401B60602068284412
:104ED00020606068002800D00120BDE8F08100005B
:104EE0002E2E5C2E2E5C2E2E5C2E2E5C2E2E5C63C7
:104EF0006F6D706F6E656E74735C647269766572E7
:104F0000735F6E72665C757362645C6E72665F641A
:104F100072765F757362642E63000000981E002035
:104F20002DE9F041064690460D46086801F01CFE4A
:104F300020B114A140F25220FAF7AEFD6C68204F68
:104F40004046444500D90446402C04D90DA14FF4F5
:104F50001770FAF7A1FD34B1224638462968F7F7F1
:104F600089FA376001E00020306074606868001BD7
:104F7000686028682044286014B10120BDE8F081F1
:104F80000020FBE72E2E5C2E2E5C2E2E5C2E2E5C3F
:104F90002E2E5C636F6D706F6E656E74735C6472E1
:104FA00069766572735F6E72665C757362645C6E5F
:104FB00072665F6472765F757362642E63000000D0
:104FC000981E00202DE9F041074616460C46086859
:104FD00001F0CAFD20B90CA14FF4F570FAF75CFDA1
:104FE0006568B54200D935462068C7E900056068A4
:104FF000401B60602068284420606068002800D062
:105000000120BDE8F08100002E2E5C2E2E5C2E2E9D
:105010005C2E2E5C2E2E5C636F6D706F6E656E74F1
:10502000735C647269766572735F6E72665C7573C9
:1050300062645C6E72665F6472765F757362642E22
:10504000630000002DE9F041074616460C4608684B
:1050500001F08AFD20B910A140F20B20FAF71CFDE7
:105060006568B54200D93546002D0FD0D4F8000050
:10507000C7E900056068A0EB05006060206828446F
:10508000206006D04FF00100BDE8F0814FF0000035
:10509000EEE74FF00000F7E72E2E5C2E2E5C2E2E52
:1050A0005C2E2E5C2E2E5C636F6D706F6E656E7461
:1050B000735C647269766572735F6E72665C757339
:1050C00062645C6E72665F6472765F757362642E92
:1050D000630000002DE9F04128B11E490A7822B191
:1050E0000820BDE8F0810720FBE74860012000248C
:1050F000087046024FEA040544F0800707F00F00ED
:10510000082801D3314600E040213846FFF7D4FC9F
:105110003846FCF7D7F88573641C0560E4B28560F7
:10512000092CE9D35FF0000404F00F00082801D334
:10513000314600E040212046FFF7BEFC2046FCF748
:10514000C1F88573641C0560E4B28560092CEBD35B
:105150000020C6E78000002003480078022801D321
:10516000012070470020704780000020024800782E
:10517000002800D0012070478000002010B5FFF704
:10518000EBFF28B12720F8F7C7FE08B1012010BDBA
:10519000002010BD0148807870470000800000208A
:1051A000502001F0CDBB10B5FFF752FE58B1EFF320
:1051B000108472B64C2001F0C3FB4C2001F0C0FB00
:1051C00084F3108810BDBDE810404C2001F0B8BB3E
:1051D0000021016041601149096801700F49091DF2
:1051E000096841700D49083109680C4A0C3212688F
:1051F00041EA02214180094910310968074A143205
:10520000126841EA02218180044918310968034A81
:105210001C32126841EA0221C1807047807402404A
:10522000542001F08DBB000070B5144C0546207869
:10523000022804D012A140F2FD60FAF72DFC0020F4
:1052400060701E4C15B9FFF703FE00B11C4C1D48E1
:10525000C0F804431C49E02081F800041A490122E7
:1052600080202339C1F88002C1F80001174802608C
:10527000BFF36F8FBFF34F8F70BD00008000002021
:105280002E2E5C2E2E5C2E2E5C2E2E5C2E2E5C6323
:105290006F6D706F6E656E74735C64726976657243
:1052A000735F6E72665C757362645C6E72665F6477
:1052B00072765F757362642E630000000714C0018C
:1052C0000714E0010070024027E000E0047502408E
:1052D000104810B50078022804D00FA140F21C70CD
:1052E000FAF7DAFB2720F8F717FE002810D004F0B1
:1052F00023FD184900200860BFF36F8FBFF34F8F65
:1053000015498020C1F8800148171449C1F80803E5
:1053100010BD0000800000202E2E5C2E2E5C2E2E54
:105320005C2E2E5C2E2E5C636F6D706F6E656E74DE
:10533000735C647269766572735F6E72665C7573B6
:1053400062645C6E72665F6472765F757362642E0F
:10535000630000000475024004E000E000700240B9
:1053600010B500242046FAF729FB12484078B0B166
:1053700004F0E2FC10480168890510D40F490122AD
:105380000A60006882054FF0000001D5086006E061
:105390000B4901240B680A4A14322BB1106000201B
:1053A000FAF73AFB204610BD49F275330B601060E6
:1053B0000B60F4E780000020007402402C7502406E
:1053C00000EC064003490248C1F80803704700009A
:1053D00004148001007002402DE9F04104460006EB
:1053E00004D521A14FF40E60FAF756FBFFF730FD0C
:1053F00001274FF000082B4D002804F00F0640460F
:1054000012D0FAF7DBFA2046FBF746FF8740A86880
:105410002549B843A86040F2C57000EB460008601B
:10542000091DC1F800801AE0FAF7C8FA2046FBF718
:1054300033FF8740A868B843A860082E0FD2200623
:1054400004D51AA140F26240FAF726FB224A02EB89
:105450008601C1F8A084BFF36F8FBFF34F8FBDE803
:10546000F0410020FAF7D8BA2E2E5C2E2E5C2E2E9C
:105470005C2E2E5C2E2E5C636F6D706F6E656E748D
:10548000735C647269766572735F6E72665C757365
:1054900062645C6E72665F6472765F757362642EBE
:1054A0006300000080000020007802402E2E5C2E59
:1054B0002E5C2E2E5C2E2E5C2E2E5C6D6F64756C19
:1054C00065735C6E7266785C68616C5C6E72665F58
:1054D000757362642E680000007002400548017810
:1054E000012901D008207047002141600170084661
:1054F000704700008000002010B500242046FAF715
:105500005DFA0E48407868B101F012FA50B10C49CA
:10551000002008600B4901240B680A4AC02014329D
:105520002BB110600020FAF777FA204610BD49F23F
:1055300075330B6010600B60F4E700008000002002
:105540002C75024000EC06400FB438B5040003D1BE
:1055500010A11C20FAF7A0FA606918B90DA11D204E
:10556000FAF79AFA206818B90AA11E20FAF794FAF5
:10557000606818B907A11F20FAF78EFA059900296B
:1055800005D006A800906A46204600F045F838BCD1
:105590005DF814FB2E2E5C2E2E5C2E2E5C2E2E5CC7
:1055A0002E2E5C65787465726E616C5C66707269D3
:1055B0006E74665C6E72665F667072696E74662E7B
:1055C0006300000010B5040003D107A10B20FAF717
:1055D00063FAA268002A05D0D4E904032168984739
:1055E0000020A06010BD00002E2E5C2E2E5C2E2E02
:1055F0005C2E2E5C2E2E5C65787465726E616C5C20
:10560000667072696E74665C6E72665F66707269EF
:105610006E74662E630000002DE9FC4791460C462F
:105620005FEA000804D183A14FF49F70FAF734FABF
:10563000D8F8140020B97FA14FF4A070FAF72CFA23
:10564000D8F8000020B97BA140F24110FAF724FA03
:10565000D8F8040020B977A14FF4A170FAF71CFA2A
:10566000002C76D014F8011B39B125290ED0404604
:10567000FAF7D8FB20780028F4D198F80C0000281D
:1056800067D04046BDE8FC47FFF79CBF00200122E1
:1056900021782B291BD02D2902D0302908D102E0F6
:1056A00040F0010001E040F00200641C002AEFD14C
:1056B00000252A290ED02178A1F130020A2A11D220
:1056C00005EB850201EB4205641C303DF1E740F03B
:1056D0000400EAE7D9F800100B1DC9F8003009688A
:1056E000641C0D44217800232E290BD114F8011FCE
:1056F000A1F130020A2A05D203EB830201EB420337
:10570000303BF3E76C290DD068290BD0692921D0F3
:105710000BDC252918D0582931D063290ED06429F3
:1057200015D117E014F8011FECE7702969D073292F
:1057300032D075291BD0782909D120E0D9F8000092
:10574000011DC9F8001001784046FAF76BFB641C94
:1057500090E76CE0D9F800100A1DC9F8002009682C
:10576000CDE900500A224046FCF7F8F9EFE7D9F8F6
:1057700000100A1DC9F8002009680A2206E0D9F8BD
:1057800000100A1DC9F8002009681022CDE9005058
:10579000404603F0A5FEDAE7D9F8001000270A1DFD
:1057A000C9F800200E68C00705D112E04046761CFB
:1057B0007F1CFAF737FB31780029F7D104E020216C
:1057C00040466D1EFAF72EFBBD42C0D9002DF6D122
:1057D000BDE74EB13046F6F780FE074604E02021D3
:1057E00040466D1EFAF71EFBBD4206D9002DF6D1CC
:1057F00003E04046761CFAF715FB31780029F8D112
:10580000A5E7D9F80000011DC9F80010056830218E
:105810004046FAF707FB78214046FAF703FB0820D9
:105820000021CDE90001034610222946B0E7BDE87A
:10583000FC8700002E2E5C2E2E5C2E2E5C2E2E5C05
:105840002E2E5C65787465726E616C5C6670726930
:105850006E74665C6E72665F667072696E74665FA7
:10586000666F726D61742E63000000002DE9F041D7
:105870001E4615460F46040003D11DA17820FAF7F5
:105880000BF9206818B91AA17920FAF705F91DB9A2
:1058900017A17A20FAF700F939462046F8F704FEF6
:1058A00040B939462046F8F7FFFD18B910A17D2010
:1058B000FAF7F2F860683946026820466A43F8F75A
:1058C000FCFD58B960683946026820466A43F8F71B
:1058D000F4FD18B906A17F20FAF7DEF820683346F8
:1058E0002A46D0F810C039462046BDE8F04160474E
:1058F0002E2E5C2E2E5C2E2E5C2E2E5C2E2E5C63AD
:105900006F6D706F6E656E74735C6C6962726172DC
:105910006965735C6673746F726167655C6E7266ED
:105920005F6673746F726167652E630070B51646AB
:105930000C46050003D108A12F20FAF7ADF81CB9D9
:1059400005A13020FAF7A8F82C60314628462268D5
:10595000BDE87040104700002E2E5C2E2E5C2E2ECF
:105960005C2E2E5C2E2E5C636F6D706F6E656E7498
:10597000735C6C69627261726965735C6673746F83
:10598000726167655C6E72665F6673746F72616781
:10599000652E63002DE9F04128B1016819B1C9698C
:1059A000BDE8F04108470D4D0D480024461B142763
:1059B0000DE000BF04EB840005EB8000016829B115
:1059C000C969884710B10120BDE8F081641CB6FBAD
:1059D000F7F0A042EED80020F6E70000C401002056
:1059E000D80100202DE9F8431D46089F1646884639
:1059F000040003D12AA16220FAF74EF81EB928A1AB
:105A00006320FAF749F8206818B925A16420FAF74D
:105A100043F81DB922A16520FAF73EF86068406896
:105A2000B5FBF0F100FB115141B1B5FBF0F100FB0A
:105A3000115018B11AA16820FAF72EF84046F8F76D
:105A40002DFD38B94046F8F729FD18B914A16B208F
:105A5000FAF722F83046F8F721FD38B93046F8F762
:105A60001DFD18B90EA16C20FAF716F82A4641461A
:105A70002046F8F722FD48B92A4641462046F8F765
:105A80001CFD18B906A16D20FAF706F800972068EA
:105A90002B463246C76841462046B847BDE8F883E2
:105AA0002E2E5C2E2E5C2E2E5C2E2E5C2E2E5C63FB
:105AB0006F6D706F6E656E74735C6C69627261722B
:105AC0006965735C6673746F726167655C6E72663C
:105AD0005F6673746F726167652E63002DE9FF4125
:105AE0001C46DDE90A7815460E46684600F010F8B7
:105AF00046EA450141EA840141EA072242EA0841B7
:105B0000009A00EB8200C0F80017BDE8FF8100009A
:105B100010B504460068302804D308A140F2A11053
:105B2000F9F7BAFF2068202802D24FF0A04010BD3C
:105B300000F01F0020600C4810BD00002E2E5C2ECF
:105B40002E5C2E2E5C2E2E5C2E2E5C6D6F64756C82
:105B500065735C6E7266785C68616C5C6E72665FC1
:105B60006770696F2E6800000003005010B504468E
:105B70000068302804D308A140F2A110F9F78CFF87
:105B80002068202802D24FF0A04010BD00F01F0076
:105B900020600C4810BD00002E2E5C2E2E5C2E2E98
:105BA0005C2E2E5C2E2E5C6D6F64756C65735C6E66
:105BB0007266785C68616C5C6E72665F6770696F54
:105BC0002E6800000003005038B50124009068469C
:105BD00031B1FFF79DFF00998C40C0F8084538BDF2
:105BE000FFF796FF00998C40C0F80C4538BD0000C7
:105BF00030B5104B014600201C69224609E0157A99
:105C0000854205D1401C0A28F7DB4FF0FF3030BD3C
:105C10005268002AF3D1421CF9D008721A6922B1E5
:105C200052684A601A69516030BD002219614A60A9
:105C300030BD0000406100207047F7F71FBF70477C
:105C400008B5034A00924023024A00F005F808BD57
:105C5000CD870F003E200020F0B595B01C461546BC
:105C60000F4608461A9E00F06DFB182109A8F6F7AA
:105C700029FC0E96CDE909540023082203A93846D1
:105C800000F075FB05980690BDF81000ADF81C00FB
:105C9000BDF81200ADF81E0000208DF82100039819
:105CA000082600F00300012802D0022818D032E0B4
:105CB00003983346850AC0F3C2008DF8200003988C
:105CC0000FA9C0F38314A200384600F050FB09A8C6
:105CD000009006AB22460FA9284600F08FFA1AE082
:105CE0000398840DC0F3C2008DF82000082C01D267
:105CF000254600E0082533462A460FA9384600F01D
:105D000036FB2E44641B09AB06AA29460FA800F0F7
:105D1000C9F9002CEAD1384600F01AFB15B0F0BDE5
:105D20000A4A012902EBC00007D0022907D0032943
:105D300007D0042907D000207047022070470420B4
:105D4000704700797047407970470000B0AE0F008F
:105D500010B5FFF772FF04210648FFF749FF00283E
:105D600003DA05491B20F9F797FE02490120487222
:105D700010BD00005401002044AA0F002DE9F04F8F
:105D80008DB0FAF75FF818B100200DB0BDE8F08FC4
:105D9000774E0020B061BFF34F8FA6F580444FF0DF
:105DA000000960680290A568284004EB800008E0C4
:105DB00021680298814201D86160E5E7284004EB40
:105DC00080000C3002A9FBF71DFF0028F0D103ABC7
:105DD000A046029901EA050408EB8402491CD26836
:105DE00043F82020401C02910228F2D3039800F0CF
:105DF0000300022802D001284CD0A2E003985022D0
:105E0000810D8A46B2EB905F00D850210C4664F3B6
:105E10009F5003900831574800F04BFA070075D0A7
:105E200000F090FA4B46082203A9384600F0A5FA84
:105E3000029909F1080B2940681A8000001D84426C
:105E400021D94D4D30B1C2B208EB8101201A9146E3
:105E50000C3104E02946E2B2002591462846C4B23E
:105E60005B46384600F089FA0BEB090325B1224660
:105E70002946384600F081FA02990AF1030001EB45
:105E8000900002903BE008EB81015B4622463846D9
:105E90000C31EFE70398C0F38310062800D30620E7
:105EA000039960F38911C1F38310801C0391810071
:105EB000304800F0FEF9070043D000F043FA4B46AB
:105EC000082203A9384600F058FA09F1080900240D
:105ED0000FE002984B4600EA0501401C08EB8101E7
:105EE0000290042238460C3100F047FA09F1040907
:105EF000641C0398C0F38310A042EAD837B1346918
:105F0000B06968B1384600F023FA2BE019E0607AF6
:105F1000012804D1226820463946126890476468F7
:105F2000002CF4D1384600F013FA0020F9F746FDB2
:105F3000B06910B90299C8F804100020F9F76CFD97
:105F400010E0346904E02168204689688847646865
:105F5000002CF8D109480221008801EB004008A17B
:105F600000F06CF8F9F76EFF80F001000DE700001B
:105F70004061002080AF0F004C2100203002002043
:105F80004261636B656E647320666C7573686564EB
:105F9000000000002DE9F84F8146264FD01C154621
:105FA0008A46800800226946BE68F9F7E9FEB8B360
:105FB000009CB846A01C0090B9683040091A8F00B8
:105FC0003F1DBD4208EB800002D82A46514608E03A
:105FD0003A4651460C30F6F74DFA1648EA1B0AEBE2
:105FE00007010C30F6F746FA4FEA1947FAF7B0FF07
:105FF00047EA0042601C304008EB8000344008EB68
:106000008401C260C8684FF6C07269F3C50090434E
:1060100065F39F5020F00300801C20F00400C8604E
:10602000054890F8200001E0FFF7A8FE0028FBD10A
:10603000BDE8F88F402100204061002000231A466F
:1060400003F068B808B5012300926A4603F062F8CD
:1060500008BD1CB5CDE9002302236A4603F05AF8B7
:106060001CBD3EB5069C8DE81C0003236A4603F068
:1060700051F83EBD7FB5DDE908458DE83C000423BD
:106080006A4603F047F87FBD70B586B00DF1280C65
:106090009CE870008DE87C0005236A4603F03AF81E
:1060A00006B070BD2DE9F0470E4680461C4692466C
:1060B00008293ED894F80C90002020731946104609
:1060C00002F014F80025B54206D218F805201AA1EE
:1060D0002046FFF739FA03E019A12046FFF734FA0A
:1060E0006D1C082DEFD317A12046FFF72DFA0025D0
:1060F000B54210D218F80570F6F7B8F90068C05D1F
:1061000010F03E0F01D03A4600E02E220EA12046AC
:10611000FFF71AFA03E00DA12046FFF715FA6D1CF0
:10612000082DE5D301222146504601F067FF84F88F
:106130000C90BDE8F0870000202530327800000088
:10614000202020007C0000002563000020000000CB
:10615000104910B540F6FF70886000200860486064
:1061600001F580418861486181F820000A4800F00B
:10617000EDF800280CD1094809490A4B401AC1081A
:10618000002002E023F82000401C8842FAD30020BF
:1061900010BD00004021002080AF0F0080AF0F0035
:1061A000B0AE0F00D801002002480349401AC008D1
:1061B0007047000080AF0F00B0AE0F0013B5684607
:1061C000FBF7C0FE08B100201CBD0248009950F842
:1061D00031001CBDB0AE0F0070B507480125046941
:1061E00080F8205005E0657221682046496888479C
:1061F0006468002CF7D170BD406100202DE9FF4795
:1062000081460C9D00200C462F7B2873984616462D
:106210002946184601F06AFF072E42D2DFE806F051
:1062200004090F161F2A360049462846FFF78CF945
:1062300037E0494628462268FFF786F931E0D4E97D
:10624000002349462846FFF77FF92AE0A06800901E
:10625000D4E9002349462846FFF776F921E0D4E93E
:106260000201CDE90001D4E9002349462846FFF7A1
:106270006BF916E004F1080007C88DE80700D4E9BF
:10628000002349462846FFF75FF90AE004F10800B9
:106290000FC88DE80F00D4E9002349462846FFF7D0
:1062A00053F900222946404601F0A8FE2F73BDE8AD
:1062B000FF872DE9F041858A80462D1F4819C01CB3
:1062C000B0FBF5F0C6B24046FBF7C6FE041E19D07F
:1062D0000020207101206071E58000272546761E90
:1062E000C4F800800BE04046FBF7B6FE60B1617970
:1062F000491C6171286005467F1CC0F80080B742C8
:10630000F1D32046BDE8F081204600F002F80020DD
:10631000F8E72DE9F041457901466B1E002201E0C6
:106320000968521C9A42FBD30F680146002605E01B
:1063300038460C68FBF7F2FE2146761CAE42F7D3D6
:10634000BDE8F0810121001DFBF75FBEFBF72ABF0E
:1063500010B504460121001DFBF778FE10F0FF0F79
:1063600004D12046BDE81040FFF7D3BF10BD38B5BB
:1063700001240094FBF79CFD38BD38B5002400943F
:10638000FBF796FD38BD0000094902220A60BFF301
:106390006F8FBFF34F8F0A1D106006480268002AF6
:1063A000FCD000200860BFF36F8FBFF34F8F7047A2
:1063B00004E5014000E4014070B50E4C0123236068
:1063C000BFF36F8FBFF34F8F00230B4D08E000BF6B
:1063D00051F8236040F823602E68002EFCD05B1C2F
:1063E0009342F5D300202060BFF36F8FBFF34F8F30
:1063F00070BD000004E5014000E4014000F180416F
:106400000868002210B101200A60704710467047EA
:1064100070B50D46060003D10BA11420F9F73CFB23
:106420001DB909A11520F9F737FB746804E0B268BB
:106430002946904718B1246820680028F7D12068C1
:106440002860256070BD00002E2E5C2E2E5C2E2E46
:106450005C2E2E5C2E2E5C636F6D706F6E656E749D
:10646000735C6C69627261726965735C736F72747C
:106470006C6973745C6E72665F736F72746C69734F
:10648000742E630010B5040003D103A13D20F9F779
:1064900003FB206810BD00002E2E5C2E2E5C2E2EDD
:1064A0005C2E2E5C2E2E5C636F6D706F6E656E744D
:1064B000735C6C69627261726965735C736F72742C
:1064C0006C6973745C6E72665F736F72746C6973FF
:1064D000742E630010B5040003D103A13720F9F72F
:1064E000DBFA6068006810BD2E2E5C2E2E5C2E2E0E
:1064F0005C2E2E5C2E2E5C636F6D706F6E656E74FD
:10650000735C6C69627261726965735C736F7274DB
:106510006C6973745C6E72665F736F72746C6973AE
:10652000742E630010B5040003D105A12B20F9F7E8
:10653000B3FA61680868002801D002680A6010BDDB
:106540002E2E5C2E2E5C2E2E5C2E2E5C2E2E5C6350
:106550006F6D706F6E656E74735C6C696272617280
:106560006965735C736F72746C6973745C6E726668
:106570005F736F72746C6973742E630070B50C4630
:10658000050003D10BA14320F9F786FA1CB909A134
:106590004420F9F781FA0021686806E0A24203D19D
:1065A00021680160012103E010460268002AF5D14C
:1065B000084670BD2E2E5C2E2E5C2E2E5C2E2E5C80
:1065C0002E2E5C636F6D706F6E656E74735C6C699C
:1065D000627261726965735C736F72746C697374F3
:1065E0005C6E72665F736F72746C6973742E630095
:1065F00030B5050600F00F030E4C03EB830004EBEF
:1066000080000AD5082B03D30B480160001D09E068
:10661000C0F80016C0F8042630BD082B04D3074884
:106620000160001D026030BDC0F80017C0F80427EB
:1066300030BD000000700240A0760240A07702400A
:1066400010B5044600F00F00092804D30BA140F256
:106650009640F9F721FA21064FF0010004F00F02ED
:1066600000FA02F001D5104901E00F49091D09683F
:10667000014201D0012010BD002010BD2E2E5C2E45
:106680002E5C2E2E5C2E2E5C2E2E5C6D6F64756C37
:1066900065735C6E7266785C68616C5C6E72665F76
:1066A000757362642E6800001075024070B5044670
:1066B000000604D415A140F29B30F9F7EDF904F07F
:1066C0000F00082804D311A14FF46770F9F7E4F91B
:1066D000200704D10DA140F29D30F9F7DDF903F058
:1066E000B9F92046FAF7EEFD817B0125032902D096
:1066F0000068002809D12046FAF7CEFD8540E9431D
:10670000BDE870401048FBF786BC70BD2E2E5C2E95
:106710002E5C2E2E5C2E2E5C2E2E5C636F6D706FA9
:106720006E656E74735C647269766572735F6E72A7
:10673000665C757362645C6E72665F6472765F75C8
:106740007362642E630000008C00002038B504469C
:10675000000604D41B4940F2BB30F9F79DF904F060
:106760000F00082804D217494FF46F70F9F794F915
:1067700003F070F92046FAF7A5FD817B0125032976
:1067800015D00068002811D12046FAF785FD854014
:10679000E9430D48FBF73FFC0C480B49806800902B
:1067A0000C398DF8024049686846884738BD204654
:1067B000FAF772FD8540E943BDE838400248FBF72F
:1067C0002ABC0000A09A0F008C00002060A10F00DE
:1067D00038B50446000604D51FA14FF47F70F9F7C1
:1067E0005BF904F00F00082804D31BA140F2FD3030
:1067F000F9F752F9200704D117A140F2FE30F9F75A
:106800004BF903F027F92046FAF75CFD817B01255F
:10681000032902D0006848B11AE02046FAF73CFD8F
:106820008540E9431B48FBF7F6FB11E02046FAF7E9
:1068300033FD8540E9431748FBF7EDFB1648154942
:10684000006900900C398DF8024049686846884715
:10685000BDE8384003F042B92E2E5C2E2E5C2E2E61
:106860005C2E2E5C2E2E5C636F6D706F6E656E7489
:10687000735C647269766572735F6E72665C757361
:1068800062645C6E72665F6472765F757362642EBA
:10689000630000008C00002060A10F0070B5054669
:1068A000000605F00F0402D5092C09D301E0092CDC
:1068B0000BD30D4940F23E40F9F7EEF8280604D517
:1068C000094940F23F40F9F7E7F8082C05D307489B
:1068D0000068C10300D5002070BD054901EB8400AC
:1068E000D0F8A00470BD0000AC540F00C07402408A
:1068F0000070024002494058002800D00120704733
:10690000007002400449084400210160BFF36F8F0A
:10691000BFF34F8F704700000070024003490860CA
:10692000BFF36F8FBFF34F8F7047000000740240BA
:1069300002480068002800D0012070472C750240F2
:106940000449084401210160BFF36F8FBFF34F8FEB
:10695000704700000070024002480068002800D024
:106960000120704700040140084810B5007918B9AB
:1069700007A19520F9F790F800F0FEF812490120E0
:1069800008600249091F087010BD0000980000202F
:106990002E2E5C2E2E5C2E2E5C2E2E5C2E2E5C6DF2
:1069A0006F64756C65735C6E7266785C6472697630
:1069B0006572735C7372635C6E7266785F636C6F32
:1069C000636B2E630000000018050040084810B5F6
:1069D000007918B907A1D420F9F75EF84FF4807058
:1069E000FBF783FF01208107C1F80403086010BD95
:1069F000980000202E2E5C2E2E5C2E2E5C2E2E5CFF
:106A00002E2E5C6D6F64756C65735C6E7266785C5F
:106A1000647269766572735C7372635C6E726678B9
:106A20005F636C6F636B2E630000000010B50A4C4F
:106A3000207918B909A1DC20F9F72EF815490120B1
:106A4000086015494FF001100A6802F001128242F5
:106A5000FAD00020607110BD980000202E2E5C2E10
:106A60002E5C2E2E5C2E2E5C2E2E5C6D6F64756C53
:106A700065735C6E7266785C647269766572735C6D
:106A80007372635C6E7266785F636C6F636B2E63A8
:106A900000000000040000400C04004010B5040099
:106AA00003D108A17C20F8F7F7FF144900200A79E8
:106AB0000AB1852010BD01220C600A7100224A71C2
:106AC00010BD00002E2E5C2E2E5C2E2E5C2E2E5C19
:106AD0002E2E5C6D6F64756C65735C6E7266785C8F
:106AE000647269766572735C7372635C6E726678E9
:106AF0005F636C6F636B2E630000000098000020E2
:106B000070B54FF480763046FBF7E8FE114CB505C2
:106B100060B13046FBF7E9FE0120C5F80803607953
:106B200020B9012060712168002088474FF48276E7
:106B30003046FBF7D3FE00280AD03046FBF7D5FEDF
:106B40000220C5F808032168BDE87040012008470D
:106B500070BD000098000020002802D0014980018B
:106B600008477047A1A10F000121B1EB507F01D16F
:106B7000012070470020704707480068012110F08D
:106B8000010F08D14FF0E020E02280F80024C0F887
:106B90008012C0F80011704700E100E0074800686B
:106BA000012110F0010F08D14FF0E020E02280F821
:106BB0000024C0F88012C0F80011704700E100E026
:106BC00070B5040003D10DA14620F8F765FF194DFB
:106BD000287808B1852070BD20781749C0F340009F
:106BE000086015492078083900F001000860FFF7B7
:106BF000D5FF01202870002070BD00002E2E5C2ED5
:106C00002E5C2E2E5C2E2E5C2E2E5C6D6F64756CB1
:106C100065735C6E7266785C647269766572735CCB
:106C20007372635C6E7266785F706F7765722E63E5
:106C300000000000A00000208005004070B54FF06B
:106C40008040D0F80453324C68070CD54FF4847060
:106C5000FFF7D4FB38B1606818B92EA1E020F8F72F
:106C60001BFF60688047A8060DD54FF48A70FFF7B8
:106C7000C5FB40B1A06818B926A1E820F8F70CFFC1
:106C8000A1680020884768060DD54FF48C70FFF787
:106C9000B5FB40B1A06818B91EA1EF20F8F7FCFEC3
:106CA000A1680120884728060DD54FF48E70FFF7A4
:106CB000A5FB40B1E06818B916A1F820F8F7ECFE82
:106CC000E16800208847E8050DD54FF49070FFF784
:106CD00095FB40B1E06818B90EA1FF20F8F7DCFE83
:106CE000E16801208847A80511D54FF49270FFF79D
:106CF00085FB00280BD0E06820B906A14FF4837013
:106D0000F8F7CAFEE168BDE870400220084770BD90
:106D1000A00000202E2E5C2E2E5C2E2E5C2E2E5CD3
:106D20002E2E5C6D6F64756C65735C6E7266785C3C
:106D3000647269766572735C7372635C6E72667896
:106D40005F706F7765722E63000000004FF0804126
:106D50004FF46070C1F8080370474FF080414FF462
:106D60006070C1F80403704703490022CA600068DC
:106D7000002800D0C8607047A00000200149002012
:106D8000C8607047A000002070B50C46050003D114
:106D90000D49D920F8F780FE1CB90B49DA20F8F725
:106DA0007BFE0A480421008801EB004008A1FFF7A0
:106DB00045F912490320C96888476869FDF756F903
:106DC000FAF7DCFC607070BD00A70F00E80100203E
:106DD00048616E646C65204E52465F4446555F4F75
:106DE000505F4F424A4543545F435245415445200A
:106DF00028636F6D6D616E642900000060000020E3
:106E000070B50C4620B9154940F20110F8F744FE60
:106E100024B912494FF48170F8F73EFE104D042654
:106E200010A1288806EB0040FFF708F91849081F51
:106E3000FDF73AF9FAF7A2FC6070012805D10020AD
:106E4000FCF7F6FE10B10A20607070BD288811A111
:106E500006EB0040BDE87040FFF7F0B800A70F0058
:106E6000E801002048616E646C65204E52465F4424
:106E700046555F4F505F4F424A4543545F45584522
:106E8000435554452028636F6D6D616E6429000081
:106E90006800002057726974696E672076616C69BA
:106EA0006420696E697420636F6D6D616E64207417
:106EB0006F20666C6173682E0000000070B50D468F
:106EC000040003D11749E720F8F7E6FD206918B957
:106ED0001449E820F8F7E0FDA08A18B91149E92023
:106EE000F8F7DAFD1DB90F49EA20F8F7D5FD0E488D
:106EF0000421008801EB00400CA1FFF79FF8A18A54
:106F00002069FDF773F8FAF739FC68702846F9F73D
:106F100085FDE168002903D02069BDE8704008477D
:106F200070BD000000A70F00E801002048616E64FA
:106F30006C65204E52465F4446555F4F505F4F424E
:106F40004A4543545F57524954452028636F6D6D3D
:106F5000616E6429000000002DE9F0410B4E0D46E2
:106F6000042730880AA107EB0040FFF767F8114CAF
:106F7000308811A107EB0040A36C226DFFF769F880
:106F8000A06CA860206D6860BDE8F081E801002079
:106F900048616E646C65204E52465F4446555F4FB3
:106FA000505F4352435F4745542028646174612910
:106FB00000000000BC1700204F66667365743A2518
:106FC000642C204352433A30782530387800000052
:106FD0002DE9F84F3E4C81460D462088042707EBEB
:106FE00000403CA1FFF72AF8FDF7E8F801264FF032
:106FF000080AC8B1D9F814204FF00308DAB13F49A4
:107000003F4813051CD0436DD1F808C013446345B5
:1070100016D020883BA106EB004000BFFFF70EF81A
:1070200085F80180BDE8F88F20883FA106EB00407D
:10703000FFF704F81EE0208849A106EB0040EDE7C9
:10704000B2F5805F07D920884CA106EB0040FEF71F
:10705000F5FF6F70E6E7436DD1F808C003EB020857
:10706000E0450AD9CDF800C020884D4906EB004024
:10707000FEF7F7FF85F801A0D4E74264C26C036510
:10708000036380468264D9F81400002200F6FF7082
:107090004FEA103C486861461844FCF757F940B184
:1070A000208840A106EB0040FEF7C8FF052068706D
:1070B000B8E7D8F848100091208840A107EB0040BD
:1070C000D8F85030D8F84420FEF7CBFFAAE70000EC
:1070D000E801002048616E646C65204E52465F44B2
:1070E00046555F4F505F4F424A4543545F435245B8
:1070F000415445202864617461290000600000202B
:10710000BC1700204F626A6563742073697A65203A
:107110006D757374206265207061676520616C69AC
:10712000676E65640000000043616E6E6F742063DB
:1071300072656174652064617461206F626A656361
:107140007420776974686F75742076616C69642047
:10715000696E697420636F6D6D616E64000000007C
:107160004F626A6563742073697A652063616E6E2D
:107170006F7420626520302E00000000496E766139
:107180006C69642073697A6520666F72206F626A29
:107190006563742028746F6F206C617267652900C5
:1071A0008CA60F004572617365206F706572617403
:1071B000696F6E206661696C656400004372656189
:1071C00074696E67206F626A65637420776974689A
:1071D0002073697A653A2025642E204F66667365B0
:1071E000743A203078253038782C204352433A20A6
:1071F00030782530387800002DE9F041154D0746EC
:107200000E462888042101EB004013A1FEF716FF6B
:107210001B4CD4E91401626C431A9A420BD02888A3
:10722000012101EB004017A1FEF713FF0820707049
:107230000120BDE8F08100216164A16CE16460651A
:107240000021384600F032F817490420C968884701
:107250000020EEE7E801002048616E646C65204E76
:1072600052465F4446555F4F505F4F424A45435434
:107270005F45584543555445202864617461290091
:10728000BC170020496E76616C696420646174618A
:107290002E2065787065637465643A2025642C201F
:1072A000676F743A20256400600000202DE9F041EA
:1072B000044686B00020FEF76DFB224E012758B130
:1072C000214A18212046F7F7CBF9020036D0308842
:1072D0001EA107EB00402FE0182227496846F5F76A
:1072E000C9F82648264D4FF00408006DA968884269
:1072F00011D1318808EB014022A1FEF79FFED5E9AC
:107300000101FCF761FF8DF80100FAF737FA8DF8FB
:107310000100254D02E08DF801700025D4E901122D
:107320006846904715B12846FCF782FC31889DF8E5
:10733000012008EB01401DA1FEF784FE06B0BDE868
:10734000F0810000E8010020AD720F004661696C19
:10735000656420746F207363686564756C65206F65
:10736000626A65637420657865637574653A203078
:107370007825782E000000001CA10F00BC1700200B
:1073800060000020506F737476616C696461746989
:107390006F6E206F66206669726D77617265206915
:1073A0006D6167652E00000055750F00526571759F
:1073B0006573742068616E646C696E6720636F6DBD
:1073C000706C6574652E20526573756C743A20304C
:1073D00078257800F8B50C4D0C46042628880BA1BA
:1073E00006EB0040FEF72AFE124813A1826CA26051
:1073F000036DB0026360E0600090288806EB0040F7
:10740000FEF72FFEF8BD0000E801002048616E6421
:107410006C65204E52465F4446555F4F505F4F4269
:107420004A4543545F53454C454354202864617496
:1074300061290000BC170020637263203D20307872
:1074400025782C206F6666736574203D2030782582
:10745000782C206D61785F73697A65203D203078E3
:10746000257800002DE9F041264F05460E46388864
:10747000042101EB004024A1FEF7E0FDFCF79EFE95
:1074800098B12B4CD4E91401401AA98A0844616CC4
:1074900088420CD93888012101EB004025A1FEF774
:1074A000CDFD03207070BDE8F0810820FAE7274980
:1074B000206B49684718E86820B925494FF4E07007
:1074C000F8F7EAFAD5E90331AA8A3846FBF7D0FF84
:1074D00020B1D5E90310BDE8F0410847A98A206B27
:1074E000134A08442063A98A206D48320844206565
:1074F000A98A2869F9F7B6FAA064B060206D7060B7
:10750000D1E70000E801002048616E646C65204E00
:1075100052465F4446555F4F505F4F424A45435481
:107520005F57524954452028646174612900000066
:10753000BC17002057726974652072657175657398
:107540007420746F6F206C6F6E6700006000002005
:1075500000A70F00074810B50088042101EB004088
:1075600005A1FEF76BFD11490620C968BDE8104072
:1075700008470000E8010020416C6C20666C6173D4
:1075800068206F7065726174696F6E7320686176D0
:107590006520636F6D706C657465642E204446557C
:1075A00020636F6D706C657465642E006000002050
:1075B000FEF712FEFEF7E2FB0028FBD10D4E64251C
:1075C0004FF47A47741C3846A0476D1EFAD10A481A
:1075D0000068C00700D000BEBFF34F8F0648E438F4
:1075E0000168064A01F4E06111430160BFF34F8F67
:1075F00000BFFDE7809F0F00F0ED00E00400FA05FA
:107600002DE9F0472F4F05464FF0040938880C4606
:107610004E4609EB00402CA1FEF710FD38882A7C6D
:1076200006EB004031A1FEF70DFD4FF44051374B02
:107630004A6801204FF002089A4200D10220344EDD
:10764000326A012A00D1401C4FF0010C84F801C0BD
:107650002A7C1AB10025012A09D01BE084F8048095
:10766000F068A0602B48E060C0F57E200FE0D1F804
:10767000048098450ED125710878142801D94869ED
:1076800000E00020A0604FF48050E0608868206136
:10769000BDE8F087824208D284F804C0B068A060D8
:1076A000FBF784FBE060B069F1E7398809EB014042
:1076B00019A1FEF7C3FCFF202071A560E5602561DC
:1076C000E6E70000E801002048616E646C65204E2A
:1076D00052465F4446555F4F505F4649524D5741B1
:1076E00052455F56455253494F4E00004669726DF0
:1076F0007761726520696D61676520726571756576
:10770000737465643A20256400000000DBE5B15124
:10771000BC17002000C00E004E6F207375636820F8
:107720006669726D7761726520696D6167650000D9
:107730002DE9F0471646894682460024DFF860802E
:10774000184F21E019F80410154801F075FCD0B964
:107750001548FCF763FBD8E901125046FCF72CF9F9
:107760001248FAF779FC0500388811D0042101EBA2
:1077700000402A460EA1FEF765FC0021ED1CC8E979
:10778000015188F80010641CB442DBD3BDE8F087D7
:10779000BDE8F047012101EB00400AA1FEF74EBC15
:1077A000908A002038020020A8AE0F0098AF0F008A
:1077B000416C6C6F636174656420627566666572A6
:1077C000202578004661696C656420746F20616CC7
:1077D0006C6F636174652062756666657221000076
:1077E000011F0148FAF79ABC98AF0F00F8B50D4693
:1077F00014460646694600F052FA00280ED0009A58
:10780000FF2A0AD8501C824207D869780223B3EBBA
:10781000911F02D02979814201D20020F8BD227047
:10782000611C304600F080FBF8BD114600F0D6B870
:10783000114600F0E3B8F8B50C4615460646694611
:1078400000F02DFA00280CD0009A501C904207D36B
:1078500061780223B3EB911F02D02179814201D2DA
:107860000020F8BD2946304600F05EFB009A00215A
:10787000A954F8BD2DE9FF410C468E681746054610
:10788000694600F023FB00280ED0A06800280BD02A
:1078900060783A46C0F3011002283146684606D0A7
:1078A00000F0DAF80199696004B0BDE8F08100F0F9
:1078B00086F8F7E77CB50D461446694600F08FF967
:1078C000002820D02879082806D0042809D00228CA
:1078D0000AD001280CD015E0DDE90001C4E900015F
:1078E0000AE00098206006E0009800B2208002E0E4
:1078F000009840B22070C117DDE900235040594084
:10790000084301D000207CBD01207CBD7CB50D4624
:107910001446694600F09EF9002820D028790828EE
:1079200007D00021042809D002280AD001280CD051
:1079300014E0DDE90001C4E9000109E000982060DD
:1079400006E0009880B2208002E00098C0B220706B
:10795000DDE9002350405940084301D000207CBDA0
:1079600001207CBD7CB50D461446694600F072F9D5
:10797000002821D02979082908D00098C2170429A5
:107980000BD002290DD001290ED014E0DDE9000250
:10799000C4E900020146134609E0C317014620600E
:1079A00005E001B2218001E041B22170CB174140D6
:1079B0005340194301D000207CBD01207CBD70B52F
:1079C0000D46064614461146284600F09AFA22460D
:1079D00029463046BDE8704000F03EB838B50C4648
:1079E0000422694600F0A0FA002806D09DF8031092
:1079F000009861F31F602060012038BD1CB50C4663
:107A00000822694600F090FA002824D09DF8011061
:107A10009DF800209DF80230080E42EA012242EA59
:107A2000034240EA13409DF803309DF8041040EAF9
:107A3000132008439DF8051042EA036240EA012042
:107A40009DF8061040EA01409DF8071040EA0160E9
:107A5000C4E9002001201CBD2DE9F04F04469DB073
:107A600000200090064601904FF0FF3A0AA800F06F
:107A700069F94FF0010BE94682E012AB05AA06A9AD
:107A8000204600F0C9F850B10AA8059900F06BF93A
:107A900060B10B98407810F0300F53D060E09DF843
:107AA0004800002870D11DB0BDE8F08F0598B042A5
:107AB00042D30B9D0AAE0B98407800F00F000828C7
:107AC00012D0304600F066F90B98A842F3D1564622
:107AD0000599B14230D3D4F8088009919DF8181067
:107AE00008910E990D6820E00B980678F0E7296858
:107AF0000F682FB1DDE9083229462046B84711E06A
:107B000011948968DDE90872097891420CD12946FF
:107B100017A8FAF71EF985F80CB017AA394611987C
:107B2000F9F727F80028BED0AD6815B1A168414526
:107B3000DDD0A168414523D19DF81810204600F002
:107B40002FFA1BE00C9840280AD200F01F010BFA14
:107B500001F00C994A0959F82230034349F82230C0
:107B6000E5682DB10AAB9DF8182020460599A84775
:107B70000AAA9DF818102046F8F7FBFF002892D0BB
:107B8000A06800287FF479AFDDE90B0445780AA8E6
:107B900000F000F90028F7D115F0300F03D10B9851
:107BA000007800B1641CC4B10020494605E000BF64
:107BB00051F82020521C0ED1401CB0EB541FF7D3BB
:107BC000600959F8201004F01F00C0F120022AFAC1
:107BD00002F0814201D0002065E7012063E71CB577
:107BE0000C46694600F036F8002814D0DDE90002A2
:107BF000C10709D051084FEA30006FEA00026FEA6E
:107C00000100C4E9002004E051084FEA3000C4E953
:107C100000014FF001001CBDF8B5074600201870A8
:107C200008700E4610601C4615466946384600F03E
:107C300036F8012140B1009850B1C10800F00700AA
:107C4000296030700120F8BDB86808B10020F8BD87
:107C50002170FBE72DE9F84300268846814634462B
:107C6000354604E0402E02D30020BDE8F883694683
:107C7000484600F085F90028F7D09DF8007032469C
:107C800007F07F00C10FF4F7E2FB29430443F61D20
:107C90000D463806E6D4C8E900410120E5E7F8B50D
:107CA0000E460746694600F06BF900280AD09DF899
:107CB0000040200616D5072504F07F0403E0202DA0
:107CC00001D30020F8BD6946384600F059F9002874
:107CD000F8D09DF8001001F07F00A8400443ED1D8E
:107CE0000806ECD401203460F8BD000059680A4A47
:107CF000896891420ED1D0E901120848491C521EF0
:107D0000C0E9011206480421008801EB004005A1EA
:107D1000FEF798B9704700000CA00F00700000201B
:107D2000F001002050423A20496E6974207061636E
:107D30006B65742064617461206C656E3A20256403
:107D400000000000C26000230160C0E901138B78CD
:107D50001A44026191F903301A44426108780028FC
:107D600000D00120704770B545680E460446606833
:107D70000178B14206D1407800F00F00082801D008
:107D8000012070BD204600F005F86068A842EED1E1
:107D9000002070BD30B541680A785AB101F10C037A
:107DA00043600A7B42B14C780A79C4F30115032D74
:107DB00007D00BE0002030BDC2680168FFF7C2FFAA
:107DC000F8E75D78C5F30115032D07D00225B5EB63
:107DD000141F09D14C7914FB02F209E08D78046973
:107DE0000022641B046103E0B5EB941F00D1042260
:107DF000497811F0300F02D18168491C81609C786C
:107E0000016921441144016193F903201144416146
:107E1000012030BD30B54168002487B0497801F0B9
:107E20000F02082A11D08A091ED00222B2EB911F3C
:107E300009D10269C1F301110229146001D003299B
:107E400001D14069047007B030BD0069056808E0E1
:107E50002C7329466846F9F77CFF6846FFF7DAFF7E
:107E6000AD68002DF4D1EEE7C1F30111012912D064
:107E70000229E6D00329E4D04268517801F00F01CD
:107E800007290BD0916881B11279006907B0BDE86C
:107E90003040F4F7EFBA41690C70EDE70169906882
:107EA00007B0BDE8304000F02CB81179006907B088
:107EB000BDE83040F4F706BB10B5034B002408C002
:107EC00080E8160010BD000009FE0E0038B50D4612
:107ED00004466946FFF7E3FE00280BD0D4E9000210
:107EE000D4E90213C5E90002C5E9021300988142F2
:107EF00001D2002038BDA860A168081AA060012046
:107F000038BD00B50A4687B001466846FFF71AFF3C
:107F1000002807D06846FFF77DFF6846FFF73AFF65
:107F20000028F7D107B000BD7FB514460546A9B9B2
:107F3000124A2868904208D110E01022694628466B
:107F4000FFF7F2FF002807D0103C102CF5D822468E
:107F500069462846FFF7E8FF04B070BDA868A04254
:107F600001D20020F8E72B682246284698470028CF
:107F7000F2D0A868001BA8600120EDE709FE0E0002
:107F800010B504468068002809D0236801222046E5
:107F90009847002803D0A068401EA060012010BDB3
:107FA00038B5002439B1012912D0022912D005298F
:107FB0001DD0002038BD0546012269462846FFF73E
:107FC000B3FF90B19DF800000006F5D4012038BD44
:107FD00008220DE005466946FFF761FE28B1002141
:107FE0002846009AFFF7A0FF38BD204638BD04227E
:107FF000BDE838400021FFF797BF000010B50C46E0
:10800000017A052908D0407A38B1084808A10268E9
:108010002046FDF799FA00E01AB106A12046FDF7C7
:1080200093FA2046BDE81040FDF7CCBA8C01002041
:10803000257300000D0A00002DE9F047254D9946F3
:108040001646044699B3254F09F50051DFF888809C
:1080500001233A88D1F804C0A06D03EB0242C44565
:1080600002D010461E490BE08B68411EC1F30B0184
:10807000401A41F6FF710844834206D2104619495E
:10808000FDF7DCFF0020BDE8F0874846F9F7F0FD7A
:1080900050B13888022101EB00401349FDF7CEFFB3
:1080A0000C481830FAF7A8FE16B1AC2001E004E045
:1080B000A520E862A06D686301E0AA20E8623EB1F5
:1080C00094F88F0010B194F8900008B96068E860E7
:1080D0000120D8E7BC170020DBE5B151F0010020FA
:1080E000FCA70F0090A70F0050A80F0038B5C38859
:1080F0000D46044633B114A0009015A216A12846DF
:10810000FDF722FA217A05291CD0607A48B1A088AF
:10811000FDF706FE164951F8202016A12846FDF766
:1081200013FAA0880021FEF749F803461049207A87
:10813000143951F8202001B02846BDE830400EA186
:10814000FDF702BA38BD00001B5B306D0000000077
:108150001B5B313B33316D0025734C6F67732064BB
:10816000726F70706564202825642925730D0A00DC
:108170008C010020257300003C25733E2025733AB6
:1081800020000000EFF30580C005C00D01D00120E4
:108190007047EFF3148040F30000401C704710B5A7
:1081A00010461A46F4F766F9002010BD2DE9F0419B
:1081B0001E681C461546074621B1012918D005291D
:1081C00023D119E000202060401C2060B0421CD860
:1081D000012229463846FFF7A7FE002806D015F8E9
:1081E000010B000601D52068EEE70120BDE8F08113
:1081F00008200246186002E0042002461860294662
:108200003846BDE8F041FFF78FBE0020EEE70000E2
:108210002DE9F0474A4F0D464B780A788046398859
:108220000469042000EB014046A1FDF712FF602025
:108230002070287860706878A070687803264FF006
:108240000109012802D00B2870D059E028780C28A9
:108250004ED2DFE800F0064D4D354D4D3B644D06E6
:1082600009242879E07067E0E11C686801F026F9CC
:10827000C01CC6B2A119A86801F020F93044C6B2EA
:10828000A119E86801F01AF93044C6B2A1192869A9
:1082900001F014F93044C6B2A119686924E02879C4
:1082A000E070211DA86801F009F9001DC6B2A119EE
:1082B000E86801F003F93044C6B2A119286913E057
:1082C000E11C686801F0FAF8C01C0AE0E11CE868EB
:1082D00001F0F4F8C01CC6B2A119686801F0EEF80C
:1082E0003044C6B2A119A86801F0E8F83044C6B21B
:1082F000182E05D9398809EB01401BA1FDF79EFE18
:10830000D8F80420314620469047002816D03988F6
:1083100009EB0140BDE8F0471CA1FDF78FBEA9881D
:10832000E170090A21710526EAE7FFE7F9F72EFA5D
:10833000E0700020F9F732FA0426E1E7BDE8F087A3
:108340003402002053656E64696E67205265737055
:108350006F6E73653A205B3078253031782C203091
:1083600078253031785D00004D6573736167652055
:108370006973206C6172676572207468616E206534
:10838000787065637465642E000000004661696C56
:10839000656420746F2073656E642064617461206D
:1083A0006F7665722073657269616C20696E7465A1
:1083B00072666163652100000846704738B50C4657
:1083C000050003D10A496D20F7F766FB1CB908497F
:1083D0006E20F7F761FB6B4622462946054800F000
:1083E00062FE04490448009AF6F71AFB38BD000003
:1083F00098AB0F00A08A002030A40F002DE9F041B7
:108400008046F8F78AFE1A4D0026F0B1686828B158
:1084100068684068696820F07F40486000F06EFE40
:10842000040012D04FF080776068B84203D2204633
:1084300000F046FF03E0606820F07F406060204667
:10844000FEF720F808B10446EEE700214046F8F7B1
:1084500089FD28B1686818B1686800F031FF6E6066
:10846000404600F091FF4046BDE8F04100F002B800
:10847000C80000202DE9F041214C0746002600BF2E
:1084800000F03CFE90B341686068406862685AB191
:108490006268002A28D0884226D96068007E18B118
:1084A00061681848FDF7B4FF00F02EFE42680546EB
:1084B00013484FF47A7300210830F8F74FFE30B1BB
:1084C0000D2807D010499C20F7F7E6FAD8E7606836
:1084D00020B106E0284600F0F3FED1E73846F8F771
:1084E00021FE6560002ECBD1BDE8F081FFE760681A
:1084F0000028F9D13846BDE8F041F8F721BE000068
:10850000C80000204CA20F0028A90F002DE9F05F41
:10851000FBF780FCDFF8CC80334D0427D8F83020FF
:10852000D8F8346000EB020BB01A411EC1F30B0106
:10853000401A00F6FF7A28882CA107EB0040D8F8F3
:108540004840FDF77BFD42F20400324900594FF0EC
:108550000109884208D0298809EB01402EA1FDF7C6
:108560006DFD0320BDE8F09FD8F830000444B04210
:1085700007D1288835A107EB0040FDF75FFD0020FB
:10858000F0E7D0B904F500500178142901D9406909
:1085900000E000203249B0FBF1F34FF44050027884
:1085A000142A01D9406900E00020B0FBF1F22888CC
:1085B0002CA107EB0040FDF74CFD08235246214655
:1085C0005846F9F7DBF9040007D0298809EB014088
:1085D0002FA1FDF733FD2046C4E7BDE8F05F002082
:1085E000FBF726BBBC17002030020020456E7465E7
:1085F00072206E72665F626F6F746C6F6164657219
:108600005F6466755F73645F636F6E74696E7565D2
:1086100000000000DBE5B151536F757263652061A6
:1086200064647265737320646F6573206E6F742069
:10863000636F6E7461696E20612076616C6964207D
:10864000536F66744465766963652E0053442061F8
:108650006C726561647920636F7069656400000005
:1086600040420F005570646174696E672053442E58
:10867000204F6C64205344207665723A2025642C88
:10868000204E6577207665723A2025640000000050
:108690004661696C656420746F20636F7079206631
:1086A00069726D776172652E0000000070B50F4C25
:1086B0000421208801EB00400DA1FDF7BFFCFFF76E
:1086C00025FF05004FF0010604D0208810A106EB1D
:1086D000004007E0F7F7F4F9050006D0208812A162
:1086E00006EB0040FDF7AAFC284670BD30020020D2
:1086F000456E746572206E72665F6466755F736442
:108700005F626C5F636F6E74696E75650000000078
:1087100053442B424C3A20534420636F70792066B7
:1087200061696C656400000053442B424C3A20425E
:108730004C20636F7079206661696C65640000008D
:1087400070B50346002002464FF4405409E000BFD4
:1087500053F82250A689B54201D1012070BD521CA8
:10876000D2B28A42F4D370BD10B5040003D11549CA
:108770003220F7F791F94FF440501349406888428E
:1087800015D1217C04F1140009B162694AB994F849
:10879000552012B1012A08D10DE0012905D96269DD
:1087A0001AB9BDE81040FFF7CBBF012010BD207CF7
:1087B00018B1606908B1002010BD20780028F4D1FC
:1087C00010BD0000DCA80F00DBE5B1512DE9F04140
:1087D0001400884618D000250E4F032608EB05012B
:1087E00022460020F5F74CF90544241A40B93878A0
:1087F000002809D008494FF47A408847761E05D0F2
:1088000001203870002CE9D1BDE8F08100203870DB
:10881000FAE700005001002011A40F00002070476B
:108820002DE9FE4308790C46012804D0022805D022
:10883000032872D172E01222404977E0B4F80700B1
:10884000092800D90920814609264FF00008F6F7CB
:10885000F1F925E0686820B939A140F29720F7F7CF
:108860001BF96868406820B935A14FF42670F7F706
:1088700013F90027009700E07F1C6868012300229D
:10888000D0F804C029466846E0470028F4D1297A88
:108890003E4401EB080000F0FF082846F6F7A6FA70
:1088A0000500D7D102A8F6F735FC0299054689459F
:1088B00004D923A140F2AD20F7F7EEF81F494A464C
:1088C00012312846F3F7D6FD85F804806E80F6F75E
:1088D000B3FA18B1E87940F02000E871F6F7AAF988
:1088E0000146264880E82202B4F80710C160002043
:1088F000F7F764F8114980200839F6F797FC04006F
:1089000005D10E4980201039F6F760FB044600209F
:10891000F7F782F82046BDE8FE830DE0E078B4F872
:108920000510F7F71DF8010006D00A7803B0601CA7
:10893000BDE8F043F6F7BEBB0620ECE7E4A20F006B
:108940002E2E5C2E2E5C2E2E5C2E2E5C2E2E5C632C
:108950006F6D706F6E656E74735C6C69627261725C
:108960006965735C757362645C6170705F75736276
:10897000645F636F72652E63000000000C200020AE
:1089800038B50D466846F6F7C5FB04460098022840
:1089900004D20CA140F26F20F7F77EF8002020806F
:1089A0002078174940F00100207049784908C9072C
:1089B00002D040F00200207002222146681CF6F727
:1089C00079FB38BD2E2E5C2E2E5C2E2E5C2E2E5C5E
:1089D0002E2E5C636F6D706F6E656E74735C6C6968
:1089E000627261726965735C757362645C617070F8
:1089F0005F757362645F636F72652E6300000000D1
:108A000010010020F8B50C46070004D142A140F245
:108A10002930F7F741F824B93FA140F22A30F7F79F
:108A20003BF8607810F0600F2AD10006494DA0781D
:108A30004FF0000626D520B1062808D008281FD1FF
:108A40000BE021463846BDE8F840FFF799BF2146C4
:108A50003846BDE8F840FFF7E3BE6846F6F75AFB34
:108A600001462878052802D0042803D008E0012018
:108A7000087000E00E700122601CF6F71BFBF8BDC9
:108A80000620F8BD0A28FBD2DFE800F0051E05131A
:108A900005060505052DF3E72878032803D00428EB
:108AA00001D0052824D1F5F7F1FE042000F0C8FE1E
:108AB00015E0B4F803000128E2D1F6F7BDF980B162
:108AC000687840F0020009E0B4F803000128D7D12B
:108AD000F6F7B2F928B1687820F00200687000203B
:108AE000F8BD0F20F8BD2878052803D0042801D050
:108AF0000820F8BDE07818B1012805D00720F8BD9E
:108B0000F5F7C4FE042002E0F5F7D8FE052000F0DA
:108B100097FE3046F8BD00002E2E5C2E2E5C2E2EC9
:108B20005C2E2E5C2E2E5C636F6D706F6E656E74A6
:108B3000735C6C69627261726965735C757362649F
:108B40005C6170705F757362645F636F72652E63E2
:108B50000000000010010020F8B50546407810F034
:108B6000600F31D120486C79A978007821B10129B2
:108B700023D0032928D111E0052801D0200729D1CD
:108B80006846F6F7C7FA06462046FBF7F9FF30803D
:108B900002223146681CF6F78DFAF8BD04F00F0189
:108BA000082911D2B5F8031071B9052801D02007A2
:108BB00010D12046FBF7CAFF14E004F00F0108298A
:108BC00002D2B5F8031009B10620F8BD052803D07C
:108BD000200701D00820F8BD2046FBF791FE204673
:108BE000FBF7E6FF0020F8BD10010020FEB50C46A3
:108BF000050004D12F494FF4D170F6F74DFF24B989
:108C00002C4940F2A310F6F747FF60784FF00606B4
:108C1000010642D5C0F3411111B1012924D125E04B
:108C200000F01F0001281FD1A07806281CD10020C9
:108C3000019002A8F6F76EFA064601A80090E278C5
:108C4000217933462846F5F795FF05280CD0019881
:108C5000402803D31749A320F6F71EFF3146601CB6
:108C6000019AF6F727FAFEBD0620FEBD2846F7F763
:108C700091FDF7F7E1F9A178212903D1B4F80710A4
:108C8000072901D03046FEBD072200F10C0103B0D8
:108C9000601CBDE8F040F6F70DBAC0F341100028A3
:108CA000F0D00128E0D103B021462846BDE8F040CD
:108CB00000F046B86CA90F00F8B50B46517806468F
:108CC000144611F0600F25D11C480906A1780078E0
:108CD0001ED511B10A291DD109E005281ED168460B
:108CE000F6F718FA01460020088002220CE0052859
:108CF00014D16846F6F70EFA054619463046F6F7DF
:108D0000EDFC287001222946601CF6F7D3F9F8BD66
:108D10000B2901D00620F8BD052801D00820F8BD98
:108D2000B4F80300FF2801D90720F8BDD27819460E
:108D30003046BDE8F840F6F7A3BC00001001002063
:108D4000F0B585B00D460746F7F724FDF7F774F93F
:108D50000446A8780026202802D022282FD12BE014
:108D6000B5F8070007282AD13846F7F713FD04465F
:108D7000F7F762F9A9780170E9794170811C0196D1
:108D800002960091407801900020F6F717FE6946A0
:108D90000020F6F795FA050008D11D4803A90068E0
:108DA000CDE903040020F6F711F905460020F6F797
:108DB00033FE284605B0F0BDB5F8070008B106201F
:108DC000F8E7207DB5F8031000F0010001F001057F
:108DD000A182A8421AD00DB1022100E00321384639
:108DE00001F026F895B93846F7F772FEFBF756FD05
:108DF0003846F7F776FEFBF751FDA6612662E66678
:108E00002667666704F12800A667A0660020D1E700
:108E1000A4A20F00FEB50F46464C202102912088E7
:108E20000325164605EB004043A1FDF707F946B1BF
:108E3000208805EB00406FB149A1FDF7FFF816202F
:108E4000FEBD2088022101EB00404BA1FDF7F6F8A2
:108E50001320FEBD4D4F4EA1BA68FDF7F3F802A9ED
:108E60005848CDE90001D7E901235749A0F58A7098
:108E7000F9F70CFE10B93278402A01D00A20FEBD65
:108E80005048711C4038F3F7F5FA20884FA105EBE4
:108E90000040FDF7D3F84B4840214038CDE90001B0
:108EA000A0F14801474AA0F5BC70029BF9F7B6FD56
:108EB0000200208836D0012101EB004048A1FDF7D7
:108EC000C1F82088042505EB00404EA1FDF7B6F857
:108ED00020883C4905EB004040224039FDF75AF814
:108EE00020884BA105EB0040FDF7A8F80298354912
:108EF00082B2208805EB0040FDF74CF8208846A19F
:108F000005EB0040FDF79AF82088402205EB004071
:108F10004449FDF73FF800BFFCF730FF0028FBD1C4
:108F20000520FEBD05EB00403FA1FDF787F80120BD
:108F3000FEBD0000F00100205369676E6174757218
:108F4000652072657175697265642E20436865637A
:108F50006B696E67207369676E61747572652E0048
:108F6000496E76616C6964207369676E61747572AD
:108F700065207479706500004E6F207369676E61BB
:108F80007475726520666F756E642E007000002027
:108F900043616C63756C6174696E6720696E697496
:108FA000207061636B657420686173682028696E46
:108FB0006974207061636B6574206C656E3A20255E
:108FC000642900004C1C0020CC9F0F00566572697C
:108FD0006679207369676E617475726500000000C0
:108FE0005369676E6174757265206661696C65644A
:108FF00020286572725F636F64653A203078257847
:10900000290000005369676E61747572653A00004B
:10901000486173683A0000005075626C6963204BC8
:1090200065793A003C9F0F00496D61676520766560
:10903000726966696564000030B528B1D0E9022321
:109040009A4203D1042030BD0E2030BD04782CB1EB
:109050000023012C10D0022C23D11EE0C02906D001
:10906000DB2906D04468531C8360A15419E000201A
:1090700030BD0121017014E0DC2905D0DD2905D0C7
:10908000022101700B2030BDC02400E0DB244568C4
:10909000511C8160AC54037003E0C02901D10370FE
:1090A0008360112030BDF0B528B121B11BB100247F
:1090B000DB261C6019E00E20F0BD0F5DC02F02D032
:1090C000DB2F0BD105E01D686F1C1F604655DC27A8
:1090D00004E01D686F1C1F604655DD271D68641C79
:1090E00005F1010CC3F800C047559442E5D3196857
:1090F000C0244A1C1A6044540020F0BD0148FDF70A
:10910000E9B900004CA20F000148FDF70BBA0000BE
:109110004CA20F002DE9F84FDFF89C80934689465A
:1091200006461F46012269461846D8F80850F6F749
:1091300027FEB0B3009800210446C246801C08E018
:1091400000EA05025BF821300AEB8202401C491C50
:10915000D360B942F4D3C846B946370CF7F7F8FEE6
:109160008346FDF721F8B84204D8144940F2831031
:10917000F6F792FC601C28400AEB80002C4047EA7E
:109180000B420AEB8401C260C86866F3C50069F34C
:10919000891068F39F2020F00300401C20F0040099
:1091A000C860074890F8200002E000BFFCF7E6FD29
:1091B0000028FBD1BDE8F88F4021002098AA0F00BD
:1091C000406100201FB5134800F15C01826B6846C6
:1091D000FEF772FE10489DE80E0080E80E000E4972
:1091E0000E48104AC8600E490020486088600E4949
:1091F0000948FEF7E4FB10B1012004B010BD0B4894
:109200000121008801EB004009A1FCF717FF0020B5
:10921000F3E70000BC170020B41B0020ED7C0F001A
:109220007000002018190020D8A00F00F0010020C5
:1092300048616E646C65723A20496E76616C69644F
:109240002070726F746F636F6C20627566666572F2
:10925000206D5F70625F73747265616D0000000065
:1092600070B50546F6F790FB124C06462078F6F7E7
:109270008BFB86420AD02846F6F786FB20B104F124
:109280000C00FBF731F901E0FBF7EEF82846F6F7A2
:1092900088FB06462078F6F784FB864208D02846ED
:1092A000F6F77FFB10B1FBF7B1F901E0FCF78AF8A4
:1092B000257070BDF0000020002800D000477047E6
:1092C00070B50446C06818B90F496120F6F7E4FB91
:1092D0000E4800250078A0B19CB1207E88B1D4E969
:1092E00003108847A06850B1217E41B161680844ED
:1092F000606021460648FDF78BF8012501E000205B
:109300002076284670BD000028A90F00C800002064
:109310004CA20F0070B5164C2078002827D11548B4
:1093200001680125C1F3004131B913490D6001689D
:10933000C1F300410029FAD0F5F73AFA08B1F5F780
:1093400073F90E4A00210E48F5F714FA18B10D49C9
:109350002E20F6F7A1FB0A48084A0121001DF5F767
:1093600009FA18B107493320F6F796FB257070BD4E
:10937000480000201804004008000040B9920F0087
:10938000B89F0F0008A50F002DE9F843244D814632
:1093900069462868F8F717FE044600274FF00108D1
:1093A000204E39E0207820B101281BD002282AD194
:1093B00022E06068017E31BB80F818804846F7F7EC
:1093C000D8FD014660684268511A174A914203D994
:1093D000416821F07F414160114861680830FDF724
:1093E00017F810E061687068814200D177600C481E
:1093F0000830FDF7C3F806E0FFF786FE08B10776F0
:10940000FAE786F8008069462868F8F7D1FD6946D2
:109410002868F8F7D8FD0446002CC3D1BDE8F883CE
:1094200044A20F00C800002017FCFF00F8B50B4C49
:109430000D46064669462068F8F7AFFD58B106703C
:10944000456069462068F8F7C9FD10B10448F7F790
:1094500053FE0020F8BD0420F8BD000044A20F0018
:10946000D000002070B515460C460646FFF752FFA7
:109470003046F5F7E7F918B10F494320F6F70CFB32
:10948000002C17D0610CE0034FF4FA72801841F100
:10949000000152000023F2F7A9FF01462A46304698
:1094A000F5F7ACF9002805D0BDE8704002494A2024
:1094B000F6F7F2BA70BD000008A50F000870020AA6
:1094C0004A70020C8A70000EC870042070470000B9
:1094D00010B50248F8F78DFD002010BD4C010020AA
:1094E0002DE9F05F8346DDE90A4A994690460D462C
:1094F0000846012703E000BFB0FBF8F07F1C4045A1
:10950000FAD2B94500D94F465FEACA7012D18CB180
:109510005FEA8A7002D5B9F1000F01D0202607E07A
:10952000302605E031465846641EF6F77BFC0CB148
:10953000A742F7D35FF00106B9F1010F02D9A9F1F3
:10954000010903E0B5FBF6F0404502D306FB08F63F
:10955000F2E7DFF83C9000BFB5FBF6F000FB1655D4
:1095600019F800105846F6F75DFCB6FBF8F6002E29
:10957000F2D15FEACA7009D0002C07D0A74205D209
:1095800020215846641EF6F74DFCF5E7BDE8F09F34
:10959000C6A30F0070B515460E46012400F0A2F8D0
:1095A000034600210A463046F9F730FC0B4E40B125
:1095B0003088012101EB004009A1FCF73FFD0424A4
:1095C0000AE0F9F709FC024628603088042101EB23
:1095D00000400AA1FCF736FD204670BDF0010020D6
:1095E00043616E27742066696E6420726F6F6D2010
:1095F000666F7220757064617465000057726974DB
:109600006520616464726573732073657420746F80
:1096100020307825303878002DE9F0410F240027DC
:1096200090F85520184E01251AB990F86430012B96
:1096300006D0D30707D090F85630012B02D002E0B5
:10964000876E0DE0876D92070AD590F85C20012A9D
:1096500006D1026E0D48C0F57E239A4204D8174405
:109660004FB101240F600CE0308809A105EB0040E8
:10967000FCF7EFFC042430880DA105EB0040FCF75B
:10968000DDFC2046BDE8F081F001002000C00E00A6
:10969000424C2073697A652028256429206F7665FD
:1096A00072206C696D69742028256429000000000F
:1096B000496E6974207061636B657420646F6573B3
:1096C000206E6F7420636F6E7461696E2076616CBA
:1096D0006964206669726D776172652073697A6565
:1096E00000000000017C19B1406908B101207047F9
:1096F0000020704702480068002800D00120704711
:10970000180100200020704770B504462B48F8F778
:1097100049FD2B4804602948F8F79EFC294C002895
:1097200043D02949C01C40F6030248600020C1E92B
:10973000020208702448254914380426416024494F
:10974000C0E9021200F13D010161208821A106EB70
:109750000040FCF773FCFAF717FF852801D00028BA
:1097600022D10020FAF730FF00281DD1F6F78CF83F
:109770001E48F5F7BDFF002816D11C482038F5F724
:1097800067F9002810D1208819A106EB0040FCF7EA
:1097900055FCF6F765F8051E06D1208818A106EBE2
:1097A0000040FCF74BFC284670BD2088012101EBEE
:1097B00000401AA1FCF742FC032070BD98AF0F00D7
:1097C000BC01002038020020908A0020BD830F00D9
:1097D000E1770F00496E697469616C697A696E6737
:1097E00020647269766572732E00000050A40F0029
:1097F0005374617274696E67205553420000000013
:10980000555342205472616E73706F727420696E8A
:10981000697469616C697A6564000000436F756CF6
:1098200064206E6F7420616C6C6F6361746520706E
:1098300061796C6F616420706F6F6C2E00000000A6
:1098400007490A78824209D00870052803D0487871
:1098500020F0020048700348F5F74CBD7047000047
:1098600010010020D0A20F002DE9FE4F804648686D
:1098700091464FF0010A0C4628B92068F5F7B6FA70
:1098800008B9A06890B1B9F1400F04D937A140F2EE
:109890007110F6F701F900260096FBF7EFFAE7687A
:1098A000834648464F4559D9074657E04FF0000ACE
:1098B000C8F800A0C8F804A054E0A068B84201D9D4
:1098C0003D4600E00546616839B10BEB06002A46CB
:1098D000F2F7D0FD002060600CE058B121680BEB7E
:1098E00006022B464868D0F804C004F11000E04797
:1098F00001200090A068A7EB0507411BA160E0686C
:109900002E44A0EB0500E06005D1009818B1206856
:10991000F5F76CFA2060E06810B1A068F0B902E0D9
:109920004FF0000A1AE0206800284FF0000001D034
:10993000019009E060609EB14E4511D24FF0000ADF
:109940000EE0A068401CA060216801230022486846
:10995000456801A8A8470028F3D12061002FACD1A9
:10996000C8E900B65046BDE8FE8F00002E2E5C2EE2
:109970002E5C2E2E5C2E2E5C2E2E5C636F6D706F17
:109980006E656E74735C6C69627261726965735C3A
:10999000757362645C6170705F757362645F636F3E
:1099A00072652E63000000001B4910B50322098870
:1099B0001A4C02EB0142082809D0092815D00A28C0
:1099C00020D00E2826D1BDE81040F5F7ABBB1046DD
:1099D00013A1FCF733FBFBF7BFFB08B9F5F7CAFB94
:1099E0002168002916D0012009E0104611A1FCF7DA
:1099F00025FBF5F7ABFF216800290BD00220BDE85D
:109A000010400847104610A1FCF718FBBDE81040B5
:109A1000F5F766BF10BD000038020020BC01002031
:109A200055534220706F7765722064657465637466
:109A30006564000055534220706F7765722072652F
:109A40006D6F766564000000555342207265616455
:109A5000790000000249002008600249C870704780
:109A60001C7C02408000002070B50446010600F016
:109A70000F0502D5092D09D301E0092D08D308A14E
:109A800040F28920F6F708F8200601D5042000E00E
:109A9000282000EB8500BDE87040FCF751BF0000B6
:109AA0002E2E5C2E2E5C2E2E5C2E2E5C2E2E5C63BB
:109AB0006F6D706F6E656E74735C647269766572DB
:109AC000735F6E72665C757362645C6E72665F640F
:109AD00072765F757362642E630000002DE9F04FAB
:109AE000514D89B0E878002846D180464FF00109F1
:109AF0003EE000BF90FAA0F0B0FA80F63046F5F7ED
:109B0000D6FF8346F7F7DEFB0446006820B947A17D
:109B100040F23150F5F7C0FF5FEA0B6007D5D4E99A
:109B20000031A28902A89847002836D037E058466D
:109B3000FBF760F9D4E9007182460346A28902A8C6
:109B4000B84707460298D0B1039951451DD202206B
:109B5000A07309FA06F0C14333480C30F8F75BFAFA
:109B60004148006B00908DF802B0696868468847EC
:109B7000D5E902100840BDD109B0BDE8F08F0398C7
:109B800050B12AA140F24D5004E0514504D027A124
:109B900040F25C50F5F780FF0FB9C4F800803349FC
:109BA0008220086085F80390A96809FA06F08143CD
:109BB000A960A06803990844A060DDE90212584634
:109BC000FCF716FDFBF744F918B3294C4FF48275E6
:109BD0002846FCF797FE5846FFF746FF0220FCF7A1
:109BE000BBFF2846FCF786FE0028F1D01E2000E0CF
:109BF0000220FCF7B1FF20688006F9D50120FCF7B0
:109C0000ABFF5846FAF7ECFFFCF774FE0028DFD0F4
:109C1000B2E75846FFF728FF5846FAF7E1FFFCF78E
:109C200069FE0028F8D0A7E7800000202E2E5C2EC9
:109C30002E5C2E2E5C2E2E5C2E2E5C636F6D706F54
:109C40006E656E74735C647269766572735F6E7252
:109C5000665C757362645C6E72665F6472765F7573
:109C60007362642E6300000060A10F001C7C024040
:109C7000747402402DE9F84307460020F5F79EFE74
:109C80003846F7F71FFB06463806294D4FF0000807
:109C90004FF003094FF0010438461ED4F7F7FCFAE1
:109CA000E96804FA00F0884303D03846FBF794FBD8
:109CB00010E03846C6F80080F7F7EEFAE96804FAD3
:109CC00000F081433846E960F7F7E6FA8440A86877
:109CD000A043A86086F80E9024E0F7F7DDFAD5E9F6
:109CE000022104FA00F061EA020108421AD0384663
:109CF000F7F7D2FAE96804FA00F081433846E960E0
:109D0000F7F7CAFA8440A8680443AC600948C6F86B
:109D1000008086F80E90006800908DF802706968E7
:109D200068468847BDE8F8430020F5F775BE000097
:109D30008000002060A10F002DE9F041104EB068B6
:109D4000040CF06824040443012712E094FAA4F000
:109D5000B0FA80F52846F5F7AAFE00F00F000828B3
:109D600004D22846F5F7A3FEFFF784FF07FA05F0B3
:109D70008443002CEAD140F2FF10B060BDE8F081CE
:109D800080000020012238B58A400C490C468B68BF
:109D900013438B606168E468094B050602EA04021C
:109DA00003D5002A09D19A6902E0002A05D1DA69AF
:109DB00000928DF802006846884738BD8000002078
:109DC00060A10F0010B5017879B10A4A0421F4F7B7
:109DD00047FC00280DD0084801210088BDE810404C
:109DE00001EB004005A1FCF729B9BDE81040F5F7EB
:109DF00081BA10BD2D9E0F0038020020436F756C94
:109E000064206E6F74207363686564756C6520559B
:109E10005342206576656E7421000000024980205F
:109E2000C1F800027047000004E000E0F5F762BAF4
:109E300070B50C460546F6F7ADFCC269002A04D0A1
:109E400021462846BDE87040104770BD0249496868
:109E5000002900D008477047C01F002030B10068BB
:109E60000549884205D048F20250704748F2015037
:109E700070470020704700006E52464870B5FCF7EE
:109E80006BFD002811D00020084A094B094C012124
:109E9000166801FA00F52E4203D004EB8005C5F8E0
:109EA0000036401CC0B20728F2D370BD080501403F
:109EB0003546526E00000140084810B54078002831
:109EC0000BD007480321008801EB004005A1FCF7F7
:109ED000B5F8BDE81040FFF7D1BF10BD4A00002023
:109EE000E0010020496E7465726E616C20666565E4
:109EF00064000000002070472DE9FC4180461C46AC
:109F000017460E460C48089DF8F77CF810B1112052
:109F1000BDE8FC81A20839463046FCF74DFA0648F8
:109F2000F8F767F833463A4601214046CDE9004547
:109F3000F7F7DEFB0020EBE74C01002065FC2BF877
:109F400016DA019ADE75D4A8477196211C875569E7
:109F5000105ABE04578FD2B0299456B8CA0363D69C
:109F600035C64DA7819FEFA7D2ECB7F307FF80AFAF
:109F70007A3B4C19B891C5143CE8766D000000009E
:109F80000338FDD870470D0E0F100B0C1819000088
:109F90000338FDD8704700000000000000000000FA
:109FA000000000000000000000000000FFFFFFFFB5
:109FB0000000000000000001100000202C00002024
:109FC00048000000002040000000000051FF0E008B
:109FD00061FF0E00FDFE0E002000000000000000EA
:109FE000000000000000000001010000010000006E
:109FF0000000000002050000210000000000000039
:10A00000000000000000000000000000011104FC3E
:10A010000400000000000000021104FC0400000025
:10A0200000000000032104FC0410000000000000F8
:10A03000041101FF0100000000000000051102FEF4
:10A040000400000000000000061104FC04000000F1
:10A0500000000000071104FC0400000000000000E4
:10A06000081701FF22000000E89F0F00091001FF00
:10A0700001000000E49F0F0000000000000000004D
:10A0800000000000011101FF0100000000000000BD
:10A09000021702FE940000000CA00F000000000058
:10A0A0000000000000000000010700009800000010
:10A0B00084A00F0002010000010000000000000069
:10A0C0000305000041000000000000000000000047
:10A0D0000000000000000000011704FC98000000D0
:10A0E00084A00F00021704FCDC000000A8A00F00F1
:10A0F000000000000000000000000000020000005E
:10A100000000000000000000000000000600000049
:10A11000000000000000000000000000040000003B
:10A12000000000000000000000000000000000002F
:10A13000000000000001000000000000000000001E
:10A14000000000000000000000000000000000000F
:10A1500000000000000000000000000000000000FF
:10A1600006000003010000000600000006000000D9
:10A1700006000000060000000600000006000001C6
:10A1800005000000020000000300000004000000C1
:10A1900006000002000000000000000000000000B7
:10A1A0000338FDD870470000D1160F000D160F00C0
:10A1B000A1130F00D5130F00DB130F00E1130F00E5
:10A1C000E7130F00ED130F00F3130F00F9130F0047
:10A1D0003D150F00FF130F0005140F0065140F004D
:10A1E0006B140F0071140F0077140F007D140F0013
:10A1F00083140F0089140F0091140F00D1150F0064
:10A2000011160F0059150F00DD140F0008010C0185
:10A210001001140118011C01200124012C0130013E
:10A22000340138013C014001440148014C01500116
:10A2300002030405060708090B0C0D0E0F1011127E
:10A2400013140000D80000200000070000000000E8
:10A25000EC000020530A0F00800000000B8100007A
:10A260008200000083000000840D0E030B0000003C
:10A270000C0008000000090000000A0000000000B7
:10A2800001F80E00F5F20E000000000000000000D2
:10A290005D000F00F5000F0000000000000000004E
:10A2A00000000000AD070F000000000009000F00D3
:10A2B0000000000009000F0000000000D5080F009A
:10A2C00000000000000000000A0000000000000084
:10A2D0000F0000001D880F000000000069980F00AB
:10A2E0000C200020120100020000004015191F522E
:10A2F00000010102030109020000000100C0FA0090
:10A3000049EE0E0000000000000000000000000008
:10A31000000000002001002000A30F000100020344
:10A3200000800000040309002A034E006F00720041
:10A330006400690063002000530065006D0069003F
:10A3400063006F006E0064007500630074006F00AE
:10A35000720056034E006F007200640069006300D3
:10A360002000530065006D00690063006F006E00FF
:10A3700064007500630074006F00720020005300D9
:10A38000650063007500720065002000440046000F
:10A390005500200042006F006F0074006C006F00D9
:10A3A00061006400650072000E03550073006500D3
:10A3B00072002000310000010203040000000000D0
:10A3C0000338FDD8704730313233343536373839B9
:10A3D00041424344454600000010000004000000D4
:10A3E00001000000511B0F00D1940F009F810F004E
:10A3F000F99E0F0059130F00B9830F00F59E0F004F
:10A40000611C0F00415C0F003F5C0F00395C0F00C6
:10A410000338FDD870470000000000000000000075
:10A42000DD0E0F0000000000000000000000000032
:10A43000EC71002090A20F000200010601020482CC
:10A44000810100000000010181000000F5080F00FB
:10A45000C59D0F00A9990F000000000065790F004D
:10A460000D790F00B5780F002B780F0031780F00B1
:10A47000ED770F0037780F0075780F0000000000AF
:10A480000040404040404040404041414141414007
:10A4900040404040404040404040404040404040BC
:10A4A000400502020202020202020202020202024B
:10A4B0000220202020202020202020020202020250
:10A4C00002029090909090901010101010101010A8
:10A4D00010101010101010101010101002020202B4
:10A4E00002028888888888880808080808080808F8
:10A4F00008080808080808080808080802020202F4
:10A500004000000081A40F002E2E5C2E2E5C2E2E0B
:10A510005C2E2E5C2E2E5C636F6D706F6E656E749C
:10A52000735C6C69627261726965735C626F6F748F
:10A530006C6F616465725C6E72665F626F6F746C83
:10A540006F616465725F6466755F74696D6572736F
:10A550002E6300002E2E5C2E2E5C2E2E5C2E2E5C8A
:10A560002E2E5C636F6D706F6E656E74735C6C69BC
:10A57000627261726965735C626F6F746C6F616443
:10A5800065725C6E72665F626F6F746C6F6164653A
:10A59000725F66775F61637469766174696F6E2E4E
:10A5A0006300000043524320636F6D7075746174E3
:10A5B000696F6E206661696C656420666F722063E6
:10A5C0006F70696564206170703A207372632063F4
:10A5D00072633A203078253038782C2072657320E9
:10A5E0006372633A20307825303878004120536F09
:10A5F000667444657669636520686173206A757363
:10A6000074206265656E2061637469766174656447
:10A610002E2049742773206C696B656C79207468EF
:10A62000617420616E206170706C69636174696F20
:10A630006E2077696C6C20636F6D6520696D6D6548
:10A6400064696174656C79006E72665F6673746FBD
:10A65000726167655F777269746528616464723DD1
:10A6600025702C207372633D25702C206C656E3D27
:10A670002564206279746573292C20717565756570
:10A680002075736167653A20256400004372656137
:10A6900074696E6720746865206F626A65637420F0
:10A6A000776974682073697A652030782530387846
:10A6B00020776F756C64206F766572666C6F77209B
:10A6C0006669726D776172652073697A652E204FB5
:10A6D0006666736574206973203078253038782079
:10A6E000616E64206669726D776172652073697A44
:10A6F00065206973203078253038782E00000000FE
:10A700002E2E5C2E2E5C2E2E5C2E2E5C2E2E5C634E
:10A710006F6D706F6E656E74735C6C69627261727E
:10A720006965735C626F6F746C6F616465725C64A1
:10A7300066755C6E72665F6466755F7265715F6890
:10A74000616E646C65722E63000000002E2E5C2E1C
:10A750002E5C2E2E5C2E2E5C2E2E5C636F6D706F29
:10A760006E656E74735C6C69627261726965735C4C
:10A77000626F6F746C6F616465725C6466755C6E49
:10A7800072665F6466755F7574696C732E63000032
:10A7900054686520536F66744465766963652073F9
:10A7A000697A6520696E2074686520696E666F201D
:10A7B00073747275637420697320746F6F20736D86
:10A7C000616C6C20636F6D70617265642077697471
:10A7D00068207468652073697A65207265706F728D
:10A7E00074656420696E2074686520696E697420E0
:10A7F000636F6D6D616E642E00000000546865200B
:10A80000536F667444657669636520646F65732071
:10A810006E6F7420636F6E7461696E20746865205A
:10A820006D61676963206E756D626572206964652C
:10A830006E74696679696E6720697420617320613E
:10A8400020536F66744465766963652E00000000CE
:10A85000496E76616C69646174696E6720617070BD
:10A86000206265636175736520697420697320696E
:10A870006E636F6D70617469626C6520776974686E
:10A880002074686520536F66744465766963652E2D
:10A89000000000002E2E5C2E2E5C2E2E5C2E2E5CD8
:10A8A0002E2E5C636F6D706F6E656E74735C6C6979
:10A8B000627261726965735C626F6F746C6F616400
:10A8C00065725C6466755C6E72665F6466755F7601
:10A8D000616C69646174696F6E2E63002E2E5C2E4C
:10A8E0002E5C2E2E5C2E2E5C2E2E5C636F6D706F98
:10A8F0006E656E74735C6C69627261726965735CBB
:10A90000626F6F746C6F616465725C6466755C6EB7
:10A9100072665F6466755F7665725F76616C6964A6
:10A920006174696F6E2E63002E2E5C2E2E5C2E2EAF
:10A930005C2E2E5C2E2E5C636F6D706F6E656E7478
:10A94000735C6C69627261726965735C74696D6570
:10A95000725C6578706572696D656E74616C5C615E
:10A9600070705F74696D6572322E63002E2E5C2EDE
:10A970002E5C2E2E5C2E2E5C2E2E5C636F6D706F07
:10A980006E656E74735C6C69627261726965735C2A
:10A99000757362645C636C6173735C6364635C6154
:10A9A000636D5C6170705F757362645F6364635F45
:10A9B00061636D2E630000002E2E5C2E2E5C2E2E09
:10A9C0005C2E2E5C2E2E5C636F6D706F6E656E74E8
:10A9D000735C6C69627261726965735C74696D65E0
:10A9E000725C6578706572696D656E74616C5C64CB
:10A9F00072765F7274632E63000000002E2E5C2E50
:10AA00002E5C2E2E5C2E2E5C2E2E5C636F6D706F76
:10AA10006E656E74735C6C69627261726965735C99
:10AA20006578706572696D656E74616C5F6D656D7A
:10AA30006F626A5C6E72665F6D656D6F626A2E63CF
:10AA4000000000002E2E5C2E2E5C2E2E5C2E2E5C26
:10AA50002E2E5C636F6D706F6E656E74735C6C69C7
:10AA6000627261726965735C6578706572696D6543
:10AA70006E74616C5F6C6F675C7372635C6E726640
:10AA80005F6C6F675F64656661756C745F6261635C
:10AA90006B656E64732E63002E2E5C2E2E5C2E2E44
:10AAA0005C2E2E5C2E2E5C636F6D706F6E656E7407
:10AAB000735C6C69627261726965735C65787065FC
:10AAC00072696D656E74616C5F6C6F675C737263E5
:10AAD0005C6E72665F6C6F675F66726F6E74656ED8
:10AAE000642E63007761726E696E670064656275DB
:10AAF000670000001B5B313B33306D001B5B306D2A
:10AB0000000000001B5B313B33316D001B5B313BB0
:10AB100033326D001B5B313B33336D001B5B313BCC
:10AB200033346D001B5B313B33356D001B5B313BB8
:10AB300033366D001B5B313B33376D00696E666FDA
:10AB4000000000006572726F720000002E2E5C2EF5
:10AB50002E5C2E2E5C2E2E5C2E2E5C636F6D706F25
:10AB60006E656E74735C6C69627261726965735C48
:10AB7000626F6F746C6F616465725C73657269613A
:10AB80006C5F6466755C6E72665F6466755F736544
:10AB90007269616C2E6300002E2E5C2E2E5C2E2EB0
:10ABA0005C2E2E5C2E2E5C636F6D706F6E656E7406
:10ABB000735C6C69627261726965735C626F6F74F9
:10ABC0006C6F616465725C73657269616C5F646609
:10ABD000755C6E72665F6466755F73657269616CE1
:10ABE0005F7573622E6300006170705F74696D65DC
:10ABF000722E6D5F6466755F696E616374697669F4
:10AC000074795F74696D6572000000006170705F37
:10AC100074696D65722E6D5F7764745F66656564D7
:10AC20005F74696D657200006E72665F626F6F744B
:10AC30006C6F616465725F77647400006E72665F4A
:10AC40006466755F666C6173680000006E72665FB3
:10AC50006466755F7265715F68616E646C657200D1
:10AC60006E72665F6466755F73657474696E677330
:10AC7000000000006E72665F6466755F76616C69E5
:10AC8000646174696F6E00006E72665F6466755F02
:10AC90007665725F76616C69646174696F6E0000DD
:10ACA000636C6F636B00000055534244000000006A
:10ACB000434C4F434B0000005052530055415254F7
:10ACC000450000006170705F74696D65720000007E
:10ACD00061746669666F2E6D5F7265715F66696625
:10ACE0006F0000006170705F7573626400000000A7
:10ACF0006364635F61636D006170705F757362644C
:10AD00005F636F72650000006D656D5F6D6E6772E9
:10AD1000000000006E72665F6673746F7261676533
:10AD200000000000736F72746C697374000000009F
:10AD300062616C6C6F632E6C6F675F6D656D706FB9
:10AD40006F6C0000617070006E72665F6466755FA4
:10AD500073657269616C00006E72665F6466755F30
:10AD600073657269616C5F757362000062616C6C1F
:10AD70006F632E6D5F7061796C6F61645F706F6F70
:10AD80006C0000000200000000000000E5D90E0089
:10AD900091D90E0067E6096A85AE67BB72F36E3C17
:10ADA0003AF54FA57F520E518C68059BABD9831F96
:10ADB00019CDE05BFFFFFFFFFFFFFFFFFFFFFFFF7E
:10ADC0000000000000000000000000000100000082
:10ADD000FFFFFFFFFCFFFFFFFFFFFFFFFFFFFFFF86
:10ADE0000000000000000000000000000100000062
:10ADF000FFFFFFFF512563FCC2CAB9F3849E17A76A
:10AE0000ADFAE6BCFFFFFFFFFFFFFFFF0000000001
:10AE1000FFFFFFFF0000000096C298D84539A1F45B
:10AE2000A033EB2D817D0377F240A463E5E6BCF807
:10AE300047422CE1F2D1176BF551BF376840B6CBD2
:10AE4000CE5E316B5733CE2B169E0F7C4AEBE78ECE
:10AE50009B7F1AFEE242E34FFFFFFFFF7F000000EF
:10AE6000800000000000000000000000FFFFFFFF66
:10AE70007F000000800000000000000000000000D3
:10AE8000B0AF0F00080000203802000058C50E00C7
:10AE900024B00F0040020020D8A8000014E00E00EB
:10AEA000C5FF0E00FDFF0E0009970F0005970F006C
:10AEB000E8AB0F00000000030CAC0F000000000323
:10AEC00028AC0F00000004043CAC0F000000040498
:10AED0004CAC0F000000040460AC0F000000040440
:10AEE00074AC0F000000040488AC0F0000000404E0
:10AEF000A0AC0F0000000000A8AC0F000000000094
:10AF0000B0AC0F0000000000B8AC0F000000000063
:10AF1000BCAC0F0000000000C4AC0F00000000003B
:10AF2000D0AC0F0000000003E4AC0F0000000000F4
:10AF3000F0AC0F0000000000F8AC0F0000000000B3
:10AF400008AD0F000000000014AD0F000000040465
:10AF500024AD0F000000000030AD0F000000000322
:10AF600044AD0F000000040448AD0F0000000404CD
:10AF700058AD0F00000004046CAD0F00000000038A
:10AF8000680100206001002068010020802000206E
:10AF90002C02002018000000B4010020B0010020A5
:10AFA000B3010020707200203C0200200408000061
:10AFB000011C13D8010218200A19DC1C410270017F
:10AFC00015100140110A1004170A1402A80425657F
:10AFD000F50E1424A30F1A28041A52041324201B5C
:10AFE00020A80801180B1804A41CC11444AB0F14AA
:10AFF000E4AA0F1A3C081AEC081AFC041AF4041A02
:10B0000004101A0C041A14041A1C041A24041A2C0E
:10B01000041A340401118490D0031B590D203A10F6
:04B02000EE016900D4
:020000041000EA
:0810140000C00E0000E00F0017
:00000001FF
